:020000040800F2
:100000000000022055F4000851F4000851F40008E3
:1000100051F4000851F4000851F4000800000000F9
:1000200000000000000000000000000051F4000883
:1000300051F400080000000051F4000851F40008D9
:1000400051F4000851F4000851F4000851F400087C
:1000500051F4000851F4000851F4000851F400086C
:1000600051F4000851F4000851F4000851F400085C
:1000700051F4000851F4000851F4000851F400084C
:1000800051F4000851F4000851F4000851F400083C
:1000900051F4000851F4000851F4000851F400082C
:1000A00051F4000851F4000851F4000851F400081C
:1000B000FD79000851F4000851F4000851F40008DB
:1000C00051F4000851F4000851F4000851F40008FC
:1000D00051F40008FDC20008A9C3000851F400084B
:1000E00051F4000851F4000851F4000851F40008DC
:1000F00051F4000851F4000851F4000851F40008CC
:1001000051F4000851F4000851F4000851F40008BB
:1001100051F4000851F4000851F4000851F40008AB
:1001200051F4000851F4000851F4000851F400089B
:1001300051F4000851F4000851F4000851F400088B
:1001400051F4000851F4000851F4000851F400087B
:1001500051F4000851F4000851F4000851F400086B
:1001600051F4000851F4000851F4000851F400085B
:1001700051F4000851F4000851F4000851F400084B
:1001800051F4000851F400080348044B834202D0A4
:10019000034B03B1184770479C0900209C090020BD
:1001A0000000000005480649091A891001EBD171C9
:1001B000491002D0034B03B1184770479C09002037
:1001C0009C0900200000000010B5064C237843B9BC
:1001D000FFF7DAFF044B13B10448AFF300800123AB
:1001E000237010BDA0090020000000001CAA040814
:1001F00008B5044B1BB104490448AFF30080BDE8C7
:100200000840CFE700000000A40900201CAA040851
:10021000A3F5803A704700BF154B002B08BF114B68
:100220009D46FFF7F5FF00218B460F461148124A05
:10023000121A10F081F90C4B002B00D098470B4B91
:10024000002B00D098470020002104000D000B482F
:1002500010F070F810F0A2F82000290008F072FBEE
:1002600010F06EF800000800000000000000000020
:1002700000000000A00900206C140120690301089F
:10028000F8B504460D4600F038FA294604F5987092
:1002900000F00AFC0023C4E9643304F5CC77A4F829
:1002A0008C3104F509713A4622F8023B8A42FBD1AF
:1002B0004FF0000204F50E76C4F82432A4F8283278
:1002C00084F82A22A4F82C32C4E98C3304F5227273
:1002D0003346002543F8045B9A42FBD14FF4807308
:1002E000A4F88832002384F89432A4F8AC3284F85D
:1002F000AE32C4F8B03284F8B432C4F88C52C4F8C8
:100300009052C4F89852C4F89C52C4F8A052C4F851
:10031000A452C4F8A8520B200FF0D6FF3023A4F843
:100320008C310D4BC4F894310723A4F82C320B4BBD
:10033000C4F82402C4F89071C4F83062C4F83432AE
:10034000C4F89852C4F89C52C4F8A052C4F8A452FD
:10035000C4F8A8522046F8BD040000206400002024
:1003600030B5B0F82822D0F824420346551CA05CD2
:10037000A3F82852A154B3F828220A2A84BF0022E5
:10038000A3F8282230BD90F82A3280F82A125B1A8E
:1003900058425841704738B5B0F8AC22052A044697
:1003A0000D4603D149B3012380F8AE32002DB4F8D5
:1003B000B03216BF80210021551C41EA5301B4F828
:1003C000B232A4F8B01218BFADB20133A4F8AC52E7
:1003D00094F8AE529BB2A4F8B2324DB37E2912D03B
:1003E000FE294FF000050CD1A4F82C5184F8B4522A
:1003F00084F8AE52A4F8B25203E084F8AE12A4F826
:10040000AC12284638BDB4F82C31102B04D9204644
:1004100000F08EF9054610B90025A4F82C510123EF
:1004200084F8B432002384F8AE32A4F8B232E8E79C
:1004300094F8B422012A04D0022AE2D1082BE0D198
:1004400004E0082BDDD1022384F8B432204600F00A
:1004500061F9CFE700F5987000F018BBD0EDA47AF1
:100460009FED0A7AF4EEC77AF1EE10FA05D801236F
:1004700080F8943290F894027047B0EE087AF4EE67
:10048000C77AF1EE10FAF5DB0023F1E79999193FED
:10049000D0F8A432C0F8A832D0F8A032C0F8A43204
:1004A000D0F89C32C0F8A0321249D0F89832C0F887
:1004B0009C3280EDA60A00F5277300F52B72B3EC91
:1004C000017AF1EC016AD0EDA67AE6EEC77A9342A2
:1004D000C0EDA67AF3D1084B9FED080A00F526700F
:1004E000F0EC017AB3EC017A9042A7EE270AF7D13B
:1004F000704700BF5C0B01086C0B01080000000096
:1005000010B52DED028B90F8882290F88932D0ED4D
:10051000A37A8A4282B00446B2EE047A01D1102B4B
:1005200046D9F4EEC77AF1EE10FAC4BFB3EE047AFE
:1005300077EEC77A9FED2C8AC8BFC4EDA37A07EE89
:10054000903AD4EDA36A84F88812F8EE677A102BFB
:1005500086EEA77A4FF0010301AA694604F50B70F5
:10056000B1EE040A88BFB0EE408A8DED007A0FF03C
:100570002DFB9DED000AB5EEC00AF1EE10FA4CBF5E
:1005800038EE400A30EE080A2046FFF781FFD4ED2E
:10059000A37ADDED016A84EDA40AB6EE007AE6EEF8
:1005A000C77A012384F88932C4EDA37A00200EE0D3
:1005B000F4EEC77AF1EE10FAF8DDB3EE047A77EED6
:1005C000C77A0133C0EDA37A80F889320120D4EDD7
:1005D000A37AB7EE007A77EE877AC4EDA37A02B0F9
:1005E000BDEC028B10BD00BF000000002DE9F04FF4
:1005F00085B00DF10409054617461E464A460223FA
:1006000000F5987000F040FA4FF0000A0DF108086C
:10061000574511D039F81A40E443C4F3C034214699
:100620002846FFF79DFE6040C0B24000013828F820
:100630001A000AF1010AEBE70DF10C0A4146022308
:10064000524605F5C6700FF065F94FF00008C14637
:10065000C346B8452FD03AF81840E443C4F3C03439
:1006600021462846FFF74CFF60B195F82A1285F81D
:100670002A420B1B594259412846B9F1000F04D0B8
:10068000FFF789FE08F10108E3E7FFF784FE8146E2
:100690000028F7D04FF49672294630460FF0B2FE8C
:1006A000B5F82C31A6F82C31B5F82E31A6F82E313C
:1006B000A5F82CB1E6E7484605B0BDE8F08F30B5A7
:1006C0000023044600F5967504F8013BAC42FBD1CB
:1006D000A0F82C31A0F82E3100239CB2A2420BD9F5
:1006E000B3F5957F08D0B0F82C41651CA0F82C51CB
:1006F000CD5C05550133F0E730BD024600F596713B
:10070000002302F8013B9142FBD1A0F82C31A0F864
:100710002E317047B0F82C31B3F5967F1FBF5A1CAD
:10072000A0F82C21C154012008BF00207047000010
:1007300070B5B0F82C11124E4FF0FF338C1E002212
:10074000551C92B2944209D9825C5A40D2B2C3F38A
:10075000072336F8122053402A46F1E7DB439BB2C9
:10076000045DDAB2944209D1014411F8012CB2EBD4
:10077000132F03D1A0F82E31012070BD0020FCE71B
:10078000800B0108B0F82C2170B50F4D4FF0FF33EE
:1007900004461618B44209D014F8011B5940C9B2D6
:1007A000C3F3072335F811104B40F3E7DB439BB24B
:1007B000A0F82E31911C8354013292B2C3F3072367
:1007C000A0F82C11835470BD800B010870B5002572
:1007D00000F10C0604460580C0E9015500F5A6733A
:1007E000304620F8025B9842FBD10321FFF748FD19
:1007F000062104F20440FFF743FD092104F2BC6026
:10080000FFF73EFD822323800B4BA3601E23C4F819
:100810007C390A4BC4F884394BF24033A4F8883948
:100820000F23A4F874596660C4F87859C4F8805945
:1008300084F88A39204670BD8000002080000001C5
:1008400090F8860970472DE9F041CEB20F46F11EAF
:10085000054649B200F5A67014469846FFF7FAFD22
:10086000394605F20440FFF7F5FDC4EB0414F11C12
:1008700049B205F2BC602401FFF7ECFDC5F87C49E4
:1008800085F88489BDE8F08190F88A1990F8883954
:1008900090F887294B40534090F8892980F888398F
:1008A0001A44D2B280F8892901EB5202534080F8F1
:1008B0008A39704790F8873990F88A1990F8882912
:1008C00001334A40DBB280F88739534090F88929D8
:1008D00080F888391A44D2B280F8892901EB520293
:1008E0005340DBB280F88A39184670472DE9F04151
:1008F0000446CEB09046022301AA0FF00BF8D4F8BC
:1009000078390133C4F8783902A804F5A677FFF7DF
:10091000F4FE02AB424601A93846FFF767FED0B1AC
:10092000BDF83631B4F874299A4203D1D4F8782945
:10093000022A0CD9BDF83421A4F87439023A0023F4
:10094000C4F8783992B202A94A480AF001FB4A4930
:1009500048480AF0B1FB04F2044602AB424601A942
:100960003046FFF743FED0B1BDF83631B4F87429F4
:100970009A4203D1D4F87829022A0CD9BDF834213F
:10098000A4F87439023A0023C4F8783992B202A963
:1009900038480AF0DDFA394936480AF08DFB04F28E
:1009A000BC6502AB424601A92846FFF71FFED0B145
:1009B000BDF83631B4F874299A4203D1D4F87829B5
:1009C000022A0CD9BDF83421A4F87439023A002364
:1009D000C4F8783992B202A926480AF0B9FA28492F
:1009E00024480AF069FBD4F88039D4F87C29023312
:1009F0009342C4F8803922D30023C4F880393846A2
:100A0000FFF72CFD07463046FFF728FD064628462F
:100A1000FFF724FD94F8853905460FB906B988B16A
:100A200053B90121174806F085FA0121154806F04F
:100A30008DFA012384F88539002384F886394EB075
:100A4000BDE8F0814BB101460E4806F073FA294625
:100A50000C4806F07BFA84F88559204694F88459AE
:100A6000FFF728FF854234BF0020012084F8860963
:100A7000E5E700BFE0D90020800D0108930D0108D3
:100A8000A60D0108908A00200EF044BF03460922FB
:100A900023F80C2B06314360C9B2024B53F82130C6
:100AA0008360704784010020002310B500F10C0220
:100AB00004460380C0E901335C3022F8023B9042D7
:100AC000FBD12046FFF7E2FF10BD024600F516718C
:100AD000002302F8013B9142FBD14FF4B472A0F81D
:100AE0005832A0F85A32A0F85C22A0F85E3280F8A2
:100AF00060327047F0B58DB002AEB0F85E32114F83
:100B00001424324637F91350D1B1AD1006339BB2DD
:100B1000772B88BF783B04F1FF344FEA650588BF27
:100B20009BB214F0FF0426F8025BEBD1A0F85E3212
:100B30000B2100941423044806F0D4FD0DB0F0BD41
:100B40000B33E4E7CA0D0108908A002070B5B0F8B5
:100B500058320446002B31D0194B1B782BB319485F
:100B6000194E06F0C9F90546142D27D9B4F85A32A2
:100B7000D91003F00702615CB25C01331142A4F8A2
:100B80005A3214BF012100212046FFF7B3FFB4F809
:100B90005A22B4F85832143D9A42ADB2E4D300233D
:100BA000A4F85A32A4F8583208E0B0F85A32002BB0
:100BB000D5D10648FFF744FE0028D0D170BD00BF54
:100BC00031070020908A0020B90D0108880A002012
:100BD00001EB41018900A0F85C127047B0F858029F
:100BE00000280CBFFF200020704729B990F8603220
:100BF00083F0010380F8603290F8600270470000D3
:100C00002DE9F043CDB004466846FFF758FD68462D
:100C1000FFF7B8FD634DB4F85CC20023A4F8583266
:100C2000A4F85A3284F86032A4F85E329AB294453D
:100C300017D994F86002B4F8582280F0010002F04D
:100C40000701D61084F860026F5CA15D30B13943B2
:100C50000132A1550133A4F85822E7E721EA070140
:100C6000F6E7504F08223E4616F8013B13F07E0F80
:100C700014BF012100212046FFF7B7FFB4F8583216
:100C8000002853D0D91003F00700615C285C0143B1
:100C9000D810013A013392B22154A4F85832002AF4
:100CA000E2D1DFF804819146BDF82C0193B2B3EB99
:100CB000C00F19464DD2C2F3CC0103F007031DF853
:100CC000016018F803301E4014BF012100212046A6
:100CD000FFF78BFFB4F8583280B3D91003F0070048
:100CE000615C285C0143D8102154591C89B2A4F8D6
:100CF0005812C6B109F10106F6B2052E13D194F8C7
:100D00006002CE1080F0010001F0070184F860025B
:100D100015F801C0A15DC8B14CEA01010233A1552B
:100D2000A4F8583200260132B146BDE703F00701AE
:100D3000685CD910615C21EA0001A9E703F00701B2
:100D4000685CD910615C21EA0001CCE721EA0C0162
:100D5000E4E7082217F8013B13F07E0F14BF0121CE
:100D600000212046FFF741FFB4F8583290B1D91066
:100D700003F00700615C285C0143D810013A01339D
:100D800092B22154A4F85832002AE3D110464DB053
:100D9000BDE8F08303F00701685CD910615C21EACB
:100DA0000001EAE7B90D0108C10D0108002310B5E3
:100DB000044603804360083004F12A01024602F829
:100DC000013B9142FBD184F82A30222202490FF0E4
:100DD00019FB204610BD00BF7D0F010830B50F4D37
:100DE000847DC1EBC1016B18695C5A78C2759A7831
:100DF0000276DA7842761A7982765A79C2769B79C7
:100E0000027F24F00F0402F00F0201F00F0123F023
:100E10000F030C431A438475027730BDC30E0108DB
:100E200030B50F4D847DC1EBC1016B18695C5A78F8
:100E3000C2759A780276DA7842761A7982765A7989
:100E4000C2769B79027F24F00F0402F00F0201F0BA
:100E50000F0123F00F030C431A438475027730BD52
:100E6000ED0E010810B504462E4802F075FB2D4822
:100E700002F0E5F9002835D06378013B032B4FD809
:100E8000DFE803F00217313C0121264802F0AAF9FD
:100E900009222549234802F0CBF822222349214880
:100EA00002F018FA01211F4802F00CF902236370C6
:100EB00018E094F82A102046FFF790FF222204F150
:100EC0000801184802F006FA94F82A30052B06D1DA
:100ED000002384F82A30237823B90323E7E701337A
:100EE00084F82A3010BD222211490E4802F0F2F98E
:100EF0000C4802F099F904236060D8E7094802F031
:100F000093F963681E339842ECD90021054802F03A
:100F1000D9F8044802F082F9002384F82A30C6E7A1
:100F20000023C4E7A4580020BA0E0108170F0108D7
:100F3000390F010810B504461D4801F001F91C489D
:100F400001F0AEF968B16378022B0BD0032B24D0EB
:100F5000012B29D122221749154801F0A9F90223B2
:100F6000637010BD94F82A102046FFF759FF222223
:100F700004F108010E4801F09BF994F82A30052B82
:100F800007D1002384F82A302378002BE9D10323EA
:100F9000E6E7013384F82A30E3E7222206490448D1
:100FA00001F086F90023DBE700236370F2E700BF5E
:100FB000B83100205B0F01089F0F010808B5124BE4
:100FC0001B785C3B062B1DD8DFE803F0181C1404CB
:100FD0001C1C0400017841B10C48012102F07CF88E
:100FE0000A48BDE8084002F0B7BA0848BDE8084022
:100FF00002F072B8BDE80840FFF734BFBDE8084012
:10100000FFF798BF08BD00BFC99A0020A458002070
:10101000012A11D1097801290CBF01230023037093
:101020000CD1437853B9064A127802F0FD025C2ACB
:1010300000D14170184670470423FBE70023F9E70D
:10104000C99A0020002303600371836000F10C0241
:1010500000F13C0122F8023B9142FBD14FF000032A
:1010600080F83C307047000037B5836890F83C202A
:1010700000294FEA4303B8BF43F001038360531CC8
:10108000DBB2172B00EB420280F83C3088BF002314
:101090009181044688BF80F83C30806820F07F430F
:1010A0002D4858400BF020FB022825D82B4A04F18C
:1010B0000C0104F13C054FF47A5331F9020B8242E2
:1010C000B8BF02468342A8BF03468D42F5D1D11A6C
:1010D000052911DD00218DF800108DF80220111274
:1010E0001A128DF801108DF80320694605221C485C
:1010F0008DF8043009F090FFA06820F07F43194874
:1011000058400BF0F1FA022824D8144A04F10C01DB
:101110004FF47A533C3431F9020B8242B8BF024695
:101120008342A8BF03468C42F5D1D11A052911DDAF
:1011300080218DF800108DF8022011121A128DF8FE
:1011400001108DF803206946052205488DF804300A
:1011500009F062FF03B030BD68B4AA0080C1FFFF90
:10116000E0D90020974B55002DE9F04104460E468A
:101170000025174643F23338ABB29F4221D936F9E6
:1011800015102379CA0F934209D02368B3F5004F95
:101190002ABF6FF4CC7003F299131B1823602368E5
:1011A000227103EB0802B2F5803F02D222600135C2
:1011B000E2E7A3F54C43CD3B23602046FFF754FF05
:1011C000F5E7BDE8F0810022027042807047000020
:1011D00030B5044685B07E4803F0A6F9237873B392
:1011E0007B4803F077FA042829D901AA79480C230F
:1011F0001146013B10F8015B02F8015B13F0FF039D
:10120000F7D162881520B2FBF0F300FB13239BB2E9
:1012100043B1012A15D130238DF80D304DF602630C
:10122000ADF80E300C226A4803F0A2FA638840F24F
:1012300076210133B3FBF1F201FB1233638005B079
:1012400030BD022A05D134238DF80D304DF61963D7
:10125000E6E7032A05D131238DF80D304DF66F6393
:10126000DEE7042A05D11F238DF80D304FF22B63E2
:10127000D6E7052A05D132238DF80D304BF2223303
:10128000CEE7062A05D124238DF80D304EF22A032D
:10129000C6E7072A05D133238DF80D304BF23B33D7
:1012A000BEE7082A01D1502354E0012B05D12523A4
:1012B0008DF80D3049F24F33B2E7022B05D1702380
:1012C0008DF80D304DF60B23AAE7032B05D125230E
:1012D0008DF80D304DF21D63A2E7042B05D13323A9
:1012E0008DF80D304BF21B339AE7052B05D12523E2
:1012F0008DF80D304DF26F7392E7062B01D1392333
:10130000E6E7072B05D125238DF80D304CF20C7341
:1013100086E7082B05D150238DF80D304DF26F0371
:101320007EE7092A4DD0092B05D125238DF80D30F4
:101330004DF21E0374E70A2A43D00A2B05D121235C
:101340008DF80D304CF20C236AE70B2A39D00B2BA9
:1013500005D125238DF80D304BF26F3360E70C2A51
:101360002FD00C2B05D13D238DF80D304DF202739B
:1013700056E70D2A25D00D2B01D1252364E70E2A2F
:101380001FD00E2B8FD00F2A1BD00F2B05D125235A
:101390008DF80D304DF21B6342E7102A11D0102B4F
:1013A00005D123238DF80D3043F61B2338E7112A8E
:1013B00007D0112B05D121238DF80D304FF2255385
:1013C0002EE716238DF80D304FF2295328E700BF82
:1013D000607A0020C10F0108012A38B5044616D1F1
:1013E0000B78012B0CBF01250025037809D12BB9FF
:1013F000438029220749084803F094F9257000200A
:1014000038BD002BFAD0044803F0D8F9F6E70420E1
:10141000F6E700BFCD0F0108607A002000224FF4EC
:10142000C061C0E900228160027370472DE9F34179
:10143000444E027B33789A42044668D0663B40F6BD
:10144000BF12052B55D8DFE803F003070A0D101370
:101450004FF46F7323800CE040F20F43FAE740F241
:10146000DF43F7E740F26163F4E740F61F03F1E77B
:101470000280238893423ED040F61F0293423CD024
:1014800040F2616293423AD040F2DF42934238D058
:1014900040F20F42934236D0B3F56F7F4ED1052311
:1014A000294F17EBC30749D060687B88638008B178
:1014B0000EF034FF608840000EF006FF00256060EB
:1014C000A8466288ABB29A421FD940460EF0E0FEB1
:1014D000B4F90830626883FB0001C30F43EA41039B
:1014E000A9B203F30F0322F811307B680135984449
:1014F000E7E70023AEE70023D2E70123D0E702238A
:10150000CEE70323CCE70423CAE733782373A37A17
:10151000A3B10E480D4F05F0EFFC4FF00008054653
:101520006388AB420AD2CDF80080626831783846D1
:1015300006F0D8F86388ED1AADB2F1E702B0BDE865
:10154000F08100BFC99A0020F80F0108908A00209E
:10155000012A06D10B785A1E534253418372002050
:1015600070470420704700220270704710B504468F
:10157000084807F017F823785BB1064807F0C5F86C
:10158000012806D9312204490248BDE8104007F07D
:10159000C4B810BDCC95002028100108012A06D13E
:1015A0000B785A1E534253410370002070470420A9
:1015B00070470022027042708270704710B5044676
:1015C000104807F04FFE0F4807F013FFA8B16378EB
:1015D000012B13D1A1780C4B0A48C1EBC101C1EB1F
:1015E000C1011944312207F00CFFA378013303F045
:1015F0000303A370237803B9637010BD00236370E5
:10160000A370FAE748AA002059100108012A0BD15B
:101610000A78012A0CBF01230023037006D1437806
:1016200023B94270184670470423FBE70023F9E70B
:10163000002202704270704710B504460F4808F04F
:10164000D5FC0E4808F06CFD68B16378012B03D01F
:10165000022B09D0002305E0D9220949074808F0E8
:1016600067FD0223637010BDD9220649034808F0C4
:101670005FFD2378002BF5D00123F3E720D2002073
:1016800026030020FF030020012A0BD10A78012A3B
:101690000CBF01230023037006D1437823B94270A5
:1016A000184670470423FBE70023F9E70022027085
:1016B0007047000008B5037853B1064805F01CFCDC
:1016C000A52805D9AA210448BDE8084008F0B4BD02
:1016D00008BD00BF908A0020A0D70020012A06D1B3
:1016E0000B785A1E53425341037000207047042068
:1016F00070470022C0E900224FF6FF7282607047F7
:101700002DE9F743DFF8689004460E46002517469A
:1017100045F6BF58ABB29F4226D936F815206189ED
:1017200063689142218938BF62819142134488BF26
:1017300022812268636001324245226012D9B3FBE4
:10174000F2F3A16809BA5BBA0091062269464846DD
:10175000ADF8043009F088FC0023C4E900334FF6EB
:10176000FF73A3600135D5E703B0BDE8F08300BF88
:10177000E0D90020024600F57A71002302F8013B0F
:101780009142FBD1A0F8E833A0F8EA3380F8EC33BB
:10179000704700002DE9F341B0F8E8330446002B10
:1017A0003BD01F481F4FDFF884801D4E05F0A4FB7F
:1017B0000546182D31D9B4F8EA33D91003F00702E1
:1017C000635CBA5C13401BBF002300930093182393
:1017D0000ABF1823144A42466121304605F082FFB1
:1017E00094F8EC330133DBB2183D312BADB284F801
:1017F000EC3307D9B4F8EA330133A4F8EA33002311
:1018000084F8EC33B4F8EA23B4F8E8339A42D0D33E
:101810000023A4F8EA33A4F8E83302B0BDE8F0816D
:10182000908A002030130108D8040020580A0020B4
:101830002DE9F74F04460E46904600214FF47A7288
:101840000EF07AFE0823A4F8E833DFF8C4E00023A2
:10185000A4F8EA3384F8EC33DDB2454542DA0021DE
:101860000C20CAB242430EEB02001EF80220BAB3AB
:10187000775D974201F10101F2D190F808B0019033
:101880004FF0000C4FF000455FFA8CF18B45B4F837
:10189000E82325D902F007071A4810F807A0019895
:1018A0004FEAE209476814F8091035EA07000CBF4F
:1018B00041EA0A0121EA0A0104F8091040F2E23182
:1018C0008A420CF1010C06D90023A4F8E833042065
:1018D00003B0BDE8F08F0132A4F8E8236D08D3E728
:1018E0000133B9E7B4F8E823082AEDD0053292B203
:1018F000A4F8E8230448054912B209F0BFFE00200D
:10190000E6E700BF30130108E0D9002038130108D2
:10191000201101080023A0F8E833A0F8EA3380F88A
:10192000EC3370470023C0E90033C0E902330361A0
:1019300000F1140200F6543122F8023B8A42FBD136
:1019400042F20F72C0F8543BC0F8583BA0F85C2B31
:10195000C0F8603BC0F8643BC0F8683BC0F86C3B23
:10196000C0F8703BC0F8743BA0F8783B00F5B55266
:101970004FF0000380F87A3B1C3200F67C330021E4
:1019800023F8021B9A42FBD170470023C0F8603B4A
:1019900080F8753B80F8763B80F8783BC0F8583B80
:1019A00042F20F73A0F85C3B704700002DE9F74F3F
:1019B000BDF83040BDF93880BDF934A0DFF8909013
:1019C00004EB420292B20192C8F1000B019AA242CA
:1019D0003BD000EB4102671C958ABFB2A5EB0A051C
:1019E0004FEAE40E04F007062DB2FA1007F00707DD
:1019F00002345D4513F80EC019F8066019F8077037
:101A0000A4B206DA2CEA060603F80E609D5C2F43AA
:101A100008E0002D11DA2CEA060603F80E609D5C42
:101A200025EA07079F544A1D92B2B2F5B46F24BF4E
:101A3000A1F29B518AB21146C8E74CEA060603F8A8
:101A40000E6045459D5CE2DAEAE703B0BDE8F08F41
:101A5000541301082DE9F04FB0F8543B50F82330EF
:101A60000446924823F07F43584089B088460AF0E4
:101A70003BFEC31EDBB2122B814640F2B880B4F8A5
:101A8000563B8B4DDFF83CE203F22D5189B2B1F5A4
:101A9000B46F24BFA3F1730189B200224FF47A53CB
:101AA0000846049316464FF6FD7A4FF0030B04EBFD
:101AB0004007049BB7F91470BD42B8BF3D46BB4216
:101AC000A8BF3B46B9F1020F04938ABF794B12F9C4
:101AD0000EC012F903C0BCF1010F00F08B80BCF105
:101AE000030F05D0BCF1FF3F40F086803E4401E08B
:101AF00017FB0A66471DBFB2B7F5B46F28BFA0F247
:101B00009B5002F101022CBF80B23846182ACED178
:101B1000D4F8600BB0426ADA049B2B445B101FB20E
:101B2000ED1A44F631435D4345F3CF3504230DF1FF
:101B3000180A0093CDE9017553462046FFF736FF9A
:101B4000B9F1020F5C4969D84FF0000B5B4AD946E6
:101B500011F8013B1AF80BC012F8010B059103EACA
:101B60000C03584004920AF0AFFD0BF1010B8144C5
:101B7000BBF1070F5FFA89F9DDE90421E8D1B9F17A
:101B8000030F34D8B8F1000F39D0A4F8725BA4F871
:101B9000705BA4F86E5BA4F86C5BA4F86A7BA4F895
:101BA000687BA4F8667BA4F8647B002384F8743B0C
:101BB000C4F8606B402384F8753BB4F8563BA4F836
:101BC000583B03F21A4292B2B2F5B46F28BFA3F5A4
:101BD000C372A4F85A2B03F20D1292B2B2F5B46F8D
:101BE0002ABFA3F29343A4F85C2BA4F85C3B09B092
:101BF000BDE8F08FF61B7DE717FB0B667AE794F8DC
:101C0000743B04EB43020133DBB2032BA2F86C5BA1
:101C1000A2F8647BCAD984F8748BC9E74FF0000B33
:101C2000274AD94611F8013B1AF80BC012F8010BEC
:101C3000059103EA0C03584004920AF045FD0BF1AC
:101C4000010B8144BBF1070F5FFA89F9DDE904213B
:101C5000E8D1B9F1030FCAD8B8F1000F16D0A4F833
:101C6000725BA4F8705BA4F86E5BA4F86C5BA4F8DC
:101C70006A7BA4F8687BA4F8667BA4F8647B0023E5
:101C800084F8743BC4F8606B202394E794F8743BA9
:101C900004EB43020133DBB2032BA2F86C5BA2F826
:101CA000647BEDD984F8748BECE700BF6E28760076
:101CB00080C1FFFF891301085C1301086313010849
:101CC0006A1301087113010880F8771B7047000040
:101CD000B0F85A3B3C3370B40A469BB24FF40775D8
:101CE000002400EB43015E1CB6B2B6F5B46FB1F848
:101CF0007C1B05F1FF3528BFA3F29F53ADB20C4406
:101D00002CBF9BB23346002DEBD14FF40773B4FBCD
:101D1000F3F4C4F3072382F8223082F8234024230B
:101D20000121024870BC08F097BE00BFE0D9002036
:101D300070B50446B0F8560B04EB400300299982B5
:101D4000A3F87C2BB4F8542B54F822304FEA430309
:101D5000B8BF43F0010344F8223094F8783B8EB0CA
:101D6000002B6AD101212046FFF774FEB4F85C2BEA
:101D7000B4F8563B934240F09780B4F9662BB4F91F
:101D8000645BB4F96C6B1544B4F9682B1544B4F971
:101D90006A2B1544B4F96E2B1644B4F9702B03F278
:101DA00012311644B4F9722B89B2B1F5B46F1644EE
:101DB00028BFA3F28E2194F8752B8DF814204FF0D4
:101DC000080345F38F0546F38F0628BF89B20093B9
:101DD000CDE9015605AB84222046FFF7E7FD94F8D4
:101DE000753B402B40F0C18004A801F023F80DF1B1
:101DF00013030DF112020DF1150104A801F048F8CA
:101E000094F8772B9DF812309A4248D100239DF820
:101E1000142084F8763B84F8793B9DF813301A43FC
:101E20008DF814200A2B00F29A80DFE803F07A6A1A
:101E300084989898265757985700B4F8581B01F281
:101E40009F539BB2B3F5B46F01F1010292B224BF6C
:101E500001F1FF339BB2B2F5B46F24BFA1F29F52E0
:101E600092B2934206D2984280D390423FF67EAF20
:101E7000002178E79842F8D3FAE72B46B4F9582BBB
:101E80006449654800960AF060F905A92046FFF705
:101E90001FFF022384F8783B002384F87A3B002359
:101EA000C4F8603B84F8753BB4F8563B94F8780B63
:101EB00001339BB2B3F5B46F28BF0023A4F8563B9F
:101EC000B4F8543B01339BB2042B88BF002300308D
:101ED00018BF0120A4F8543B0EB070BD94F8783BB5
:101EE000022BDCD12B46B4F9582B4C494A480096BA
:101EF0000AF02BF905A92046FFF7EAFE9DF81330FA
:101F0000CBE7B4F9582B464900962B4642480AF0D5
:101F10001CF905A92046FFF7DBFE012384F8783B76
:101F2000BDE794F8783B012BF7D100962B46B4F926
:101F3000582B3C49EAE794F8783B012BAFD1B4F930
:101F4000582B394900962B4633480AF0FEF82046B4
:101F500005A9FFF7BDFE2046FFF717FD9FE7009696
:101F60002B46B4F9582B3149EEE7202B12D12B46E2
:101F7000B4F9582B2E49284800960AF0E6F805A92E
:101F80002046FFF7A5FE002384F8763B0123A4F842
:101F9000783B84E794F8783B73B194F8763B01334F
:101FA000DBB20C2B84F8763B06D91B48012108F0E4
:101FB00083FD2046FFF7E9FC94F8783B012B17D10D
:101FC00094F8793B1448042B8DBF20230133DBB2F6
:101FD0008DF8143087BF002384F8793B84F8793B6F
:101FE0008DF8143005AA2223012108F035FD56E7AB
:101FF000022B7FF454AF94F87A3B002B3FF44FAFA1
:1020000043F0400305A920468DF81430FFF760FE29
:1020100045E700BFA1130108E0D90020D213010851
:1020200004140108361401086B140108A1140108F6
:10203000CB1401082DE9F04100240E460546174651
:1020400098462146444509D036F9141037F8142033
:102050002846FFF76DFE01340146F3E70248BDE86C
:10206000F04104F067BF00BF908A002070B50446BD
:1020700000254FF4B9702581208065816573257333
:102080000EF022F9C4E9045504F11C066060A56154
:1020900004F13C03324622F8025B9342FBD104F286
:1020A000EC41002203F8012B9942FBD1F023C4F844
:1020B000EC24C4F8F0342022002130460EF03CFA23
:1020C0000523237409236382024B2046C4E90536A5
:1020D00070BD00BF08050020F0B58FB00A46002390
:1020E00002A94FF4E37540F252564FF6AE274FF671
:1020F0003A6C02F0C004802C1DD0C02C18D0002CEB
:102100000CBF64463C4621F8134001339200042B77
:10211000D2B2EED104AA10300DF000FA00230093E1
:1021200004AA14230221054805F0DCFA0FB0F0BD23
:1021300021F81360E9E721F81350E6E7908A0020C0
:1021400038B5B0F8EC340446E3B13C4804F0D4FEB2
:102150000546142D45D9B4F8EE345A1C2344A4F88E
:10216000EE2493F83C102046FFF7B6FFB4F8EE24B7
:10217000B4F8EC34143D9A42ADB2EAD30023C4F86B
:10218000EC342EE0428903899BB2934212D1037B47
:102190003BB303882BB32A4B1B781BBBD4F8F0242A
:1021A0005F20591C9BB29A4212D9234483F83C0009
:1021B0000B46F6E7438902899A429DBF428901880E
:1021C000038903898CBF42895B189B1A9BB2E1E7A4
:1021D000A4F8EC240023A4F8EE34B4F8EC34002B7B
:1021E000B3D138BD04F13C0304F15D000021258921
:1021F000628992B2AA4201D1227B72B1656862897A
:1022000092B2AA5C1A7021736289013292B2628121
:1022100062892588954298BF618101338342E6D166
:10222000084A04F1840112F8010B03F8010B8B42F8
:10223000F9D14823A4F8EC34CCE700BF908A002001
:10224000CA9A0020FB1401080C234FF4167203FBFA
:102250000121B1F5966F8ABF4FF49663C0F8F01470
:10226000C0F8F03470474189038902889BB28B42E1
:1022700005D1037B002B0CBF10460020704743891B
:102280000189994287BF038940894389008986BFB4
:102290008018C01A181A80B2904288BF0020704778
:1022A00008B5FFF7E0FF2323B0FBF3F0C0B208BD91
:1022B000222AF8B504460D4624D1FFF7D4FF202882
:1022C00022D901231946227B02F0FF002AB1617353
:1022D0000133222BF7D10020F8BD66682289EF5C1C
:1022E00092B2B7542289013292B222812289268881
:1022F000964298BF20812089628992B2824208BFAB
:102300002173E5E70420E7E70520E5E70023C0E9BE
:102310000033C0E90233036100F1140200F23C51C2
:1023200022F8023B9142FBD1C0F83C3542F20F72D9
:10233000C0F84435C0F848354FF00003A0F84025F8
:1023400080F84C3570470023C0F84435C0F8483554
:10235000C0F83C3542F20F73A0F8403570470000DA
:102360002DE9F74FBDF83040BDF93880BDF934A0F4
:10237000DFF8909004EB420292B20192C8F1000B98
:10238000019AA2423BD000EB4102671C958ABFB282
:10239000A5EB0A054FEAE40E04F007062DB2FA1089
:1023A00007F0070702345D4513F80EC019F8066000
:1023B00019F80770A4B206DA2CEA060603F80E60D4
:1023C0009D5C2F4308E0002D11DA2CEA060603F885
:1023D0000E609D5C25EA07079F544A1D92B2B2F534
:1023E000257F24BFA1F28F218AB21146C8E74CEAAB
:1023F000060603F80E6045459D5CE2DAEAE703B0A5
:10240000BDE8F08F22150108B0F83C2550F82230C5
:1024100000294FEA4303B8BF43F001032DE9F04F11
:1024200040F82230B0F83E3500EB43030446998271
:1024300050F822307B4823F07F4391B058400AF097
:1024400053F9022800F29080B4F83E35DFF8E8E155
:10245000754F03F2212189B2B1F5257F24BFA3F185
:10246000730189B20A4618254FF47A5300264FF6B5
:10247000FD784FF0030904EB42001EF901CBB0F9DF
:1024800014008742B8BF07468342A8BF0346BCF189
:10249000010F00F0C280BCF1030F05D0BCF1FF3F7B
:1024A00040F0BD80064401E010FB0866501D80B27C
:1024B000B0F5257F28BFA2F28F2205F1FF352CBF92
:1024C00092B2024615F0FF05D5D1D4F84425B242A8
:1024D0004ADA3B445B100FFA83F8FB1A44F63147A3
:1024E0005F4347F3CF3704230DF11C0A00931822F2
:1024F000CDE9018753462046FFF732FFDFF83CB1B4
:102500004A4AA94612F8013B1AF809101BF8010BB8
:102510000B405840CDE904220AF0D6F809F1010930
:102520000544B9F1070FEDB2049AEBD1032D1BD886
:102530003B4642463E493F4809F0D0FDB4F83E359F
:10254000C4F8446503F20D1292B2B2F5257F24BFA0
:102550006FF4C3729B18A4F84885A4F84A7534BF79
:10256000A4F84025A4F84035B4F84025B4F83E3529
:1025700093423CD1991D89B2B1F5257F28BFA3F2C2
:102580008E21B4F94A350293B4F9483501934FF0DE
:10259000080328BF89B284220093204607ABFFF7C7
:1025A000DFFE06A800F046FC0DF11B030DF11A0238
:1025B0000DF11D0106A800F06BFC94F84C259DF868
:1025C0001A309A420CD19DF81B30032B08D1C3233B
:1025D0008DF81C3007AA22230021164808F03CFA87
:1025E00042F20F73A4F840350023C4F84435B4F820
:1025F0003E3501339BB2B3F5257F28BF0023A4F8F5
:102600003E35B4F83C3501339BB2042B88BF002320
:10261000A4F83C3511B0BDE8F08F361A46E710FB40
:10262000096643E76E28760080C1FFFF2A1501087E
:1026300050150108E0D900203815010831150108AE
:1026400070B505460C4601EB4206B44205D034F99C
:10265000021B2846FFF7D8FEF7E770BD80F84C153F
:10266000704710B50021044600F062F8012104F61D
:10267000546000F05DF8204610BD00002DE9F84FD1
:10268000064600249DF828B0884691469A46204682
:10269000254606F65467A3B29B451BD91AF80430A9
:1026A000042B15D0082B02D1304600F074F839F80D
:1026B000142038F91410304600F01EFA39F81420AE
:1026C00038F914100546384600F016FA0134E2E7EE
:1026D0003846EAE7002D14BF294601460248BDE806
:1026E000F84F04F027BC00BF908A002038B504469C
:1026F0000D4600F0D5F9294604F65460BDE838408F
:1027000000F0CEB938B504460D4600F0CCF92946A4
:1027100004F65460BDE8384000F0C5B910B5044671
:1027200000F043F804F65460BDE8104000F03DB8F6
:102730000023C0E90133C0E903330170436100F1B4
:10274000180200F5E46122F8023B8A42FBD142F212
:102750000F72C0F82037C0F82437C0F82C37C0F803
:102760003037C0F83437C0F83837C0F83C37C0F8D5
:102770004037C0F844374FF00003C0F8282780F8EE
:10278000483700F6526200F24A73002123F8021B18
:102790009A42FBD170470023A0F82A37C0F82037AF
:1027A000C0F82C3780F841377047002342F20F728F
:1027B00080F8413780F8423780F84637C0F8203734
:1027C000C0F82437C0F82827C0F82C37704700001D
:1027D0002DE9F74FBDF83040BDF93880BDF934A080
:1027E000DFF8849004EB420292B20192C8F1000B30
:1027F000019AA24235D001F10C02671C30F8125048
:10280000BFB2A5EB0A054FEAE40E04F007062DB2AD
:10281000FA1007F0070702345D4513F80EC019F8E7
:10282000066019F80770A4B206DA2CEA060603F867
:102830000E609D5C2F4308E0002D0ADA2CEA0606A4
:1028400003F80E609D5C25EA070705319F5489B2A5
:10285000CEE74CEA060603F80E6045459D5CE9DAD2
:10286000F1E703B0BDE8F08F7C150108B0F8203720
:102870002DE9F04F00EB830304465B68814823F0A9
:102880007F43584089B0884609F02EFFC31EDBB253
:10289000122B814640F29880B4F822177A4DDFF867
:1028A000FCE1733989B200224FF47A530F46049346
:1028B00016464FF6FD7A4FF0030B07F10C00049B10
:1028C00034F910008542B8BF05468342A8BF0346CD
:1028D000B9F1020F04938ABF6C4B12F90EC012F9C2
:1028E00003C0BCF1010F72D0BCF1030F04D0BCF1E6
:1028F000FF3F6ED1064401E010FB0A660132053746
:10290000182ABFB2D9D1D4F82C07B0425CDA049BA4
:102910002B445B101FB2ED1A44F631435D4345F37F
:10292000CF3504230DF1180A0093CDE90175534604
:102930002046FFF74DFFB9F1020F55495BD84FF024
:10294000000B544AD94611F8013B1AF80BC012F893
:10295000010B059103EA0C035840049209F0B4FE00
:102960000BF1010B8144BBF1070F5FFA89F9DDE937
:102970000421E8D1B9F1030F26D8B8F1000F2BD00C
:10298000A4F83E57A4F83C57A4F83A57A4F838578F
:10299000A4F83677A4F83477A4F83277A4F830771F
:1029A000002384F84037C4F82C67402384F841376B
:1029B000B4F82237A4F82437A3F5C37203F20D1339
:1029C000A4F82627A4F8283709B0BDE8F08F361AF6
:1029D00094E710FB0B6691E794F8403704EB430251
:1029E0000133DBB2032BA2F83857A2F83077D8D9DD
:1029F00084F84087D7E74FF0000B274AD94611F8F3
:102A0000013B1AF80BC012F8010B059103EA0C0305
:102A10005840049209F058FE0BF1010B8144BBF1C0
:102A2000070F5FFA89F9DDE90421E8D1B9F1030F55
:102A3000CAD8B8F1000F16D0A4F83E57A4F83C57F6
:102A4000A4F83A57A4F83857A4F83677A4F834779E
:102A5000A4F83277A4F83077002384F84037C4F81C
:102A60002C672023A2E794F8403704EB430201339C
:102A7000DBB2032BA2F83857A2F83077EDD984F8EF
:102A80004087ECE76E28760080C1FFFFB115010892
:102A9000841501088B150108921501089915010884
:102AA00080F843177047A0F84417704730B4B0F867
:102AB000264704F13C0304F51674A5B20A469BB2FE
:102AC0000024591C00EB4303B3F84A371C448BB273
:102AD000AB42F6D14FF40773B4FBF3F4C4F307230E
:102AE00082F8223082F8234001780248242330BC47
:102AF00007F0B2BFE0D9002070B5B0F82A3704461D
:102B00000133B4F844579BB29D42A0F82A378EB0E7
:102B100090F8460704D9003018BF01200EB070BDF0
:102B2000B4F82237B4F828579D42F4D3B3F5617F47
:102B3000F1D204EB43050029A5F84A272983B4F80C
:102B4000205704EB85056A684FEA4202B8BF42F09D
:102B500001026A60002865D1A3F5C8735A2B03D817
:102B600001212046FFF782FEB4F82837B4F8221777
:102B700099427BD1B4F93237B4F93057B4F9386798
:102B80001D44B4F934371D44B4F936371D44B4F943
:102B90003A371E44B4F93C371E44B4F93E371E445C
:102BA00094F841378DF8143045F38F05082346F328
:102BB0008F06A1F28E210093CDE9015605AB842248
:102BC00089B22046FFF704FE94F84137402B40F0CD
:102BD000C38004A800F02EF90DF113030DF11202C9
:102BE0000DF1150104A800F053F994F843279DF85E
:102BF00012309A423AD100239DF8142084F84237CB
:102C000084F847379DF813301A438DF814200A2BA7
:102C100000F29780DFE803F0695478959595123BB0
:102C20003B953B00B4F82427511E89B28B429BD3BD
:102C3000013292B2934297D8002192E723787549E6
:102C40007548002B18BF0222B4F9243708BF0122AF
:102C5000CDE9005609F0C0FA05A92046FFF726FF86
:102C6000022384F84637002384F84837B4F8223723
:102C700094F846070133A4F82237B4F8203701331B
:102C80009BB2042B88BF0023A4F8203743E794F8B5
:102C90004637022BEAD1237860495F48002B18BFE2
:102CA0000222B4F9243708BF0122CDE9005609F009
:102CB00093FA05A92046FFF7F9FE9DF81330D3E7F4
:102CC00023785749CDE90056002BB4F9243714BFB7
:102CD00002220122504809F07FFA05A92046FFF799
:102CE000E5FE012384F84637C0E794F84637012B08
:102CF000F7D123784B49002BCDE90056B4F924379E
:102D000014BF02220122E5E794F84637012BADD12A
:102D100023784549CDE90056002BB4F9243714BF78
:102D2000022201223C4809F057FA05A92046FFF784
:102D3000BDFE002384F8463742F20F73A4F828370B
:102D400094E723783949002BCDE90056B4F92437AC
:102D500014BF02220122E5E7202B18D12378344941
:102D60002D48002B18BF0222B4F9243708BF0122D6
:102D7000CDE9005609F030FA05A92046FFF796FE86
:102D8000002384F842370123A4F846376EE794F80D
:102D9000463793B194F842370133DBB20C2B84F8F9
:102DA00042370AD921781C4807F086FE002384F8B0
:102DB000463742F20F73A4F8283794F84637012BB0
:102DC00017D194F8473721781348042B8DBF20235F
:102DD0000133DBB28DF8143087BF002384F8473706
:102DE00084F847378DF8143005AA222307F034FE03
:102DF0003CE7022B7FF43AAF94F84837002B3FF4BE
:102E000035AF43F0400305A920468DF81430FFF795
:102E10004DFE2BE7C9150108E0D900200016010876
:102E20003816010870160108AB160108E7160108EC
:102E30001717010870470000B1F5006F10B50DD3EA
:102E400007484FF4802340F675440B4201D15B08DC
:102E5000FBE7DA0A624351400142F6D1084610BD51
:102E600000F8FFFF10B54C780B78E40004EBC324A6
:102E70008B7804EB53142146FFF7DEFF034B53F826
:102E800020006040C0F3C72010BD00BF50170108EC
:102E900073B51E464B7B0C7B15469A0942EA8402A9
:102EA0000C7DC97C8DF8042089009B0023F03F0332
:102EB00001F03C01194341EA9411A4008DF805107A
:102EC00024F00F0401A98DF80640FFF7CBFF03099A
:102ED00000F00F002B70307002B070BD02F00F02D6
:102EE00042EA0111C8B2197B124A21F03F0141EABE
:102EF000900130B532F810401973597BE5B2AA0839
:102F000001F00F0141EA801102F0300001435973D2
:102F1000D97C02F00F0221F00F0111431A7DD97400
:102F200002F00302A40A42EA851204F03C042243A0
:102F30001A7530BD503701082DE9F04100254FF4D6
:102F4000B976044605810680458145730573304690
:102F50000DF0BAF9258360602682658330462577B7
:102F600065770DF0B1F9C4E9085504F12C066061EC
:102F7000A56204F14C02334623F8025B9A42FBD16E
:102F80004FF0000384F84C3004F16E0104F14D035E
:102F9000002203F8012B9942FBD104F16F0884F859
:102FA0006E2004F17B074346002203F8012B9F4269
:102FB000FBD104F187023B46002103F8011B9A4232
:102FC000FBD104F1AF03002102F8011B9342FBD1B6
:102FD00004F1D702002503F8015B9A42FBD1C4E952
:102FE0003655C4E93855A4F8E8502022002130466F
:102FF0000DF0A2FA052384F82030092363840A4BDC
:103000000A49C4E909360C2238460DF0FBF90C22B6
:10301000064940460DF0F6F9C4E93855A4F8E850E1
:103020002046BDE8F08100BF620500205839010844
:10303000092A2DE9F04104460D4627D10C22002132
:103040007B30134E134F0DF077FA002316F8011B57
:1030500004EBD10001F0070103F0070817F801C0E5
:1030600090F87B20D910013315F801E017F808100B
:103070001EEA010F14BF42EA0C0222EA0C02442BA2
:1030800080F87B20E2D10020BDE8F0810420FBE73E
:103090006439010850390108012A04D1097801294D
:1030A00003D0022908D0042070470023C0F8E03084
:1030B00080F8E810184670470023C0F8E43080F824
:1030C000E920F7E7002380F84C10C0E93733C0F857
:1030D000E430A0F8E8307047002914BF052300232E
:1030E00080F84C30704700002DE9F04194B006465E
:1030F0001746002403AD4FF4E37240F252504FF6EE
:10310000AE2C4FF63A6E01F0C003802B2AD0C02BB4
:1031100025D0002B0CBF7346634625F814300134CC
:103120008900042CC9B2EED10DF11408142200213B
:1031300040460DF001FA23460AAA294606F120006E
:103140008DF81E700CF0EAF9CDF8008014230AAA5D
:103150000221064804F0C6FA14B0BDE8F08125F853
:103160001400DCE725F81420D9E700BF908A00207E
:103170001B4B1B78622B10B512D100F1870300F1B5
:10318000A8025F24002183F8284003F8011B934222
:10319000F9D12123A0F8D8300023A0F8DA3010BDEF
:1031A0005F2BF9D100F1870300F18E025524002135
:1031B00083F8284003F8011B9342F9D15F2380F87C
:1031C000B63000F1960200F18F03FF24002183F84E
:1031D000284003F8011B9342F9D10F23DAE700BF1F
:1031E000C99A002037B500F14D040D462122074948
:1031F00020460DF007F901A8FFF71CFE234609221F
:10320000294601A8FFF76AFE03B030BDA8390108BE
:1032100000230381437343810373704700230383B7
:103220004377438303777047D0F8DC00704708B5D5
:10323000FFF719F82323B0FBF3F0C0B208BD08B5BF
:103240001030FFF710F82323B0FBF3F0C0B208BD35
:10325000222AF8B504460D4633D1FFF704F820289A
:1032600031D994F8E83033B100232381637363814B
:1032700084F8E830237301231946227B02F0FF0013
:1032800052B161730133222BF7D1114B1878E0B999
:10329000012384F84C30F8BD66682289EF5C92B255
:1032A000B7542289013292B222812289268896421D
:1032B00098BF20812089628992B2824208BF21731F
:1032C000E0E70420E7E70520E5E70020E3E700BFAB
:1032D000CA9A0020222AF8B504460D4634D110308F
:1032E000FEF7C1FF202831D994F8E93033B100232B
:1032F00023836377638384F8E930237701231946B6
:10330000227F02F0FF0052B161770133222BF7D107
:10331000104B1878E0B9012384F84C30F8BD666989
:10332000228BEF5C92B2B754228B013292B222838D
:10333000228B268A964298BF2083208B628B92B282
:10334000824208BF2177E0E70420E7E70520E5E7B0
:103350000020E3E7CA9A0020428903899BB2934286
:1033600005D1027B02F0FF0382B1008870474389D8
:1033700002899A429DBF42890389008803898BBFD5
:103380004089C018181A801A80B2704718467047D2
:10339000F8B5D0F8DC300133C0F8DC30D0F8E030DC
:1033A0000133C0F8E030D0F8E4300133C0F8E43045
:1033B00090F86E300B2B04460F46164600F16F0551
:1033C00013D9002380F86E302046FFF7C5FF002890
:1033D00068D104F11000FFF7BFFF002862D1354922
:1033E0000C2228460DF00EF801E0002BECD094F8EA
:1033F0006E100322294404F1AF000DF003F8012EF2
:103400000CBF0823042384F88930D4F8DC30002072
:10341000132B84F8870084F8880006D904EB061083
:10342000FFF79AFF003018BF01207B1E94F86E2032
:1034300059425941002A39D0B2F1090C18BF4FF056
:10344000010C012594F8AF30012F80EA010643EA10
:10345000C0100CBF08230023184394F8B03084F840
:10346000AF0043EAC513694043EACC03AE4214BF40
:10347000022500252B4384F8B03094F8B130614523
:1034800014BF202100211943664514BF02260026DF
:10349000032331431A4484F8B110C4F8D83084F8B7
:1034A0006E20F8BD0C2204F17B019AE715464FF01F
:1034B000010CC7E758390108F8B500EB01160546BD
:1034C00030460C46FFF748FF202809D9D5F8DC30F4
:1034D000132B05D904F1380355F82330052B10D8E8
:1034E0002C44002284F8E82005F14D0305F16E011B
:1034F00013F8010B83F861008B4283F83920F7D170
:1035000026E005EB041405F1870105F1A807234621
:103510000020B4F808C0628992B2624501D1227BD2
:1035200092B1D6F804C05A8992B21CF8022081F8F0
:10353000282018735A89013292B25A815A89B6F8F2
:1035400000C0944598BF588101F8010B8F42E0D12B
:103550002123C5F8D830F8BD38B590F84C30044672
:10356000002B41D0B0F8D820F2B1234803F0C4FCBE
:103570000546142D38D9B4F8DA30E218013392F840
:10358000AF1092F88720A4F8DA302046FFF7ACFDA0
:10359000B4F8DA20B4F8D830143D9A42ADB2E8D38A
:1035A0000023C4F8D8301FE0013B042B1DD8DFE80E
:1035B00003F0031C100A15000021FFF77DFF042310
:1035C00084F84C300CE000220121FFF7E1FE0323D8
:1035D000F6E70121FFF770FF0223F1E7FFF7C8FDCF
:1035E000B4F8D830002BC0D138BD01220021FFF73C
:1035F000CFFE0123E4E700BF908A002003460022AB
:1036000030B503F8082B002400F130020025E3E870
:1036100002459A42FBD100F5D0530C33002122F829
:10362000021B9342FBD100F5EE511A460C310023E8
:1036300022F8023B9142FBD141F6CC522F498350F4
:1036400041F6D052815041F6D4522D49815041F675
:10365000D85242F20F71815241F6DC524FF0000114
:10366000835000F5EF52136041F6E452835241F665
:10367000E652815441F6E8520021835041F6EC5263
:10368000835041F6F052835041F6F452835041F694
:10369000F852835000F5EF5200F5F5531C32043315
:1036A00042F8041B9342FBD11A4600F5FA530C333F
:1036B000002142F8041B9342FBD11A4600F5FF5348
:1036C0001433002142F8041B9342FBD11A4600F543
:1036D00002531C33002142F8041B9342FBD100F536
:1036E00003510631002203F8012B9942FBD142F22B
:1036F000C803C25042F2CC03C25230BD00000F27B3
:103700000F270F2741F6DC5200230370835000F58A
:10371000EF520F49136041F6CC52835041F6D0521C
:10372000815041F6D4520B49815041F6D85242F2B1
:103730000F71815241F6E452835241F6E6528354AE
:1037400042F2C802835042F2CC028352704700BF5B
:1037500000000F270F270F2710B542F2CC030446B5
:10376000C05AB0B142F2C8032B22E358B3FBF0F3C6
:10377000C3F3072081F8290081F82A30064807F0B2
:10378000D7F842F2C8020023A35042F2CC02A3525F
:1037900010BD2922F2E700BFE0D9002010B542F2A7
:1037A000CC030446C05AA0B142F2C8030E22E3582B
:1037B000B3FBF0F3C3F3072008734B73064807F01D
:1037C000E3F842F2C8020023A35042F2CC02A35213
:1037D00010BD0C22F2E700BFE0D9002070B541F621
:1037E000CC530446C35A0133002150F833302048EB
:1037F00023F07F43584008F08BFF022835D841F66C
:10380000D0531C4DE25A02F26D139BB2B3F5F07F18
:1038100024BFA2F173039BB21820002103F60452C7
:1038200004EB420215F8016BB2F90420DEB1891AEB
:103830005A1D92B2B2F5F07F24BF6FF4ED729B185F
:1038400000F1FF302CBF9BB2134610F0FF00E5D112
:1038500041F6DC53E2588A4204DAE15041F6CE5395
:10386000E052012070BD1144E2E70020FAE700BFFA
:103870005076550085410108F8B541F6CC530578DE
:10388000C35A0133044650F83330364823F07F439F
:10389000022D80EA03004FF0000118BF002508F058
:1038A00037FFA8425BD841F6D0532F4EE25A02F2BE
:1038B0006D139BB2B3F5F07F24BFA2F173039BB2EB
:1038C0001820002503F6045104EB410116F8017B92
:1038D000B1F90410002F40D06D1A591D89B2B1F50D
:1038E000F07F24BF6FF4ED77DB1900F1FF302CBFC0
:1038F0009BB20B4610F0FF00E4D104F5EF531968BA
:10390000A94229DA1D6041F6E45341F6D251E05252
:1039100041F6D453E252531D9BB2B3F5F07F24BF5E
:103920006FF4ED7013186352531C9BB2B3F5F07F24
:1039300028BF6FF4EF7341F6D85128BFD3186352F4
:1039400002F2DF139BB2B3F5F07F41F6D65128BFE8
:1039500002F1FF3363520120F8BD0D44BDE70020A2
:10396000FAE700BF68B4AA006D41010838B5044603
:103970000D46FFF733FFB0B141F6E6530522E2549E
:1039800041F6CE52A35A03F11800013324F8105027
:10399000A35242F2C8020023A35042F2CC02A35227
:1039A0000123237038BD2046FFF766FF0028F9D0B9
:1039B0000649074807F080FB0121064803F0BAFAE0
:1039C0000121044803F0C2FA0223EAE70742010892
:1039D000E0D90020908A00202DE9F043079EBDF831
:1039E00020C0DFF84CE0DFF84C800025ACB29C42F0
:1039F0001BD231F9129004F00704EF10B9F1000F57
:103A0000F05DB4BF18F804401EF8044002F105024E
:103A100092B2B4BF20432040624528BFA2EB0C0203
:103A2000F05528BF92B20135E0E7BDE8F08300BF52
:103A3000DA3B0108E23B01082DE9F04141F6CC53A5
:103A40000446C35A0133002550F83330504886B03D
:103A50005840294608F05CFE012818D84D494E48C8
:103A600007F02AFB29464D4803F064FA29464B48E3
:103A700003F06CFA484806F0D1FF41F6DC53E550FC
:103A800004F5EF531D60257006B0BDE8F08141F6E6
:103A9000D653E15A41F6D853E25A41F6D0539142F7
:103AA000E35A24D2994204D89A4202D32046FFF71F
:103AB000E3FE41F6E45834F80830952B1AD938491A
:103AC000354807F0F9FA0021344803F033FA0021B1
:103AD000324803F03BFA304806F082FF41F6DC52F0
:103AE0000023A35004F5EF5213602370CCE79942F2
:103AF000DAD8DBE741F6D05341F6D857E25AE35B18
:103B00009A42C1D14FF4F07341F6D25602AD0193FF
:103B1000009504F5D0516023A25B0C312046FFF7DD
:103B20005BFF34F808201521B2FBF1F301FB1323EE
:103B30009BB233BBA2B955238DF8113041F22D63EE
:103B4000ADF8123041F6D6531649E35E0193E35FB8
:103B5000009341F6D453A25FE35E0F4808F03CFBAC
:103B600029462046FFF71AFE41F6E452A35A0133D4
:103B7000A35241F6DC520023A35004F5EF54236016
:103B800082E70C222946044806F0FEFEECE700BF5F
:103B90005E13AAAA9D410108E0D90020908A002066
:103BA000BD410108E541010841F6E8532DE9F04F18
:103BB000C45841F6EC5304F0070250F803E00B68D8
:103BC0000EEB030841F6F4534746C6580B6906EB63
:103BD000030CE045A8BF6746E308E04500EB83031C
:103BE000B5BFDFF8F8C0DFF8F8C01CF802C01CF859
:103BF00002C041F6FC5941F6A46853F80950B4BF1D
:103C00000CEA05054CEA050543F809504D68AE4439
:103C10004D692E44B645F446A8BFB446B645B4BF78
:103C20002E4E2F4E53F80850B5BFB65CB65C3540EB
:103C3000354343F8085041F6F0558E6950F805E0D9
:103C40008D680EEB050A41F6F855D046455905EB4F
:103C50000609CA45A8BFC846CA45B5BFDFF87C906B
:103C6000DFF87C9019F8029019F8029041F64C7B2D
:103C700053F80B60B4BF09EA060649EA060643F8A2
:103C80000B60CE68C96976440D44AE4241F6F479C2
:103C9000B646A8BFAE46AE4253F8091019DA0F4D2A
:103CA000AA5C0A4043F8092041F6EC530134C7509E
:103CB00041F6F05340F803C041F6F45340F8038056
:103CC00041F6F85340F803E041F6E853C450BDE82C
:103CD000F08F034DAA5C0A43E4E700BFCA3B01082A
:103CE000D23B010870B5D1E9003288B083F00105FC
:103CF000D11882F001062A44334400917419CDE9A9
:103D00000512694601940293CDE903240793FFF756
:103D10004BFF08B070BD0000F0B500222F4D304FB2
:103D200040F24911134642F29C04032B1DD8DFE8F0
:103D300003F002203846CE1006F27E7601F007032B
:103D400000EB860615F803C073681CEA030318BF6E
:103D5000022300EBD20C02F007061CF804E0BE5D63
:103D600006EA0E060CF80460013211F1FF31DCD2D4
:103D7000F0BDCE1006F5F56601F0070300EB8606F0
:103D800015F803C073681CEA030318BF022300EB95
:103D9000D20C02F007061CF804E0AE5D46EA0E06FF
:103DA000E0E7CB1003F2D27300EB830301F00706C8
:103DB0005B68AE5D1E420CBF01230323C9E7CE1032
:103DC00006F2FC7600EB860601F0070C766815F823
:103DD0000CC01CEA060F08BF0123D8E7D23B01083C
:103DE000CA3B010830B5124D4FF0FF32481E01F1B9
:103DF000260410F8013F5340DBB2C2F3072235F826
:103E00001330844283EA02031A46F2D1DB439BB2A9
:103E100091F82700DAB2904207D191F82820B2EB4E
:103E2000132F0CBF0120002030BD0020FCE700BF95
:103E3000CA3901082DE9F0430546904899B0164665
:103E40004B1E01F1520413F8017F10F8012B9C4224
:103E500082EA07021A70F6D1002303AA184601333A
:103E6000542B02F8010BFAD1DFF818E20022744655
:103E700080270EEB4200B2F5257F64DB41F6EC5261
:103E80000024AC5041F6F0524FF08008AC5041F69F
:103E9000F4524027AC5041F6F852AC5041F6E8528B
:103EA000AC5018AB03EBE403284613F8542C04F091
:103EB000070328FA03F1114227FA03F314BF012183
:103EC0000021134214BF012300230291023401A9EF
:103ED0000193FFF707FFB4F5257FE2D1FFF71CFF41
:103EE000731E06F12802002103F8011F9A42FBD13C
:103EF00040F24912624F104642F29C044FF0010C0E
:103F000005EBE20102F0070811F804E017F80810C9
:103F10001EEA010FA0EB020309D0D90803F0070342
:103F200016F801E00CFA03F343EA0E03735412F19E
:103F3000FF32E5D231462846FFF754FF19B0BDE8FD
:103F4000F0831A4697E7D31011F803C01CF0010F55
:103F50000CD090F8008018AB9844437818F8549C23
:103F600027FA03F343EA090308F8543C1CF0020F54
:103F70000CD090F8028018AB9844C37818F8549C81
:103F800027FA03F343EA090308F8543C1CF0040F32
:103F90000CD090F8048018AB9844437918F8549CDE
:103FA00027FA03F343EA090308F8543C1CF0080F0E
:103FB0000CD090F8068018AB9844C37918F8549C3C
:103FC00027FA03F343EA090308F8543C131DB3F539
:103FD000257F00F10800B4DA1CF0100F0FD014F8A0
:103FE00013000DF1600804EB430340445B7810F8C4
:103FF000548C27FA03F343EA080300F8543C1CF0FE
:10400000200F10D0531D0DF1600814F8130004EBBD
:10401000430340445B7810F8548C27FA03F343EAD7
:10402000080300F8543C1CF0400F10D0931D0DF114
:10403000600814F8130004EB430340445B7810F865
:10404000548C27FA03F343EA080300F8543C1CF0AD
:10405000800F10D0D31D0DF1600C14F8130004EB89
:10406000430360445B7810F854CC27FA03F343EA27
:104070000C0300F8543C0832FBE600BFEA3B0108A1
:10408000D23B0108453C010870B541F6E655A2B0A7
:10409000435D04460E4623B1FFF7A0FB635D013B81
:1040A000635541F6CE52A35A03F1180001339BB277
:1040B00024F81060A35240F6E942934219D140F629
:1040C000E4430DAD0193052204F130012046009533
:1040D0004FF42573FFF780FC02AA29462046FFF71C
:1040E000A9FE78BB41F6DC532070E05004F5EF5395
:1040F000186041F6CE53E25A40F6EE439A421FD181
:1041000041F6E4530022E25241F6D0534FF0EE72F2
:10411000E25041F6D453124AE25041F6D8524FF4DD
:10412000EC73A3524FF4EB72CDE900320D490E4807
:1041300040F2D7134FF4EE7208F04EF802232370CA
:1041400022B070BD0121094802F0F4FE01210748A8
:1041500002F0FCFE02A92046FFF7FEFAC9E700BF05
:10416000D701D60128420108E0D90020908A00201A
:104170002DE9F04700F5EE5804460D4616461F4659
:104180004FF0000908F10C081FFA89F39F424AD941
:1041900042F2C80236F81910A3580B44A35042F259
:1041A000CC0241F6D05AA35A0133A352B8F80020EA
:1041B00035F9191004EBC202D2E90230DB18404194
:1041C0000029B8BF43F00103C2E9023034F80A30D5
:1041D00003F6045304EB430399802378012B05D0A5
:1041E000022B1CD02046FFF7C1FB02E02046FFF760
:1041F0004BFF34F80A3001339BB2B3F5F07F28BF90
:10420000002324F80A30B8F8003001339BB2042BA5
:1042100088BF0023A8F8003009F10109B4E720465F
:10422000FFF70AFCE5E7BDE8F087000070B504463B
:1042300000254FF4B9702581208065816573257351
:104240000CF042F8C4E9045504F11C066060A56155
:1042500004F14403324622F8025B9342FBD104F599
:104260002771002203F8012B9942FBD13C23C4F8AB
:104270009C22A4F8A0322822002130460CF05CF9E0
:104280000523237403236382024B2046C4E90536C9
:1042900070BD00BFBC0500202DE9F04F501E99B045
:1042A00003AD02F152090346002403F8014F99457A
:1042B00005F8014BF9D14B1E0093DFF8C0A1002394
:1042C0001D461C46009911F8016FAC46CDE9001659
:1042D00025461E460027012101FA07F401992142D3
:1042E00014BF0124002404EB0C0EAC44A4441CF0C5
:1042F000010F0EF0010E0CD006F0070C18A91AF8E9
:104300000C8001EBD60C1CF854BC48EA0B080CF8E6
:10431000548CBEF1000F0ED006F1010C18A901EB70
:10432000DC0E0CF0070C1EF8548C1AF80CC04CEA8A
:10433000080C0EF854CC0137082F06F10206AC46E3
:1043400040F088801033B3F5287FBBD1DFF830C14F
:104350000023644601250CEB4301B3F5257F7DD294
:1043600018AE06EBD30616F8546C37060AD591F84A
:1043700000E04F7812F80E8005FA07F747EA0807C1
:1043800002F80E7077060AD591F802E0CF7812F89D
:104390000E8005FA07F747EA080702F80E70B7061D
:1043A0000AD591F804E04F7912F80E8005FA07F764
:1043B00047EA080702F80E70F7060AD591F806E0FA
:1043C000CF7912F80E8005FA07F747EA080702F8D6
:1043D0000E701F1DB7F5257F01F108013CD2310792
:1043E0000BD514F817E004EB4707797812F80E7034
:1043F00005FA01F1394302F80E1071070CD5591D69
:1044000014F8117004EB410112F807E0497805FA3D
:1044100001F141EA0E01D155B7070CD5991D14F8E9
:10442000117004EB410112F807E0497805FA01F137
:1044300041EA0E01D155F1070AD5D91D14F81160D2
:1044400004EB4101975D497805FA01F13943915533
:10445000083380E725463EE73B467EE7064A10F8EC
:10446000011F12F8013B484583EA01030370F6D1AE
:1044700019B0BDE8F08F00BF514201084942010860
:10448000AC42010870B59AB00C460023012202A983
:1044900040F249354FF6B74632EA040C0CBF21F81A
:1044A000136021F8135001335200082BD2B2F3D11C
:1044B00006AA10300BF032F80023009306AA282336
:1044C0000121024803F00EF91AB070BD908A002055
:1044D00001EB4101490001F59671B1F5167F8ABFE4
:1044E0004FF41673A0F8A012A0F8A032704703464C
:1044F00000895A8992B2824203D11A7B02F0FF00EE
:1045000082B158685A8992B2825C0A70002119738C
:104510005A89013292B25A815A891888904298BFBA
:10452000598101207047000070B542890389B0F8B5
:104530009C529BB29342A2B0044620D1037B0BB1A4
:1045400003880BB9002D5BD0638962689BB2D35C92
:10455000002B4ED1002D56D15C4B1B78EBB9B4F833
:10456000A002AA22A9B28842B4F89C323DD9591CB3
:104570002344A4F89C12013583F84420F2E74389D0
:1045800002899A429DBF42890188038903898CBFB1
:1045900042895B189B1A9BB2D3E70DF103012046B9
:1045A000FFF7A5FF01AB591920460135FFF79FFF23
:1045B000292DF7D10DF13202204601A9FFF76CFE3B
:1045C0004AF2EA63ADF83030B4F89C320CA800220D
:1045D000991814FA81F1013210F8015B81F8445006
:1045E000552AF5D15533A4F89C320023A4F89E3205
:1045F00003E0012B06D0022B38D0B4F89C3213B95B
:1046000022B070BDE5B1324802F076FC0546282D97
:10461000F6D9B4F89E325A1C2344A4F89E2293F88B
:1046200044102046FFF72EFFB4F89E22B4F89C32C7
:10463000283D9A42ADB2EAD30023C4F89C32DFE7AA
:104640000CA92046FFF753FF0C25B4F89C124B1C15
:104650004431A4F89C3221442046013DFFF747FF36
:1046600015F0FF05F1D1A4F89E52C6E7002DCAD17E
:104670000CA92046FFF73BFFB4F89C3203F112016E
:1046800089B25522C8267A25E01880F84420581CA3
:1046900014FA80F080F84420981C14FA80F080F816
:1046A0004420D81C14FA80F080F84420181D14FA15
:1046B00080F080F84460581D063314FA80F09BB2F5
:1046C0008B4280F84450DFD18DE700BFCA9A0020AA
:1046D000908A002008B5FDF7C6FD0D23B0FBF3F06E
:1046E000C0B208BD037B10B503F0FF021BB101236C
:1046F0004373002010BD446803899BB2E1540389D1
:1047000001339BB2038103890188994298BF0281DA
:10471000028943899BB293424FF0010308BF0373A0
:104720001846E7E7292A70B506460C4619D1FDF769
:104730009AFD292806D802B20B490C4806F09EFFC4
:10474000052070BD00213046FFF7CCFF651E2834E0
:1047500015F8011F3046FFF7C5FFA542F8D100202C
:10476000EFE70420EDE700BFD4470108E0D90020BF
:104770000C2A70B506460C4619D1FDF774FD0C28BD
:1047800006D802B20B490C4806F078FF052070BD30
:1047900001213046FFF7A6FF651E0B3415F8011FF7
:1047A0003046FFF79FFFA542F8D10020EFE7042035
:1047B000EDE700BF11480108E0D9002010B504461C
:1047C000FDF751FD024628B90548064906F056FF97
:1047D000052010BD02212046FFF784FF0020F8E7E6
:1047E000E0D90020F447010800224FF48041026024
:1047F00081808271826002737047C9010180D20199
:104800004942418082807047B0F9003030B593B1A1
:10481000827932B98B420ADC0123837100238360E1
:1048200003738368B3F5166F07D900211AE0B0F956
:1048300002308B42F0DA084630BD047B0E49B0F9F5
:10484000045051F82410621CD2B20B2A027301FBEF
:1048500005F188BF00224FEAE13188BF027301F3FE
:104860000F0109B2013342F6DF6293428360E2D95D
:1048700000238371DFE700BF3048010838B500F638
:1048800078450446284602F0AAF8A0B1284602F06E
:10489000ABF880B10849094806F00EFC002384F803
:1048A0004C3C284602F091F804F6584002F08DF88E
:1048B000012384F8983C38BD6F490108E0D90020F5
:1048C000034670B5D0E90254D0E904026A431E6879
:1048D00000FB0122986906FB0022D8695E6800FB94
:1048E0001422186A06FB1020C01300F30E0000B259
:1048F000C3E90054C3E9021070BD38B50025044671
:1049000080F84C5C00F5456002F05FF804F6584012
:1049100002F05BF804F6684002F057F804F54760CF
:1049200002F053F804F6784002F04FF804F54860BE
:1049300002F04BF804F6884002F047F804F54960AD
:1049400002F043F804F5406001F026FD04F58060B4
:1049500001F030FF04F5006001F02CFF204601F06B
:1049600029FF04F5446002F017F8A4F8585D04F537
:104970005660A4F85A5D84F85D5D84F85C5D02F0D1
:1049800055F804F5526001F0F3FD04F6284001F0FB
:10499000C3FF84F8985CA4F8805D38BD2DE9F74F1B
:1049A0009DF834409DF830509DF83CB0C4EB0414A1
:1049B0009946A4009DF838300193A4B29DF8483080
:1049C00080F84F3C0F4690469DF840109DF84420DB
:1049D00080F84D1C00F5466A80F84E2C06460022F1
:1049E0002146504601F0DFFFC5EB0511890089B271
:1049F000002206F5456001F0D6FF14B1504601F0E3
:104A0000DFFF019B0C9342464B4639463046CDF8BA
:104A100034B003B0BDE8F04F01F0C2BD2DE9F0475E
:104A2000BDF824709DF820609DF828500446884603
:104A3000914600213A4600F678409A4601F0B3FFCD
:104A40002EB13A46314604F5476001F0ACFFCDE99E
:104A5000085553464A46414604F58060BDE8F04794
:104A600001F09EBD2DE9F04F85B01D469DF8383010
:104A700000939DF83C3001939DF84030029304462A
:104A80009DF85C309DF84CE09DF850C09DF85400B6
:104A90009DF844B0039316469DF864309DF8582065
:104AA000A4F81C3D84F818ED84F819CD9DF848A0B1
:104AB00084F81A0D84F81B2D04F6584000229DF846
:104AC00060709DF868909DF86C8001F06CFF00228A
:104AD000594604F6684001F066FF0022514604F58D
:104AE000486001F060FF314604F5446001F022FFA8
:104AF0003246494604F60850FFF77FFE3A460399CE
:104B0000A4F83E8D04F6284001F083FEDDE9002381
:104B1000294604F5406001F0B5FB40B9029A2946E8
:104B200004F5426005B0BDE8F04F01F03FBC05B0B0
:104B3000BDE8F08F70B401269DF81040A0F81E2D3E
:104B40001D4680F83C6DBDF80C302A46CDE9034483
:104B500000F5006070BC01F023BD000070B5044694
:104B60000D4600F5456001F033FF294604F6584034
:104B700001F02EFF294604F5466001F029FF294681
:104B800004F6684001F024FF294604F5476001F06F
:104B90001FFF294604F6784001F01AFF04F6884604
:104BA000294604F5486001F013FF2946304601F01C
:104BB0000FFF04F54960294601F00AFF304601F075
:104BC0000EFF68B1304601F00FFF48B194F84C1C5D
:104BD000044806F07FF93046BDE8704001F0F0BEB1
:104BE00070BD00BFE0D9002038B504460D46D9B1EC
:104BF00000F65845284601F0F2FE40B3284601F081
:104C0000F3FE20B31248134906F056FA042384F841
:104C10004C3C284601F0D9FE94F83C3DBBB10C4811
:104C2000BDE8384006F076B90B4802F083F9294612
:104C3000094802F08BF90949054806F03DFA0323BB
:104C400084F84C3C04F6784001F0BAFEE4E738BD45
:104C5000E0D90020BB480108908A0020CF48010815
:104C600070B5044600F678450E4699B10121144806
:104C700002F060F90121124802F068F91148124966
:104C800006F01AFA022384F84C3C2846BDE870402E
:104C900001F09BBE284601F0A2FE78B1284601F043
:104CA000A3FE58B10949074806F006FA284684F8D9
:104CB0004C6C01F08AFE04F65840E7E770BD00BF77
:104CC000908A0020E0D900205A4901086F49010864
:104CD00038B50446A9B100F65845284601F07FFED4
:104CE000E0B1284601F080FEC0B10D480D4906F044
:104CF000E3F9092384F84C3C2846BDE8384001F02C
:104D000064BE0748084906F0D7F9082384F84C3CEC
:104D100004F67840BDE8384001F052BE38BD00BF0F
:104D2000E0D90020034901081849010810B50446DC
:104D300061B10848084906F0BFF9072384F84C3CE4
:104D400004F67840BDE8104001F03FBEBDE81040D9
:104D5000FFF794BDE0D900208249010838B5044628
:104D60000D4699B90A4802F0E5F82946084802F0CC
:104D7000EDF80848084906F09FF9052384F84C3CF3
:104D800004F67840BDE8384001F01ABE38BD00BFD7
:104D9000908A0020E0D90020A248010870B504469E
:104DA00000F678450E4699B10121144802F0C2F888
:104DB0000121124802F0CAF81148124906F07CF9A4
:104DC000042384F84C3C2846BDE8704001F0FDBD4A
:104DD000284601F004FE78B1284601F005FE58B1DE
:104DE0000949074806F068F9284684F84C6C01F038
:104DF000ECFD04F65840E7E770BD00BF908A002044
:104E0000E0D90020BB4801086F49010810B50446ED
:104E100061B90748074906F04FF90A2384F84C3C6A
:104E200004F67840BDE8104001F0CABD10BD00BFD7
:104E3000E0D90020E948010810B5044661B10848EE
:104E4000084906F039F9092384F84C3C04F6784007
:104E5000BDE8104001F0B9BDBDE81040FFF70EBD40
:104E6000E0D900200349010838B500F5466504463D
:104E7000284601F0B4FD78B1284601F0B5FDA0B197
:104E80000A490B4806F018F9204601F0ACFC284608
:104E9000BDE8384001F094BD0548044906F00CF91E
:104EA0002046BDE8384001F09EBC38BD604801088E
:104EB000E0D9002070B5044600F668450E46E9B119
:104EC000284601F091FD002843D02249224806F0EF
:104ED000F3F8022384F84C3C284601F076FD94F860
:104EE0004D3CB3B394F84F3C9BB32046FFF7BCFF57
:104EF00004F54560BDE8704001F062BD174802F05E
:104F000019F83146154802F021F81549124806F003
:104F1000D3F8284684F84C6C01F057FD04F658404D
:104F200001F053FD04F5476001F04FFD04F54560C5
:104F300001F04BFD04F6884001F047FD012384F8A1
:104F4000983C94F83C3D23B10348BDE8704005F01F
:104F5000E1BF70BD5A490108E0D90020908A0020C5
:104F60006F49010838B504460D4699B300F6584517
:104F7000284601F034FDD8B1284601F035FDB8B11E
:104F80001E491F4806F098F8042384F84C3C04F5A9
:104F9000476001F01AFD284601F017FD04F5446052
:104FA00001F0F4FC94F83C3D13B1154805F0B2FF54
:104FB00004F54565284601F012FDF0B1284601F0E0
:104FC00013FDD0B12046FFF74FFF2846BDE838401B
:104FD00001F0F6BC0B4801F0ADFF2946094801F08D
:104FE000B5FF0949064806F067F8032384F84C3CEE
:104FF00004F6784001F0E4FCD4E738BDBB48010872
:10500000E0D90020908A0020CF48010870B50446FE
:1050100000F6784529B301212B4801F08BFF0121CF
:10502000294801F093FF2948294906F045F8022351
:1050300084F84C3C284601F0C8FC04F54565284638
:1050400001F0CDFC00283ED0284601F0CDFC002820
:1050500039D02046FFF708FF2846BDE8704001F030
:10506000AFBC284601F0BBFC0028E6D0284601F082
:10507000BBFC0028E1D01548164906F01DF804F5E0
:1050800047660B2384F84C3C304601F0A8FC18B16D
:10509000304601F0A9FC50B10F490C4806F00CF85D
:1050A00004F5806001F09FFB304601F08EFC28463D
:1050B00001F08BFC04F6584001F087FC04F54860D1
:1050C00001F07EFCB9E770BD908A0020E0D9002095
:1050D0005A490108334901084149010870B504469D
:1050E00000F668450E46E1B1284601F07DFCA0B30C
:1050F0001A491B4805F0E0FF072384F84C3C28467A
:1051000001F063FC94F84D3C3BB394F84F3C23B35F
:105110002046FFF7A9FE04F54560BDE8704001F0A8
:105120004FBC10490E4805F0C7FF284684F84C6C68
:1051300001F04BFC04F6584001F047FC04F54760D1
:1051400001F043FC04F5456001F03FFC04F68840A3
:1051500001F03BFC012384F8983C70BD82490108B2
:10516000E0D900206F49010838B5044669B300F65C
:105170005845284601F033FCA8B1284601F034FC1C
:1051800088B11849184805F097FF092384F84C3C6A
:1051900004F5476001F019FC284601F016FC04F5FF
:1051A000446001F0F3FB04F54565284601F017FC67
:1051B000B8B1284601F018FC98B12046FFF754FE1C
:1051C0002846BDE8384001F0FBBB0849064805F019
:1051D00073FF082384F84C3C04F6784001F0F0FBA0
:1051E000E1E738BD03490108E0D90020184901086A
:1051F00070B5044600F67845E9B12848284905F01D
:105200005BFF072384F84C3C284601F0DEFB04F5E5
:105210004565284601F0E3FB00283ED0284601F012
:10522000E3FB002839D02046FFF71EFE2846BDE8E4
:10523000704001F0C5BB284601F0D1FB0028E6D044
:10524000284601F0D1FB0028E1D01448154905F0AB
:1052500033FF04F547660B2384F84C3C304601F0DD
:10526000BEFB18B1304601F0BFFB50B10E490B48F0
:1052700005F022FF04F5006001F0B5FA304601F0B8
:10528000A4FB284601F0A1FB04F6584001F09DFB69
:1052900004F5486001F094FBB9E770BDE0D9002047
:1052A00082490108334901084D49010838B50446CF
:1052B0000D46B9B9154801F03DFE2946134801F0E5
:1052C00045FE1349134805F0F7FE052384F84C3CCE
:1052D00094F84E3C13B12046FFF7C6FD04F6784023
:1052E00001F06EFB04F54565284601F078FB58B1E6
:1052F000284601F079FB38B12046FFF7B5FD284676
:10530000BDE8384001F05CBB38BD00BF908A00208A
:10531000A2480108E0D9002038B5044600F67845D7
:1053200021B30121284801F005FE0121264801F0A2
:105330000DFE2648264905F0BFFE042384F84C3CA8
:10534000284601F042FB04F54565284601F047FB7D
:10535000002838D0284601F047FBA0B32046FFF7CD
:1053600083FD2846BDE8384001F02ABB284601F0FD
:1053700036FB0028E7D0284601F036FB0028E2D0B3
:105380001449124805F098FE0B2384F84C3C04F5B0
:10539000446001F001FB10490C4805F08DFE04F556
:1053A000806001F020FA284601F00FFB04F5476009
:1053B00001F00BFB04F6584001F007FB04F54860D0
:1053C00001F0FEFABFE738BD908A0020E0D9002046
:1053D000BB480108334901084149010838B5044672
:1053E00051B90F480F4905F067FE0A2384F84C3C79
:1053F00004F6784001F0E4FA04F54565284601F02A
:10540000EEFA58B1284601F0EFFA38B12046FFF71E
:105410002BFD2846BDE8384001F0D2BA38BD00BFA8
:10542000E0D90020E948010838B5044600F678457F
:10543000E1B12548254905F03FFE092384F84C3C9D
:10544000284601F0C2FA04F54565284601F0C7FA7E
:10545000002838D0284601F0C7FAA0B32046FFF74D
:1054600003FD2846BDE8384001F0AABA284601F0FD
:10547000B6FA0028E7D0284601F0B6FA0028E2D0B4
:105480001349114805F018FE0B2384F84C3C04F531
:10549000446001F081FA0F490B4805F00DFE04F558
:1054A000006001F0A0F9284601F08FFA04F547608A
:1054B00001F08BFA04F6584001F087FA04F54860D1
:1054C00001F07EFABFE738BDE0D9002003490108AA
:1054D000334901084D49010810B5044600F658400B
:1054E00001F06EFA04F54760BDE8104001F068BABB
:1054F000F8B50446174600F5456571B301212E48FD
:1055000001F018FD01212C4801F020FD2B492C4809
:1055100005F0D2FD022384F84C3C2A49284805F0C6
:10552000CBFD04F5806001F045F904F5006001F061
:1055300041F92046FFF7D0FF284601F050FA002835
:1055400038D0284601F050FAA0B32046FFF78CFC73
:105550002846BDE8F84001F033BA2AB11A49184884
:1055600005F0AAFD0723D6E700F54866304601F0AE
:1055700036FA0028E0D0304601F036FA0028DBD0B9
:1055800012490F4805F098FD304684F84C7C01F034
:105590001CFA04F6884001F018FA94F84E3C13B156
:1055A0002046FFF761FC284601F00FFA012384F83A
:1055B000983CC1E7F8BD00BF908A00205A49010815
:1055C000E0D900206E480108824901086F490108AE
:1055D00008B500F5566001F0C9FAF023B0FBF3F00E
:1055E000C0B208BD08B500F5566001F028FA0020E9
:1055F00008BD037B10B503F0FF021BB10123437309
:10560000002010BD446803899BB224F8131003895D
:1056100001339BB2038103890188994298BF0281BB
:10562000028943899BB293424FF0010308BF037381
:105630001846E6E770B518254D43002400F554667A
:10564000AC4205D000213046FFF7D3FF0134F7E725
:1056500070BD00002DE9F041044600F08CFF04F518
:10566000806000F088FF04F5006000F084FF04F51E
:10567000406000F0F9FD04F5426000F093FE04F68E
:105680002840002501F0BDF804F5446001F04AF916
:10569000C4F84C5C04F5456001F081F904F658400B
:1056A00001F07DF904F5466001F079F904F66840EF
:1056B00001F075F904F5476001F071F904F67840DE
:1056C00001F06DF904F6884804F5486001F067F9C7
:1056D00004F54967404601F062F9384601F05FF988
:1056E0004FF43573C4F8AC3CC4F8B43C4FF4B56225
:1056F000484BC4F8B02CC4F8B83C474AC4F8D82C7E
:1057000045F26833C4F8BC3C444AC4F8DC2C4FF47E
:105710000043C4F8D03CC4F8F43CC4F8FC3C44F664
:105720006C223F4BC4F8E02CC4F8003D3D4AC4F85D
:10573000F82C47F6E423C4F8043D84F8985CC4F8D8
:10574000A45CC4F89C5CC4F8A85CC4F8A05CC4F871
:10575000D45CC4F8C85CC4F8C05CC4F8CC5CC4F8C1
:10576000C45CC4F8EC5CC4F8E45CC4F8F05CC4F855
:10577000E85C04F60850FFF737F801264FF00113F4
:105780004FF4C871C4F81C3DC4F8186D04F552609C
:1057900000F062FE40F66113A4F8485DA4F8403DB5
:1057A000A4F84A5D84F83C5DA4F83E6D84F84C5D35
:1057B00084F84D5D41F2C2200AF086FD4FF4166375
:1057C000A4F8503DA4F8585DC4F8440DA4F85A5DFF
:1057D00084F85D5D84F85C5D4FF496500AF074FDCA
:1057E000C4F8540D04F5566001F009F92A46314613
:1057F0004046A4F8805D01F0D6F896222946384646
:1058000001F0D1F820466421FFF714FF2046BDE8DF
:10581000F08100BFF96BFFFF0080FFFF5D3BFFFFE2
:10582000B505FFFF0000FFFF70B518254D430024AC
:1058300000F55566AC4205D000213046FFF7D9FE91
:105840000134F7E770BD000038B5044600294BD09D
:1058500000F66845284601F0AEF8C0B1404941481D
:1058600005F02AFC012384F84C3C284601F0A8F8F6
:1058700094F84D3C2BB194F84F3C13B92046FFF7F8
:10588000F3FA94F84C3C013B012B0BD938BD364957
:10589000344805F011FC022384F84C3C94F84D3C4C
:1058A000002BEBD132212046FFF7BEFF2046FFF749
:1058B00013FE04F5456001F083F804F5496001F03A
:1058C00084F80121294801F035FB0121274801F026
:1058D0003DFB04F6884001F073F894F84C1C214815
:1058E000BDE8384005F0F6BA002ACFD000F668458A
:1058F000284601F060F8C0B11D491A4805F0DCFBEC
:10590000062384F84C3C284601F05AF894F84D3CA4
:105910002BB194F84F3C13B92046FFF7A5FA94F841
:105920004C3C063B012BB1D80AE012490D4805F06A
:10593000C3FB072384F84C3C94F84D3C002BEBD17F
:1059400032212046FFF770FF2046FFF7C5FD04F522
:10595000456001F035F804F5496001F036F8B8E724
:1059600077480108E0D900205A490108908A0020B0
:105970008C4801088249010838B590F84C3C04462F
:105980000B2B0AD8DFE803F00635393D4145494E77
:1059900053585D622046FFF757FF94F84C3C3BBBE1
:1059A00004F5806000F00FFF10BB04F5006000F00C
:1059B0000AFFE8B9204600F006FFC8B904F54965BA
:1059C000284601F00CF828B994F8983C13B1284601
:1059D00000F0F6FF284601F002F848B1284601F031
:1059E00003F828B1284600F0F0FF002384F8983C23
:1059F00038BD2046FFF75EFACFE72046FFF7B2FA40
:105A0000CBE72046FFF702FBC7E72046FFF74EFC37
:105A1000C3E72046FFF780FCBFE711462046FFF7AB
:105A20005DFBBAE711462046FFF79EFBB5E711463E
:105A30002046FFF7DDFBB0E711462046FFF7CEFC1E
:105A4000ABE711462046FFF7EFFCA6E72046FFF73D
:105A50004FFDA2E710B5044609B31849184805F0F0
:105A60002BFB02230121174884F84C3C01F062FA19
:105A70000121144801F06AFA04F6584000F0A0FF32
:105A800004F5496000F0A1FF04F6884000F098FF9B
:105A900094F84C1C0A48BDE8104005F01BBA5AB1F6
:105AA0000949074805F008FB072384F84C3C3221DC
:105AB0002046FFF7B9FEDFE710BD00BF5A490108D5
:105AC000E0D90020908A00208249010838B590F87A
:105AD0004C3C04460A2B0AD8DFE803F00609272BC2
:105AE0002F2F0933383D42002046FFF7B3FF94F8CB
:105AF0004C3CCBB904F54965284600F070FF28B945
:105B000094F8983C13B1284600F05AFF284600F05C
:105B100066FF48B1284600F067FF28B1284600F02C
:105B200054FF002384F8983C38BD2046FFF75CF80A
:105B3000DDE72046FFF794F8D9E72046FFF70EF996
:105B4000D5E711462046FFF7C3F8D0E711462046B7
:105B5000FFF7ECF8CBE711462046FFF757F9C6E709
:105B600011462046FFF768F9C1E7000070B504460A
:105B700015460E4611B390F8803DEBB901213B4824
:105B800001F0D8F90121394801F0E0F994F8813D9C
:105B90007BB93749374805F08FFA022304F688406D
:105BA00084F84C3C00F00CFF94F84C1C314805F094
:105BB00091F9012384F8803D0DB940E0EAB194F8F1
:105BC000813DCBB994F8803D7BB92B49294805F03C
:105BD00073FA072304F6884084F84C3C00F0F0FE8A
:105BE00094F84C1C234805F075F932212046FFF744
:105BF0001BFE012384F8813DBEBB94F8803DEBB1D0
:105C000000211A4801F096F90021184801F09EF988
:105C100094F8816D4EB91748184905F04DFA84F88B
:105C20004C6C04F6884000F0D0FE002384F8803DE0
:105C300094F83C3D13B10F4805F06CF9ADB994F8F8
:105C4000813D93B194F8805D4DB90A480B4905F048
:105C500033FA84F84C5C04F6884000F0B6FE012369
:105C600084F8983C002384F8813D70BD908A002020
:105C70005A490108E0D90020824901086F4901080A
:105C800090F8193D0BB1FFF771BF034B1B780BB1B7
:105C9000FFF772BEFFF71ABF3107002003460089E5
:105CA0005A8992B2824203D11A7B02F0FF008AB174
:105CB00058685A8992B230F912200A80002119736B
:105CC0005A89013292B25A815A891888904298BFF3
:105CD00059810120704700002DE9F04F9B4690F854
:105CE0001A3D85B004460E4690460BB181F0010680
:105CF00059462046FEF732FFAD4F08EB4B0B04F63A
:105D0000284AC34500F0518138F9021BB4F93E3DE1
:105D1000090291FBF3F194F81B3D09B2ADF80C10A8
:105D20001BB1504600F078FD06460DF10E0104F55A
:105D3000566000F0D9FE054608B194F83C5D94F831
:105D4000183D012B1CD09BB1022BBDF90C1004F5A2
:105D5000406000F0DC8000F0B3FA0DB950B166B1DC
:105D60003B780A2B09D000282A4608BF0146DFE00D
:105D70001DB916B93B780A2BC3D12A4631461CE01F
:105D8000BDF90C1004F5406000F09AFA04F5546374
:105D9000BDF90C10019381461846FFF72AFC019BC0
:105DA00003A91846FFF77AFF3B7855B9B9F1000F00
:105DB00007D10A2BA5D12A4649462046FFF760FFA6
:105DC0000AE00A2BF7D02A4649462046FFF758FF3B
:105DD00094F84C3C002B94D03B780A2B91D194F84A
:105DE0004C3C002B00F0AD8094F84C3CBDF90C10FD
:105DF000B4F91C5D9A1FD2B2012A03D8BDF90E1066
:105E0000B4F91E5D6B480078002800F0B680013BB5
:105E1000012B02D9012A00F2C38004F60850FEF7D4
:105E2000F3FC94F83C3D81464BB194F84C3C013B6B
:105E3000012B04D8014604F5526000F021FB19FB48
:105E400005F52DB2204600F0C0FC04F5806948B984
:105E500004F5006000F0B9FC20B9484600F026FCCB
:105E600005442DB2204600F0B0FC48B9484600F089
:105E7000ACFC28B904F5006000F018FC05442DB214
:105E8000484600F0A2FC78B904F5006000F09DFCE3
:105E900050B994F84C3CADB22046002B40F08280C3
:105EA00000F004FC05442DB2294604F69C40FEF7A0
:105EB00007FD014604F54C60FEF702FD014604F6BD
:105EC000E440FEF7FDFC0546204600F07EFC70B97C
:105ED000484600F07AFC50B904F5006000F075FC0B
:105EE00028B904F5446000F029FD05442DB204F5FD
:105EF000496000F074FD014604F5426000F09AFA32
:105F0000284401B204F55560FFF773FBF9E600F091
:105F1000D7F901463DB928B93B780A2B7FF4F1AE99
:105F20002A464AE75EB13B780A2B04D000292A466C
:105F300018BF314649E7002918BF3146F0E731461E
:105F4000EEE704F5806000F03EFC00287FF44CAFE3
:105F500004F5006000F037FC00287FF445AF2046D0
:105F600000F031FC00287FF43FAF04F5496000F0F9
:105F700036FD00287FF438AFC3E6012A02D811FBB2
:105F800005F55EE794F83C2D002A3FF4BAAE013BDC
:105F9000012B3FF6B6AE04F5526000F071FAB0E6A0
:105FA00000254FE700F0C4FB7CE705B0BDE8F08FAB
:105FB000C99A0020310700202DE9F04F994690F84A
:105FC0001A3D85B004460E4690460BB181F001069D
:105FD00049462046FEF7C2FD634F08EB490904F627
:105FE000284AC84500F0BC8038F9021BB4F93E3D90
:105FF000090291FBF3F194F81B3D09B2ADF80C10C6
:106000001BB1504600F008FC06460DF10E0104F5E8
:10601000566000F069FD054608B194F83C5D94F8BF
:10602000183D012B1BD093B1022BBDF90C1004F5C8
:1060300040607BD000F044F90DB950B166B13B78B7
:106040000A2B09D000282A4608BF01467FE01DB967
:1060500016B93B780A2BC4D12A46314619E0BDF95E
:106060000C1004F5406000F02BF904F5546B01901E
:10607000BDF90C105846FFF7BCFA03A95846FFF7C4
:106080000DFE019B3A7845B93BB90A2AA9D12A46A7
:1060900019462046FFF7F4FD0AE00A2AF7D02A46FF
:1060A00019462046FFF7ECFD94F84C3C002B98D0A5
:1060B0003B780A2B95D194F8803D6BB194F83C3D28
:1060C00053B1BDF90C1004F60850FEF79DFB0146D4
:1060D00004F5526000F0D4F994F8813D002B80D093
:1060E000BDF80E30B4F81E1D11FB03F109B204F621
:1060F0009C40FEF7E5FB014604F54C60FEF7E0FB33
:10610000014604F6E440FEF7DBFB054604F5496072
:1061100000F065FC014604F5426000F08BF9291897
:1061200009B204F55560FFF764FA5AE700F0C8F8C1
:1061300001463DB928B93B780A2B7FF452AF2A4675
:10614000A7E75EB13B780A2B04D000292A4618BF86
:106150003146A6E7002918BF3146F0E73146EEE7A1
:1061600005B0BDE8F08F00BFC99A002010B490F8C8
:10617000194D1CB15DF8044BFFF71EBF5DF8044BD1
:10618000FFF7AABD2DE9F0470446C0B0344800F03F
:10619000B3FEB4F85A2DB4F8583D9BB2934249D19E
:1061A00094F85C3D43B3B4F8502D0A2824D9632AEF
:1061B00022D9023885B2642D04AF4FF0000628BF03
:1061C0006425B946B04604F5556A01360DF10E0155
:1061D0005046B6B2ADF80E80FFF760FDBDF80E3048
:1061E00027F8023BB542F0D1CDF800802B464A4655
:1061F0000A211B4801F076FA94F83C3DBBB104F546
:106200005264204600F098F94F2810D904AD0026BA
:106210002F4629462046013600F06EF9502E05F132
:106220000305F6D1F02239460E4804F00BFE40B0CB
:10623000BDE8F087B4F85A3DB4F8582D9A429DBF96
:10624000B4F85A3DB4F8501DB4F8582DB4F8582D90
:106250008CBFB4F85A3D5218D21A92B2A5E700BFCB
:10626000908A0020E0D9002030B5002200240025CB
:10627000C0E90045C0E902220282C0E90522027796
:1062800030BD0000F0B500250024C0E900450B4DED
:106290002601775D8F4209D13544D5E9024554EA9C
:1062A0000501C0E9004505D10420F0BD0134322CC0
:1062B000EED1F9E7C0E902230020F6E7984901088A
:1062C0002DE9F743D0E90576D0E900254FEAE779D3
:1062D00007FB05F302FB0933A7FB028999444FEA48
:1062E000D87301EB610143EA490303F31E03C6EBD4
:1062F00043035E18038A876101339BB241F27071D8
:106300008B420446466103823DD190F81CE086FB37
:106310000601C30F43EA410387FB070187FB0667BA
:106320004FEAD07CF00F40EA470000F31E00C71789
:1063300045434CEA410C02FB0755A0FB020103F365
:106340001E030CF31E0C29446344C20F42EA4102AF
:1063500002F31E02A3EB4202A368BEF1000F00D0BD
:10636000E3689A42B4BF002101217145217706D02C
:1063700000911BB212B20649064805F0E6FE002362
:10638000C4E905332382207F03B0BDE8F08300BF5A
:10639000B84C0108E0D900200023C0E90533037799
:1063A000038270470022C0E9002270472DE9F047C0
:1063B0001F4D06461446002315F833208A4205D1A6
:1063C00015EBC30506D10420BDE8F0870133322B5D
:1063D000F2D1F8E730686B88B38008B109F09EFF0E
:1063E000B088400009F070FF04EB440A04EB8A0A0D
:1063F000002430602746B288BBB29A4215D92046A5
:1064000009F046FF4FEAE079A0FB0A010AFB0911F7
:10641000C30F43EA4103326803F30F03B9B20137F4
:1064200022F811306B681C44E5E70020CCE700BF80
:10643000D84C0108C3885A1C92B210B50468C280B7
:1064400034F91330848894429CBF0022C28009B181
:106450005B421BB2184610BD38B5002504460581C5
:10646000018045814573057301EB410009F02CFF64
:1064700004F110036060256125766361204638BD14
:10648000037EF0B501F5006143B1032B09D0013360
:10649000DBB2052B88BF00230376F0BD0903016141
:1064A000F5E702691143027B016102F0FF0522B1A9
:1064B0000122427300220261E9E74269446892F8CE
:1064C00000C057789678028902EB4202A11804F8BE
:1064D00002C002894F70013292B28E70028102892D
:1064E0000188914298BF05810189428992B28A420E
:1064F00004BF01220273DDE7034600895A8992B284
:10650000824203D11A7B02F0FF00A2B15A68588977
:1065100000EB400002441088088092788A700021C5
:1065200019735A89013292B25A815A891888904255
:1065300098BF598101207047428903899BB29342D9
:1065400005D1027B02F0FF0382B1008870474389C6
:1065500002899A429DBF42890389008803898BBFC3
:106560004089C018181A801A80B2704718467047C0
:106570000023037670470246002302F8013B00F235
:10658000E93102F8013B9142FBD1A0F8EA33C0F8AF
:10659000EC33A0F8F033C0E9FD33C0F8FC337047AA
:1065A0002DE9F74F0446DFF8008101930020A4F89D
:1065B000EA03C5B24D5D002D43D04FF0000C0C270F
:1065C0005FFA8CF67E4308EB060718F80660B6B350
:1065D000B5420CF1010CF2D197F808B04FF0000E63
:1065E0004FF0004C5FFA8EF5AB4528D9B4F8EA536A
:1065F0002C4B05F0070A04EBD50913F80AA07B68B9
:1066000099F801603CEA030340F2E2330CBF46EA2A
:106610000A0626EA0A069D4289F801600EF1010E7B
:1066200007D90023A4F8EA330425284603B0BDE8BF
:10663000F08F0135A4F8EA534FEA5C0CD2E7013041
:10664000B7E79DF83010D4F8F403A4F8FC139DF8D4
:106650003410A4F8FE13019B45F6C051B1FBF2F2D1
:10666000B1FBF3F3A4F8EE23A4F8F83308B109F072
:1066700055FEB4F8F80309F027FE0023C4F8F4032C
:106680001F464FF0010CB4F8F86398B28642CCD99B
:10669000D4F8F413B0EB560F34BF01F800C00F5418
:1066A0000133F0E778500108684E010830B5034621
:1066B0000078002839D0B3F8EC231C4DB3F8FA1356
:1066C00003EBD20002F0070440782C5D204007D095
:1066D000D3F8F443B3F9FC03645C0CB9404200B254
:1066E000B3F8F843013189B28C42A3F8FA139CBF86
:1066F0000021A3F8FA13B3F8F013B3F8EE43013115
:1067000089B28C42A3F8F0130FD80132B3F8EA43F0
:1067100092B200219442A3F8EC23A3F8F0139EBF99
:106720001970A3F8EC13A3F8FA1330BD78500108E0
:1067300030B503460078002839D0B3F8EC231C4D5F
:10674000B3F8FA1303EBD20002F0070440782C5D93
:10675000204007D0D3F8F443B3F9FE03645C0CB9CE
:10676000404200B2B3F8F843013189B28C42A3F839
:10677000FA139CBF0021A3F8FA13B3F8F013B3F88F
:10678000EE43013189B28C42A3F8F0130FD80132E5
:10679000B3F8EA4392B200219442A3F8EC23A3F8A1
:1067A000F0139EBF1970A3F8EC13A3F8FA1330BDD1
:1067B0007850010800230370A0F8EC33A0F8F03300
:1067C000A0F8FA33704700787047B0F8EC3343B95B
:1067D000B0F8F0332BB9B0F8FA03003018BF01203D
:1067E00070470120704708B50246FFF7EEFF38B941
:1067F00001231370A2F8EC03A2F8F003A2F8FA0345
:1068000008BD0022C0E900220281C0E90322828281
:106810007047C0E9001270472DE9F743D0E90376CD
:10682000394D0289076105FB07F34FEAE37901322D
:10683000DB0F92B243EA490303F31E03C6EB4303A3
:1068400003EB81113C2A0446C160028152D181FBD5
:106850000189037D4FEAD87040EA490087FB078928
:106860004FEAD87281FB076742EA490202F31E0C25
:10687000F20F42EA470202F31E026A43D71700F3FF
:106880001E00D20F604442EA470202F31E02A0EB50
:106890004202002B32D06068824206DA002106E014
:1068A000617D0131C9B2617502E0A17D0131A1753F
:1068B000617D092916D9A17D09298CBF00210121FB
:1068C00021758BB191B9A175009103B212B20F4934
:1068D0000F4805F03AFCA37D627D0E490C4805F097
:1068E000FDFB03E00021EBE70029EDD10023C4E923
:1068F00003332381207D03B0BDE8F083206882420A
:10690000CEDB1946CFE700BF4DC5FB3080500108F4
:10691000E0D90020A85001080023C0E90333037523
:10692000038170474FF480420280002282704260EF
:106930000272704701EB8101018070470246807846
:1069400010B5E8B1546842F6DF639C4219D9117A58
:106950000D4B108833F8113013FB00F3DB1303F3F6
:106960000F0318B24B1CDBB23B2B88BF0023137202
:10697000013445F6BF518C428ABF002354605360F6
:1069800010BD0020F4E700BFC4500108012383704C
:106990000023436003727047002383707047002216
:1069A000C0E90022704718235A4345F6C05303FB41
:1069B00001210160704700681823B0FBF3F07047B5
:1069C00003680BB1012343607047002343607047A5
:1069D00043681BB102680AB11944416070474068BE
:1069E000003018BF01207047036833B1406828B1F8
:1069F00083422CBF0020012070471846704738B5ED
:106A000000254FF46163044685820570C582C0E9A4
:106A1000015583810576457642F6302009F054FC15
:106A2000231D20612577A360204638BD0023838283
:106A30000370C38243600376437603777047032372
:106A4000B2FBF3F202EB42022DE9F0410A440124C9
:106A5000914227D0037E03F0FF0713B14476033140
:106A6000F6E70669838A91F8008091F801E091F8D1
:106A700002C003EB4303F51806F80380838A85F808
:106A800001E001339BB285F802C08382838A858945
:106A90009D4298BF8782858AC38A9BB2AB4208BF5A
:106AA0000476DCE7037F7BB9C28A838A9BB2934278
:106AB0000CD1027E02F0FF0302B18389B3F5967F09
:106AC00094BF002301230377BDE8F081C38A828A43
:106AD0009A429DBFC28A8189838A838A8CBFC28A77
:106AE0005B189B1A9BB2E9E70346007FF0B580B1C3
:106AF0001A781AB1032A35D000222AE09C8ADA8A51
:106B000092B2A24206D11C7E04F0FF0214B91A7799
:106B10001046F0BD1D69DA8A02EB4202AC18AF5C88
:106B20006678A57800221A76DC8A0134A4B2DC8269
:106B3000DC8AB3F80CC0A4451C4698BFDA8244F83E
:106B4000042F1F715E719D715A689C60120BA2F533
:106B500000620A801A780132D2B2052A88BF002268
:106B60001A70D6E75A68C2F30B02F0E7C18A838A2B
:106B700082899BB28B4208D1037E002B0CBF10464A
:106B8000002000EB400080B27047C38A818A99429E
:106B900087BF838AC08AC38A808A86BF8018C01A4A
:106BA000181A80B2824238BF0020EAE770B5044666
:106BB0000625002686F001063146204601F020F821
:106BC0003146204601F02CF83146204601F030F8DD
:106BD0003146204601F034F83146204601F038F8BD
:106BE0003146204601F03CF83146204601F040F89D
:106BF000013DFA21204601F079F815F0FF05D9D1C1
:106C00002946204601F014F82946204601F018F8DC
:106C10002946204601F01CF82946204601F020F8BC
:106C20002946204601F024F82046012101F000F811
:106C30002046FA2101F05AF82046012101F000F81F
:106C40002046FA2101F052F82046012101F000F817
:106C50002046FA2101F04AF82046012101F000F80F
:106C60002046FA2101F042F82046012101F000F807
:106C70002046FA2101F03AF82946204600F0F8FFB4
:106C80002046FA2101F032F82946204600F0E8FFBC
:106C90002046FA2101F02AF82946204600F0D8FFC4
:106CA0002046FA2101F022F82946204600F0C8FFCC
:106CB0002046FA2101F01AF829462046BDE8704026
:106CC00000F0B6BF2DE9F74F00254FF416760446C5
:106CD00085810570C5818680057445744FF4166002
:106CE00009F0F2FA4FF4FA73A382A583A060E5835A
:106CF00084F8215084F820504FF4FA6009F0E4FA47
:106D0000A585A061E585A68484F8305084F83150CB
:106D10004FF4966009F0D8FA1022A062294604F1D7
:106D2000340009F009FCC4E91155C4E91355C4E95C
:106D3000165504F1440304F1600A0193A4F8545079
:106D400004F1B002534623F8025B9A42FBD1C4E936
:106D50002D5504F1BC09A4F8B05004F5A4714A46BD
:106D6000002322F8023B9142FBD104F5AA78A4F853
:106D70004831C4E9533304F5F0714246002322F848
:106D8000023B9142FBD104F5F677A4F8E031C4E967
:106D9000793304F50A713A46002322F8023B914206
:106DA000FBD104F50D76A4F82832C4E98B3304F541
:106DB00021713246002322F8023B9142FBD104F5B7
:106DC0002475A4F88432C4E9A23304F547712B4634
:106DD000002223F8022B99424FF0000BF9D14FF417
:106DE0008043A4F81E334FF04023C4E9C833C4E9FC
:106DF000CA33C4F830334FF00823C4F834330123C6
:106E000084F83823C4F83C23C4F84033A4F844235E
:106E1000C4F8482384F81CB384F84CB31022002132
:106E2000019809F089FB01236363019BA3632C4B49
:106E3000E36384F840B050220021504609F07CFB07
:106E40000C23A4F85430274BE365C4F858A08C22D7
:106E50000021484609F070FB4FF02A0AC4F8B490AC
:106E6000DFF89090A4F8B0A0C4F8B8908C2200216C
:106E7000404609F061FBA4F848A1C4E953893C22CB
:106E80000021384609F058FB0623A4F8E031164BE0
:106E9000C4F8E831C4F8E47150220021304609F00A
:106EA0004BFB0A23A4F82832104BC4F830328C2252
:106EB0000021C4F82C62284609F03EFB0C4BC4F8B4
:106EC0008C322046A4F884A2C4F8885200F084FCD6
:106ED0002046FFF76BFE204603B0BDE8F08F00BFF1
:106EE000BC060020A2060020DA0500208E06002045
:106EF0003A060020E6050020C18B838B828A9BB274
:106F00008B4206D190F82030002B0CBF1046002099
:106F10007047C38B818B994287BF838BC08BC38B98
:106F2000808B86BF8018C01A181A80B2824238BF80
:106F30000020704738B5044C22788A420D4601D0B3
:106F400000F06EFE257038BDC89A002080F841130D
:106F50007047000070B5314D2B788B4204460E46C9
:106F600037D0013B092B09D8DFE803F00512161AC8
:106F70001E262208082A002100F05AFE731E092B43
:106F800026D8DFE803F021272C3136403B25254564
:106F9000002100F055FEF1E7002100F059FEEDE779
:106FA000002100F05DFEE9E7002100F061FEE5E769
:106FB000002100F065FEE1E7002100F073FEDDE74F
:106FC000002100F081FED9E70121204600F030FECB
:106FD0002E7070BD0121204600F032FEF8E701213D
:106FE000204600F035FEF3E70121204600F038FE90
:106FF000EEE70121204600F03BFEE9E701212046B3
:1070000000F03EFEE4E70121204600F04BFEDFE702
:107010000121204600F058FEDAE700BFC99A00209F
:1070200038B5057804464DB900F0FCFC0123237007
:1070300029462046BDE83840FFF78CBF38BD2DE912
:10704000F0439DF8409080F81C334FEAC919A0F82E
:1070500030939DF844909DF820309DF81C809DF859
:1070600024E09DF828C09DF82C709DF830609DF8B4
:1070700034509DF838404FEAC919A0F83293BDF951
:107080004C9009F50069DB01A0F83493BDF94890F4
:10709000A0F820339DF83C3009F500694FEAC81884
:1070A0004FEACE1E4FEACC1CFF01F601ED01E401D0
:1070B000DB01A0F836939DF85090A0F81E83A0F84D
:1070C00022E3A0F824C3A0F82673A0F82863A0F850
:1070D0002A53A0F82C43A0F82E3380F8389319B126
:1070E000C8F10008A0F81E83B2B1CEF1000ECCF1B9
:1070F000000C7F4276426D4264425B42A0F822E37C
:10710000A0F824C3A0F82673A0F82863A0F82A5397
:10711000A0F82C43A0F82E33BDE8F083B0F842333A
:10712000003318BF01230B70B0F84433003318BF8D
:10713000012313700023A0F84233A0F844337047B2
:107140000346002290F8210083F82120704703466F
:107150000022407C5A7470470023C0F848337047BF
:10716000D0F84803704790F84C0370474289038970
:107170009BB2934205D1027B02F0FF0382B10088EB
:107180007047438902899A429DBF428903890088DA
:1071900003898BBF4089C018181A801A80B27047C3
:1071A000184670472DE9F041D0F83C33027801339E
:1071B0008CB00446C0F83C33002A00F05881D0F867
:1071C00048234BF67F339A420FD9B14B1B785A1E96
:1071D000042A40F23F81063B012B03D800212046C0
:1071E000FFF7B8FE0023C4F84833D4F83C2345F633
:1071F000BF539A420BD994F84013002381F0010148
:10720000C4F83C3384F84013204600F0F9FC94F8AD
:10721000383323B1204600F0E7FC84F84C0304F136
:107220001400FFF7A3FF60B99A4B1A784AB118709F
:1072300094F81C13204600F0EBFC9749974803F0A4
:107240003BFF201DFFF792FF012840F21D8104AD96
:107250000DF10C0C00222E46674611460DF1140E5E
:1072600040F6FF78A089E3899BB2834201D1237C59
:107270007BB1A368E08903EB800318682174E3897C
:107280000A9001339BB2E381E389A088984298BFBA
:10729000E1819DF82A300CF8013BA08DE38D9BB273
:1072A000834202D194F830308BB1A06AE38D9BB257
:1072B00030F8133084F830102EF81230E38D01339B
:1072C0009BB2E385E38DA08C984298BFE18594F84A
:1072D000413363B1BDF828309BB21BB1BDF82830F3
:1072E000984504D1B4F842330133A4F84233BDF8D1
:1072F0002830B4F83403181AB4F81E3313FB00F323
:10730000DB1303F30F0325F8023B002A00F0EE80A5
:1073100094F84C33002B40F0B780022208A9304685
:1073200008F0CCF802230AAA08A904F1340008F0F6
:1073300095FEDDE90A32134403EBD373BDF8102048
:107340005B1403F30F039BB2D21AADF81820BDF8FB
:107350001220D31AADF81A304D4B1D78002D40F095
:10736000CE804F4B1B7863B1022307AA06A904F114
:10737000540008F0CFFA022305AA07A94948FCF7F0
:10738000F7FE494B1B7863B1022307AA06A904F54F
:10739000F07008F0BFFA022305AA07A9434802F0DB
:1073A00009FD434B1B7863B1022307AA06A904F524
:1073B0000A7008F0AFFA022305AA07A93D4801F0B8
:1073C00059FE3D4B1B7883B1022307AA314604F1D5
:1073D000B00008F09FFA394B1B78002B00F0888032
:1073E000022207A93648FBF72BF9364B1B7863B10D
:1073F000022307AA06A904F5A47008F08BFA022359
:1074000005AA07A9304805F0E9FC304B1B7863B1A9
:10741000022307AA06A904F5217008F07BFA0223CB
:1074200005AA07A92A4800F0EBFF2A4B1B7843B1B5
:10743000204600F0D9FB0223014606AA2648FEF7A3
:1074400095FE264B1B78FBB1022206A92448F9F7CA
:107450004DFA19E0022B7FF4C1AE0E4B1B78002BC6
:107460003FF4BCAE00211F48FBF72CFEB6E61E49D8
:107470008B4209D990F84013C0F83C2381F00101F8
:1074800080F8401300F0BCFB0CB0BDE8F08100BFF9
:10749000C99A0020CA9A002042510108E0D9002070
:1074A000300700209059002035070020DCAF002075
:1074B00034070020CC9A00202F070020310700203D
:1074C000AC3600203707002010DC002033070020F6
:1074D000E08D002032070020087D00202E070020CC
:1074E000880A0020A45800207FA903000122B9E6E1
:1074F000022305AA07A95748FAF79CFD75E7012D55
:1075000011D1554B1B78002BBED007AA06A904F158
:107510005400022308F0FEF9022305AA07A94F48E8
:10752000FCF726FEB0E7022D25D14D4B1B78002B32
:10753000AAD02B4607AA314604F1B00008F0EAF9B8
:10754000484B1B7883B1484B1B783BB100953B46B9
:1075500005AA07A94548FBF791F895E72A4607A928
:107560004348FBF76DF88FE72B4605AA07A9394872
:10757000FAF760FD88E7032D11D13E4B1B78002BF5
:1075800082D007AA06A904F5A470022308F0C2F964
:10759000022305AA07A9384805F020FC74E7042D4A
:1075A00012D1364B1B78002B3FF46EAF07AA06A909
:1075B00004F5F070022308F0ADF9022305AA07A92B
:1075C0002F4802F0F7FB5FE7052D12D12D4B1B78FA
:1075D000002B3FF459AF07AA06A904F50A7002234D
:1075E00008F098F9022305AA07A9274801F042FDEF
:1075F0004AE7072D12D1254B1B78002B3FF444AFEF
:1076000007AA06A904F52170022308F083F90223D2
:1076100005AA07A91E4800F0F3FE35E70A2D3FF43E
:1076200007AF632D0CD107AA314604F154000223A1
:1076300008F070F9022207A91648F9F795FD23E72B
:10764000602D7FF421AF022205A91348FAF758F8FC
:107650001AE700BFFC1A00203007002090590020D4
:107660002F07002031070020CA9A0020FC3B002091
:10767000AC3600203707002010DC00203507002042
:10768000DCAF002034070020CC9A00203307002014
:10769000E08D0020A41600200017002013B5037B06
:1076A000019103F0FF0223B101234373002002B0D4
:1076B00010BD446803899BB244F823100389013349
:1076C0009BB2038103890188994298BF0281028994
:1076D00043899BB293424FF0010308BF03731846DE
:1076E000E5E700002DE9F347984603780A9D044634
:1076F0000E461746002B66D090F84C33002B62D113
:10770000324B1A7852B990F81C13012251401A706A
:1077100000F07EFA2E492F4803F0CEFC711E0A2994
:1077200046D8DFE801F0062D3033363C3945453F79
:107730004200B4F922934FF0000A04F11406D04538
:1077400041D037F81A30B4F8362313FB09F3DB13B2
:1077500003F30F0313449BB2B3F5805F22BFB4F869
:1077600044230132A4F844232DBBADF800308DF83A
:10777000025000993046FFF791FF0AF1010ADEE757
:10778000B4F92493D7E7B4F92693D4E7B4F928934E
:10779000D1E7B4F92A93CEE7B4F92C93CBE7B4F947
:1077A0002E93C8E7B4F93093C5E7B4F93293C2E732
:1077B000B4F92093BFE7ADF8043015F80A308DF81E
:1077C00006300199D6E702B0BDE8F087CA9A0020DA
:1077D0003C510108E0D900202DE9F7430225414E34
:1077E000414F684606F096F84FF400732846012191
:1077F0000124ADF806308DF8055006F079FC4FF401
:1078000000536946304600938DF8044006F034F882
:107810002146284606F06CFC4FF48043694630460A
:1078200000938DF8044006F027F82146204606F024
:107830005FFC4FF0200969463846CDF800908DF87E
:10784000044006F019F82146284606F051FC4FF492
:10785000004300936946002330468DF8043006F05B
:107860000BF82146284606F043FC4FF48068694631
:107870003046CDF800808DF8044005F0FDFF21462C
:10788000284606F035FC10236946304600938DF8F3
:10789000044005F0F1FF2146284606F029FC694620
:1078A0003046CDF800908DF8044005F0E5FF214604
:1078B000284606F01DFC08236946304600938DF8E3
:1078C000044005F0D9FF2146204606F011FC694628
:1078D0003846CDF800808DF8044005F0CDFF03B0A8
:1078E000BDE8F083000402400000024037B54FF4C9
:1078F0000063ADF8003000238DF80230828BC38B1B
:107900009BB29342044602D190F820308BB1A36918
:10791000E28B03EB82030022186884F82020E38BBB
:10792000009001339BB2E383E38BA18A994298BF15
:10793000E283BDF80010002005F0AAFE02212D48C8
:1079400005F019FE00BBADF80000022105462948EC
:1079500005F017FE274805F03BFD237C009A0192B5
:1079600003F0FF01CBB10123637494F8303003F0CE
:10797000FF0243B3012384F83130D4F84833013394
:10798000C4F8483303B030BD1A4805F04DFDADF8DA
:107990000000194805F048FDD7E7A068A3899BB20D
:1079A00040F82320A38901339BB2A381A389A28835
:1079B0009A4298BFA181A289E3899BB2934204BFF6
:1079C00001232374D1E7A16AA38D9BB221F8135040
:1079D000A38D01339BB2A385A38DA18C994298BF3F
:1079E000A285A28DE38D9BB2934204BF012384F84C
:1079F0003030C2E7002001400021014008B50121DC
:107A00004FF0804007F09FF948B14FF080400121CE
:107A100007F0A4F90248BDE80840FFF767BF08BDBA
:107A2000908A0020F0B5022195B0694805F0A3FDC9
:107A300010B16848FFF75AFF01A805F06BFF06A8D0
:107A400005F048FC0EA805F027FC0121084606F0C9
:107A50004FFB01214FF480700124002506F080FBCC
:107A6000032601A95C4801948DF808608DF80B503D
:107A700005F002FF2146204606F03AFB21464FF46E
:107A8000007006F06DFB022701A9534801978DF89D
:107A900008608DF80B5005F0EFFE062306A8CDE92F
:107AA0000635CDE9085505F001FC0EA948480E95AC
:107AB000ADF83C50CDE9105512958DF84C4005F0CD
:107AC000C5FB2146424805F08CFC2B462246294640
:107AD0003F4805F037FC21463D4805F001FC0EA962
:107AE0003E4805F0B3FB21463C4805F07AFC2246AF
:107AF0002B462146394805F025FC2146374805F03C
:107B0000EFFB01A805F006FF0AA805F073FD21466A
:107B1000204606F0EDFA21464FF0005006F012FB29
:107B2000102301A92C4801938DF808608DF80B50A3
:107B300005F0A2FE0AA92846CDE90A550D9505F0E3
:107B400043FD2146284605F05BFD2146204606F010
:107B5000F9FA22460F21204805F015FF4FF40043A3
:107B600001A91D4801938DF8087005F085FE03A852
:107B700006F074FDF92303A94FF08040CDE90334EA
:107B8000ADF814508DF8165006F02AFD2B462A4603
:107B900029464FF0804007F05EF921464FF08040C3
:107BA00006F0ACFD224621464FF0804007F0B7F8C2
:107BB0000B4B0093684605F0EBFA4FF480410948FF
:107BC00005F0D4FE2021044805F0CEFE15B0F0BD2E
:107BD00000200140908A0020000002400021014066
:107BE0001C0001010004024008B54FF400410348A5
:107BF00005F0A8FE431E5842584108BD000402404B
:107C00000A460248202105F0B3BE00BF0000024032
:107C10000A4602484FF4005105F0AABE0004024093
:107C20000A4602484FF4804105F0A2BE000402401B
:107C30000A4602484FF4806105F09ABE00040240F3
:107C40000A460248102105F093BE00BF000402401E
:107C50000A460248202105F08BBE00BF0004024006
:107C60000A460248082105F083BE00BF0004024016
:107C70000A4602484FF4806105F07ABE00000240D7
:107C800038B5074C0D460A4620464FF4806105F092
:107C90006FFE2A4620460821BDE8384005F068BE40
:107CA0000004024038B5074C0D460A4620464FF402
:107CB000806105F05DFE2A4620461021BDE838406F
:107CC00005F056BE0004024038B5074C0D460A4682
:107CD00020464FF4806105F04BFE2A4620462021C5
:107CE000BDE8384005F044BE00040240064B1A6867
:107CF00040F6B833B2FBF3F221B11346013BFDD19C
:107D00000139F9E7704700BF3009002002207047B1
:107D100008460C22014908F075BB00BF107AFF1F0E
:107D2000002303608380821D00F2867122F8023BEB
:107D30008A42FBD1154AC0F88827154AA0F8863731
:107D4000C0F88C27C0F89027C0F89437C0F898374F
:107D500000F2BC7100F29C73002223F8022B8B42CC
:107D6000FBD1A0F8BC2700F2DE7100F2BE72002346
:107D700022F8023B9142FBD16322A0F8DE3780F863
:107D8000E027C0F8E437A0F8E837704700000F2775
:107D90000F270F27632280F8E0270C4AC0F88827B6
:107DA00000230B4A0370A0F8BC37A0F8DE37A0F818
:107DB0008637C0F88C27C0F89027C0F89437C0F8F1
:107DC0009837C0F8E437A0F8E837704700000F276D
:107DD0000F270F27F7B5384E4FF47A5304464FF06C
:107DE000000C1F4630461FFA8CF5AA421ED904EB40
:107DF0004105B5F90650002D11DDA842B8BF28464F
:107E0000AF42A8BF2F464D1DADB2B5F5707F24BF60
:107E1000A1F2BB318DB20CF1010C2946E3E7AB4274
:107E2000A8BF2B46AE42B8BF2E46ECE7C21933447A
:107E300052105B10D5186D102EB2551B2DB21BB20F
:107E40001E491F48CDE9006512B204F0C5F994F847
:107E5000E037632B04F29C7104F2BC701FD10B4617
:107E600023F8026B98421D84FAD1002384F8E0378E
:107E70000023A4F8BC37A4F8DE371A4631F9025BB8
:107E80002A440D8C88422B4412B21BB2F6D1121137
:107E90001B11A4F8BC27A4F8DE3703B0F0BD04EB37
:107EA00043020133DBB20F2BA2F89C67A2F8BE5746
:107EB00084F8E037D9D8DBE780C1FFFF1B52010807
:107EC000E0D900202DE9F04F85B0DFF8B4B0BDF95E
:107ED00040A0BDF93C400294BDF838500192CAF16F
:107EE00000044FF000090394019A1FFA89F49442A8
:107EF00043D200EB410405F1010CE688029C039A91
:107F0000361B1FFA8CFC4FEAE50805F0070736B26E
:107F10004FEAEC040CF0070C0235964213F808E027
:107F20001BF807701BF80CC0ADB207DA2EEA070782
:107F300003F808701E5D4CEA060C08E0002E14DA07
:107F40002EEA070703F808701E5D26EA0C0C03F8FA
:107F500004C04C1DA4B2B4F5707F24BFA1F2BB31A4
:107F60008CB209F101092146BEE74EEA070703F882
:107F7000087056451E5DDEDAE7E705B0BDE8F08F14
:107F8000495101082DE9F0479846B0F88637034477
:107F90000446587886B04840154604F095FB9DF895
:107FA0003830984200F29180B4F88837484803F29C
:107FB0009D37BFB2B7F5707F24BFA3F12307BFB2CF
:107FC00005F1FF3CEA1D394600254FF47A534FF680
:107FD000FD7E4FF0030904EB41061CF901AFB6F931
:107FE0000660B042B8BF3046B342A8BF3346BAF1CC
:107FF000010F65D0BAF1030F04D0BAF1FF3F61D190
:10800000354401E016FB0E554E1DB6B2B6F5707F35
:1080100026BFA1F2BB3189B231469445DBD1D4F8F9
:108020009427AA4251DA94F8E027632A0AD103443C
:108030005B10A4F8BC37C31A44F63E104343DB136D
:10804000A4F8DE37B4F9DE3702930026B4F9BC3762
:1080500001930822394605AB20460096FFF732FF10
:1080600098F800309DF81400584004F02DFB98F863
:10807000013081469DF81500584004F025FB9DF81D
:108080003C304844C0B283421FD30423A4F898373D
:10809000B4F88837A4F88E3703F2973292B2B2F56B
:1080A000707F28BF293BC4F89457A4F88A7734BF5F
:1080B000A4F88C27A4F88C37012006B0BDE8F0871F
:1080C000AD1BA1E716FB09559EE70020F5E700BFB1
:1080D00080C1FFFF73B50025CDE900552C4B2D4A1B
:1080E000F2210446FFF74EFFCDE9005506462A4B24
:1080F0002A4A0D212046FFF745FF054606B9E0B1A3
:1081000094F89A37CBB9C4F8E437A4F8E8370121DA
:108110002348FEF70FFF01212148FEF717FF6323D5
:1081200084F8E037052384F89A3716B1012384F8E0
:108130009B3715B1022384F89B3794F89A3723B301
:10814000013BDBB2012B84F89A371ED1B4F88E378D
:1081500003F2BF3292B2B2F5707F28BF03F1FF3253
:10816000A4F890275A1C92B2B2F5707F24BFA3F2F4
:10817000BF33A4F8923794F89B3723704FF0000375
:1081800038BFA4F89227A4F89A3702B070BD00BF98
:108190005551010867510108535101085F51010809
:1081A000908A002010B50446B0F8E80798B1D4F8DA
:1081B000E437B3FBF0F3C3F3072081F8310081F813
:1081C00032303322054802F0A5FD0023C4F8E4371D
:1081D000A4F8E83710BD3122F4E700BFE0D9002051
:1081E00010B50446B0F8E80798B1D4F8E437B3FB0B
:1081F000F0F3C3F3072081F8310081F832303322E5
:10820000054802F0B5FD0023C4F8E437A4F8E837C8
:1082100010BD3122F4E700BFE0D90020F0B5B0F87E
:108220009017B0F89227B0F88837914293B004467F
:1082300080F0A080994239D89A4237D3012602258E
:10824000CDE90065644B654A0D21FFF79BFECDE942
:1082500000650746624B634AFD212046FFF792FE08
:1082600007B1257010B3B4F9DE37B4F98E27009347
:108270005D49B4F9BC375D4803F067FF00215C48F5
:10828000FEF758FE00215A48FEF760FE574802F0FC
:108290009DFD42F20F720023A4F88C276322237005
:1082A00084F8E027A4F89A37C4F89437B4F88827FC
:1082B000B4F88C379A425BD1B4F89837042B16D1B6
:1082C000B4F88E3703F2BF3292B2B2F5707F28BF96
:1082D00003F1FF32A4F890275A1C92B2B2F5707FD6
:1082E0002ABFA3F2BF33A4F89227A4F89237C02282
:1082F000B4F88A172046FFF76DFD2178B4F9BC3732
:10830000B4F9DE27012942D0022948D0B4F9DE377A
:108310000293B4F9BC37019308230093C02205AB44
:10832000B4F88A172046FFF7CDFDB4F89857013D01
:10833000ADB2A4F89857002D36D12E492B4802F043
:10834000BBFE29462A48FEF7F5FD29462848FEF7D8
:10835000FDFD264802F058FD42F20F73A4F88C3759
:108360006323257084F8E037A4F89A57C4F894572B
:1083700013B0F0BD994201D99A4297D30126022544
:10838000CDE90065144B154A0D2120465DE70092AA
:108390001949B4F98E27154803F0D7FEB6E70092C5
:1083A0001649B4F98E27F6E7EB1E5D425D4123784E
:1083B0008DF81450012B07D0022B09D00023C4F8EC
:1083C000943784F89B37D3E705A9FFF7EBFEF5E771
:1083D00005A9FFF705FFF1E7535101085F510108B7
:1083E00051510108575101086F510108E0D900208F
:1083F000908A0020FA5101089A510108CC510108D5
:108400002DE9F04104460D46971E01EB4308002676
:1084100045453ED037F8022FD4F8E43735F9021B32
:108420001344C4F8E437B4F88627B4F8E837224494
:108430000133A4F8E83753785B00DBB20029B8BFFA
:1084400043F001035370B4F8883704EB430320462C
:10845000D9802378013B012B18D8FFF7DFFEB4F851
:10846000883701339BB2B3F5707F38BFA4F88837E3
:10847000B4F8863728BFA4F8886701339BB2042B71
:1084800094BFA4F88637A4F88667C1E7FFF722FEF9
:10849000E5E7BDE8F081000070B5044600254FF423
:1084A0007A602581208065816573257307F00CFF54
:1084B000C4E9045504F11C066060A56104F13C03A5
:1084C000324622F8025B9342FBD104F2EC410022D7
:1084D00003F8012B9942FBD1F023A4F8F0344FF4B8
:1084E0009653C4F8EC24C4F8F434C4F8F8240021FA
:1084F0002022304608F020F80523237409236382E4
:10850000024B2046C4E9053670BD00BFD4060020EA
:10851000F0B58FB00A46002302A94FF4F77540F278
:10852000C9564FF637274FF6126C02F0C004802C64
:108530001DD0C02C18D0002C0CBF64463C4621F83E
:10854000134001339200042BD2B2EED104AA1030B2
:1085500006F0E4FF0023009304AA14230721054832
:10856000FFF7C0F80FB0F0BD21F81360E9E721F87C
:108570001350E6E7908A002010B58EB0002404AABC
:1085800002A904231030CDE9024406F0C7FF00948D
:10859000142304AA07210248FFF7A4F80EB010BD67
:1085A000908A002070B5B0F8EC3404461BB34948FB
:1085B000494EFEF7A1FC0546142D1BD9B4F8EE3444
:1085C0005A1C2344A4F8EE2493F83C102046FFF7ED
:1085D0009FFF3378143DADB21BB1D4F8F434C4F826
:1085E000F834B4F8EE24B4F8EC349A42E4D300231F
:1085F000C4F8EC3470BD428903899BB293422DD1FB
:10860000037BA3B1038893B1344B1B78002B3BD180
:10861000B4F8F054772198B2A842B4F8EC242BD3E4
:108620000023A4F8EE34B4F8EC34002BBFD1D4F816
:10863000F834002BDED02748FEF75EFC0546142DEB
:10864000D8D92046FFF798FFD4F8F834143D013B01
:10865000ADB2C4F8F834002BF1D1CBE743890289DD
:108660009A429DBF42890188038903898CBF428950
:108670005B189B1A9BB2C6E7501C2244A4F8EC047A
:10868000013382F83C10C6E730230020218962893B
:1086900092B28A4203D1227B02F0FF016AB1616883
:1086A000628992B2895C20736289013292B26281DE
:1086B00062892588954298BF6081B4F8EC24013B1B
:1086C000551C224413F0FF03A4F8EC5482F83C102C
:1086D000DCD1A5E7908A002031070020CA9A00204B
:1086E00001EB4101890001F51671B1F5966F8ABF62
:1086F0004FF49663A0F8F014A0F8F03470474FF4EC
:1087000096635943C0F8F414704708B5F9F7ABFD08
:108710003023B0FBF3F0C0B208BD312AF8B50446EF
:108720000D4624D1F9F79FFD2F2822D901231946A0
:10873000227B02F0FF002AB161730133312BF7D1A4
:108740000020F8BD66682289EF5C92B2B754228996
:10875000013292B2228122892688964298BF2081D6
:108760002089628992B2824208BF2173E5E7042022
:10877000E7E70520E5E70000014802F0C9B800BFBF
:10878000E0D9002010B55048504C03F0B9FB5048D8
:10879000FEF708FD4F4B1B782BB12378012B02D13C
:1087A0004D48FBF7C1FE4D4B1B784BB12378022B94
:1087B00006D14B4B1B78002B7BD04A48FAF7CCFEF6
:1087C000494B1B782BB12378032B02D1474804F087
:1087D000E9FB474B1B782BB12378042B02D145488A
:1087E00001F004FC444B1B782BB12378052B02D1FC
:1087F000424800F037FD424B1B782BB12378072B02
:1088000002D14048FFF7CEFE3F4B1B782BB12378B7
:10881000062B52D13D4801F05DFD3D4B1B7833B135
:1088200023780BB10A2B02D13A48F8F78FF93A4B6B
:108830001B782BB123780A2B02D13848FDF7A2FC14
:108840002378632B02D13648F8F7C2FC23785C3BCF
:10885000DBB2062B07D84D2222FA03F3DB0702D541
:108860003048F8F7ABFB2378663B052B02D82E483F
:10887000F8F7DCFD23785D2B02D12C48F8F7DCFEFD
:1088800023785B2B02D12A48F8F798FE23786C2BCB
:1088900002D12848F8F76AFE2378652B02D12648D2
:1088A000F8F708FF237873B92448BDE81040F8F7BB
:1088B00071BF2348F9F744FC82E7144801F0FEFC3D
:1088C0000028A7D1A9E710BDE0D90020C99A00204F
:1088D000908A002030070020607A00202F070020B7
:1088E00031070020A45800203707002050EF002057
:1088F0003507002020D200203407002048AA00209D
:1089000033070020CC95002036070020A0D7002098
:108910002E0700201414002032070020087D0020BC
:10892000E416002078160020E8160020FC1600202F
:10893000F9160020F8160020FE1600200C17002063
:10894000B831002008B5FFF717FFFFF71BFFFCE762
:1089500008B52F48FAF752FE2E48FBF767FC2E4861
:10896000F8F770FB2D48F8F72EFC2D48F9F7CEFCF0
:108970002C48F9F776FE2C48FAF7DEFA2B48F8F780
:10898000D1FF2B48F9F772FB2A48F8F70FFA2A486B
:1089900003F0E6FE294804F06BFA294800F060FD78
:1089A000284801F05FFA2848F8F742FE274800F00F
:1089B0006DF8274800F0AAFB2648F8F7FAFD26488C
:1089C000FFF7AEF92548FFF767FD2548F8F7CBFD1F
:1089D000244801F0FDFB2448F8F768FE2348FCF723
:1089E00039FE2348F8F71AFD2248F7F7EFFE224830
:1089F000F8F76BF82148F8F77CFE2148F8F7BAFE43
:108A0000204801F039FD2048BDE80840FEF75AB97A
:108A100090590020607A0020A4160020E41600205F
:108A2000AC360020FC3B0020A4580020FC1A00209B
:108A3000B83100207816002010DC002050EF002014
:108A4000DCAF002020D20020FC160020CC9A0020B1
:108A500048AA0020F9160020E08D0020CC950020C7
:108A6000F8160020A0D70020FE160020087D002068
:108A7000E8160020880A00201414002000170020A7
:108A80000C170020E0D90020908A00200246002127
:108A900002F8021B00F1160322F8021B9342FBD1DD
:108AA00000F61671002223F8022B9942FBD1184BD5
:108AB000C0F8183F174BC0F81C3FC0F8203F4FF0DC
:108AC0000003A0F8162FC0F8242FA0F8282F80F854
:108AD0002A3F00F64C7100F62C73002223F8022B7B
:108AE0009942FBD1A0F84C2F00F66E7100F64E7241
:108AF000002322F8023B9142FBD16322A0F86E3F93
:108B000080F8702FC0F8743FA0F8783F704700BF1E
:108B100000000F270F270F27632280F8702F0D4AC0
:108B2000C0F8182F00230C4A0370A0F84C3FA0F89F
:108B30006E3FA0F8163FC0F81C2FC0F8202FC0F8D9
:108B4000243FA0F8283F80F82A3FC0F8743FA0F8DF
:108B5000783F704700000F270F270F27F7B5394ED2
:108B60004FF47A5304464FF0000C1F4630461FFA6C
:108B70008CF5AA421FD904EB4105B5F91650002D1A
:108B800012DDA842B8BF2846AF42A8BF2F4601F168
:108B90000A05ADB2B5F5F06F24BFA1F276718DB2C2
:108BA0000CF1010C2946E2E7AB42A8BF2B46AE42CE
:108BB000B8BF2E46EBE7C219334452105B10D518EC
:108BC0006D102EB2551B2DB21BB21F491F48CDE9A7
:108BD000006512B203F000FB94F8703F632B04F6BB
:108BE0002C7104F64C701FD10B4623F8026B98428F
:108BF0001D84FAD1002384F8703F0023A4F84C3F71
:108C0000A4F86E3F1A4631F9025B2A440D8C884263
:108C10002B4412B21BB2F6D112111B11A4F84C2F27
:108C2000A4F86E3F03B0F0BD04EB43020133DBB2A6
:108C30000F2BA2F82C6FA2F84E5F84F8703FD9D8A2
:108C4000DBE700BF80C1FFFF97520108E0D9002099
:108C50002DE9F04F85B0DFF8B8B0BDF940A0BDF9FF
:108C60003C400294BDF838500192CAF100044FF024
:108C700000090394019A1FFA89F4944244D200EB4C
:108C8000410405F1010CE68A029C039A361B1FFA87
:108C90008CFC4FEAE50805F0070736B24FEAEC0412
:108CA0000CF0070C0235964213F808E01BF8077029
:108CB0001BF80CC0ADB207DA2EEA070703F80870FC
:108CC0001E5D4CEA060C08E0002E15DA2EEA0707B6
:108CD00003F808701E5D26EA0C0C03F804C001F1CD
:108CE0000A04A4B2B4F5F06F24BFA1F276718CB27D
:108CF00009F101092146BDE74EEA070703F80870AC
:108D000056451E5DDDDAE6E705B0BDE8F08F00BF31
:108D10003B520108B0F8163F00EB43032DE9F04742
:108D200004465888C0F3090080F4A67086B080F02D
:108D3000010003F0D9FC022800F2A480B4F8183F27
:108D4000DFF848E1504903F22677BFB2B7F5F06F7C
:108D500024BFA3F15A07BFB23A460A2000264FF4B7
:108D60007A534FF6FD784FF0030904EB42051EF9E4
:108D700001CBB5F91650A942B8BF2946AB42A8BFEE
:108D80002B46BCF1010F78D0BCF1030F04D0BCF12D
:108D9000FF3F74D12E4401E015FB086602F10A057D
:108DA000ADB2B5F5F06F28BFA2F2767200F1FF30D8
:108DB0002CBF92B22A4610F0FF00D6D1D4F8242F4F
:108DC000B24257DA94F8702F632A0AD10B445B1031
:108DD000A4F84C3FCB1A44F63E114B43DB13A4F8E6
:108DE0006E3FB4F96E3F02930025B4F94C3F0193F6
:108DF0000A22394605AB20460095FFF729FF237864
:108E00009DF81400AB4280F0CD000CBF4FF0010A7A
:108E10004FF0030A03F058FC80469DF8150080F0DF
:108E2000F50003F051FC81469DF8160020F00F007C
:108E300080F0900003F048FC484480445FFA88F8D2
:108E4000D0451FD80623A4F8283FB4F8183FA4F84B
:108E50001E3F03F21B7292B2B2F5F06F28BF653B62
:108E6000C4F8246FA4F81A7F34BFA4F81C2FA4F808
:108E70001C3F012006B0BDE8F087761B8EE715FB8E
:108E800009668BE70020F5E780C1FFFF4352010828
:108E900010B50446FFF73EFFA0B194F82A3F8BB906
:108EA000C4F8743FA4F8783F01211B48FEF742F84C
:108EB00001211948FEF74AF8632384F8703F05231F
:108EC00084F82A3F94F82A3F23B3013BDBB2012BFD
:108ED00084F82A3F1ED1B4F81E3F03F27F7292B28B
:108EE000B2F5F06F28BF03F1FF32A4F8202F5A1C0F
:108EF00092B2B2F5F06F24BFA3F27F73A4F8223FC1
:108F00004FF0010323704FF0000338BFA4F8222F65
:108F100084F82A3F10BD00BF908A002010B5044697
:108F2000B0F8780F98B1D4F8743FB3FBF0F3C3F303
:108F3000072081F8310081F832303322054801F0F2
:108F40009DFE0023C4F8743FA4F8783F10BD312281
:108F5000F4E700BFE0D9002030B5B0F8201FB0F82A
:108F6000222FB0F8183F914293B004466BD2994239
:108F700004D89A4202D32046FFF7CCFEB4F8182F4B
:108F8000B4F81C3F9A425CD1B4F8283F062B16D1A6
:108F9000B4F81E3F03F27F7292B2B2F5F06F28BFB1
:108FA00003F1FF32A4F8202F5A1C92B2B2F5F06FF1
:108FB0002ABFA3F27F73A4F8222FA4F8223FC02275
:108FC000B4F81A1F2046FFF7C9FDB4F96E3F0093AD
:108FD000B4F91E2FB4F94C3F2249234803F0B5F8E9
:108FE000B4F96E3F0293B4F94C3F01930823009308
:108FF000C02205ABB4F81A1F2046FFF729FEB4F8CB
:10900000285F013DADB2A4F8285FFDB917491648A5
:1090100002F052F829461648FDF78CFF29461448FD
:10902000FDF794FF104801F057FE42F20F73A4F8C9
:109030001C3F6323257084F8703F84F82A5FC4F8CE
:10904000245F13B030BD994293D894E76B1F5D4203
:109050005D4105A98DF81450FFF760FF0023C4F8A7
:10906000243FEEE74D520108E0D900207552010877
:10907000908A00202DE9F04104460D46971E01EB31
:109080004308002645453ED037F8022FD4F8743FF8
:1090900035F9021B1344C4F8743FB4F8162FB4F822
:1090A000783F04EB42020133A4F8783F53885B0019
:1090B0009BB20029B8BF43F001035380B4F8183FB6
:1090C00004EB43032046D9822378012B18D1FFF704
:1090D00043FFB4F8183F01339BB2B3F5F06F38BFCC
:1090E000A4F8183FB4F8163F28BFA4F8186F01334E
:1090F0009BB2092B94BFA4F8163FA4F8166FC1E7E2
:10910000FFF7C6FEE5E7BDE8F0810000F8B50446CC
:1091100000254FF47A602581208065816573257371
:1091200007F0D2F8C4E90455C4E9085504F128074A
:109130006060A561A58304F148063B4623F8025B05
:109140009E42FBD104F1D4033246002122F8021BD7
:109150009342FBD104F28451002203F8012B99427F
:10916000FBD1F023A4F8883540F6B833C4F88C3529
:10917000C4F88425C4F8902500212022384607F041
:10918000DBF98C220021304607F0D6F90A2323743C
:1091900009236382044B2662C4E905371623A3839F
:1091A000024B63622046F8BD38070020EC07002020
:1091B000F0B5ADB00A460446002302A9F52540F2F9
:1091C000DF264FF621574FF60B7C02F0C0008028B7
:1091D00025D0C02820D000280CBF6046384621F892
:1091E000130001339200042BD2B2EED104AA04F191
:1091F000100006F093F918AA04A904F11C00282312
:1092000006F088FB0023009318AA282305210548AF
:10921000FEF768FA2DB0F0BD21F81360E1E721F800
:109220001350DEE7908A002030B5ADB0054600242B
:1092300004AA02A904231030CDE9024406F06EF915
:1092400018AA04A905F11C00282306F063FB00946A
:10925000282318AA05210248FEF744FA2DB030BD94
:10926000908A002070B5B0F8843504461BB353488B
:10927000534EFDF741FE0546282D1BD9B4F886351F
:109280005A1C2344A4F8862593F8D4102046FFF7EF
:109290008FFF3378283DADB21BB1D4F88C35C4F8BC
:1092A0009035B4F88625B4F884359A42E4D3002387
:1092B000C4F8843570BD428903899BB293421BD1A7
:1092C000037B002B3DD00388002B3AD03D4B19780F
:1092D00000294DD1B4F888655F25B4F8843588B28B
:1092E0005A1C864292B204EB030013D9A4F88425D9
:1092F000013180F8D450F0E7438902899A429DBF3A
:1093000042890188038903898CBF42895B189B1AB3
:109310009BB2D9E75721224480F8D410752182F8F6
:10932000D410DA1C023314FA83F3A4F88425FD2246
:1093300083F8D4200023A4F88635B4F88435002BB4
:1093400095D1D4F89035002BB4D01C48FDF7D4FD4E
:109350000546282DAED92046FFF766FFD4F8903594
:10936000283D013BADB2C4F89035002BF1D1A1E707
:10937000302300202189628992B28A4203D1227B64
:1093800002F0FF016AB16168628992B2895C207360
:109390006289013292B2628162892588954298BFC2
:1093A0006081B4F88425013B551C224413F0FF036F
:1093B000A4F8845582F8D410DCD1BBE7908A002051
:1093C00031070020CA9A002001EB4101490001F554
:1093D0009671B1F5966F8ABF4FF49663A0F8881521
:1093E000A0F8883570474FF416735943C0F88C15B0
:1093F000704708B5F8F737FF3023B0FBF3F0C0B281
:1094000008BD312AF8B504460D4624D1F8F72BFFE4
:109410002F2822D901231946227B02F0FF002AB10E
:1094200061730133312BF7D10020F8BD66682289C2
:10943000EF5C92B2B7542289013292B22281228922
:109440002688964298BF20812089628992B2824202
:1094500008BF2173E5E70420E7E70520E5E7000002
:109460000023C0E90133C0E9033300F5075203705C
:10947000436100F11801183221F8023B9142FBD1FF
:1094800042F2D81242F2DC118350224A425042F298
:10949000E011425042F2E411425042F2E81242F22C
:1094A0000F71815242F2EC120021835042F2F0120D
:1094B000835242F2F2134FF00002C25400F50753F8
:1094C00000F508523433143223F8021B9342FBD1C7
:1094D00042F214230022C15200F5085300F508514E
:1094E0001633363123F8022B9942FBD142F2362350
:1094F0006321C25242F23823C15442F23C23C2508B
:1095000000F509531A8042F242234FF00002C25480
:10951000704700BF0F270F2742F2EC1200230370A1
:10952000835042F238226321815442F2D81242F22F
:10953000DC118350114A425042F2E011425042F293
:10954000E411425042F2E81242F20F71815242F2AB
:109550001422835242F23622835242F2F012835294
:1095600042F2F212835442F23C22835000F5095237
:10957000138042F242228354704700BF0F270F2707
:10958000F7B53F4E4FF47A5304464FF0000C1F4698
:1095900030461FFA8CF5AA421FD901F10C0534F9A7
:1095A0001550002D12DDA842B8BF2846AF42A8BF13
:1095B0002F464D1DADB2B5F5875F22BFA1F586518F
:1095C0001B398DB20CF1010C2946E2E7AB42A8BF72
:1095D0002B46AE42B8BF2E46EBE7C21933445210B9
:1095E0005B10D5186D102EB2551B2DB21BB212B2E6
:1095F00024492548CDE9006502F0EEFD42F238210C
:1096000004F50752635C04F50850632B02F1340241
:1096100000F1140024D1134623F8026B98421D84F4
:10962000FAD142F238230021E15442F214210023FE
:10963000635242F236216352194632F9025B2944E1
:10964000158C90422B4409B21BB2F6D142F214227F
:109650000911A15242F236221B11A35203B0F0BDF0
:1096600004EB430742F2F41C013327F80C60DBB231
:1096700042F216260F2BBD536354D2D8D5E700BF54
:1096800080C1FFFF16540108E0D900202DE9F04FFA
:1096900085B0DFF8B8B0BDF940A0BDF93C400294F8
:1096A000BDF838500192CAF100044FF0000903944C
:1096B000019A1FFA89F4944245D201F10C0405F194
:1096C000010C30F81460029C039A361B1FFA8CFCC4
:1096D0004FEAE50805F0070736B24FEAEC040CF054
:1096E000070C0235964213F808E01BF807701BF8C8
:1096F0000CC0ADB207DA2EEA070703F808701E5D4A
:109700004CEA060C08E0002E15DA2EEA070703F8EB
:1097100008701E5D26EA0C0C03F804C04C1DA4B2B0
:10972000B4F5875F22BFA1F586511B398CB209F1D0
:1097300001092146BCE74EEA070703F808705645C1
:109740001E5DDDDAE6E705B0BDE8F08FB85201082E
:1097500042F2D8132DE9F04FC35A00EB83030446BD
:109760005B686D4823F07F4387B0584002F0BCFF30
:10977000022800F2CD8042F2DA13DFF8A4C1E35AE6
:10978000664803F583560D36B6B2B6F5875F24BF3B
:10979000A3F17306B6B23346182500274FF47A5169
:1097A0004FF6FD7E4FF0030803F10C021CF9019BFC
:1097B00034F912209042B8BF10469142A8BF11461A
:1097C000B9F1010F00F09F80B9F1030F05D0B9F195
:1097D000FF3F40F09A80174401E012FB0E775A1DBC
:1097E00092B2B2F5875F24BFA3F586521B3A05F10A
:1097F000FF352CBF93B2134615F0FF05D4D142F2CA
:10980000EC13E358BB4280F2858042F23823E35CDC
:10981000632B0CD142F214220B185B10A35244F6B6
:109820003E12C31A534342F23622DB13A35242F2D2
:1098300036231822E35E029342F214233146E35E9C
:10984000019300230093204604ABFFF71FFF23780A
:10985000DFF8D0A0002B0CBF4FF0020B4FF0040B31
:109860000DF110094FF0060819F8010B1AF8013B29
:10987000584002F029FF054408F1FF3010F0FF08BE
:10988000EDB2F1D15D4543D842F2EC130522E75029
:1098900042F2F01342F2E011E25242F2DA1342F2E3
:1098A000E812E35AA35242F2DE12A65203F58352A3
:1098B000073292B2B2F5875F28BFA3F179026252F4
:1098C0002278E2B942F2E61242F2E211A35242F2E7
:1098D000DC12A65203F2BB7292B2B2F5875F28BFC8
:1098E000A3F62512625203F2BD7292B2B2F5875FFF
:1098F00042F2E4112ABFA3F62313625263520120FD
:1099000007B0BDE8F08FBF1A69E712FB087766E77A
:109910000020F5E72846F3E7A030FB0080C1FFFFF9
:10992000C6520108C052010838B50446FFF710FFBF
:10993000B8B142F2F215635D9BB942F23C220121BB
:10994000A35004F509521D481380FDF7F3FA0121D5
:109950001A48FDF7FBFA42F238236322E2540A2345
:10996000635542F2F212A35C33B3013BDBB2012B2D
:10997000A35421D142F2E61342F2E211E35A03F278
:10998000BB7292B2B2F5875F28BFA3F6251262526E
:1099900003F2BD7292B2B2F5875F42F2E41124BFC6
:1099A000A3F6231363524FF0010338BF62522370B2
:1099B00042F2F2130022E25438BD00BF908A002028
:1099C00042F2DC13F0B5C35A03F1780189B2B1F564
:1099D000875F28BFA3F5835142F236239FB0C35E51
:1099E000029342F2142328BF0839C35E01934FF05B
:1099F000000300934FF0080204AB28BF89B204466D
:109A0000FFF744FE9DF8113042F2422203F00F03AB
:109A100083540F2B33D8DFE803F00832328D323213
:109A2000327B32323232583232B242F2DC154FF4EB
:109A3000C672415B42F23627FFF7A2FD42F21426BE
:109A400042F2E612E35F0093A25EA35F5E495F48C5
:109A500002F07BFBE35F0293A35F01930823009373
:109A60004FF4C67205AB615B2046FFF70FFE012382
:109A70008DF81430642205A9544801F089F842F2A7
:109A8000E81342F2E211E35A03F586521F3292B212
:109A9000B2F5875F28BF03F1FF3262525A1C92B2BF
:109AA000B2F5875F28BFA3F5865342F2E41124BFC5
:109AB0001F3B63524FF0020338BF6252237042F2E1
:109AC000EC130022E2501FB0F0BD42F2E61542F264
:109AD0003627B422415B42F21426FFF751FDE35FC3
:109AE0000093625FA35F3A49384802F02EFBE35FC0
:109AF0000293A35F019308230093B42205AB615B3B
:109B00002046FFF7C3FD01238DF814302E22B2E763
:109B100042F2DC15B422415B42F23627FFF730FDFA
:109B200042F2142642F2E612E35F0093A25EA35FC4
:109B30002849D9E742F2DC154822415B42F2362738
:109B4000FFF71EFD42F2142642F2E612E35F009395
:109B5000A25EA35F20491D4802F0F7FAE35F02937B
:109B6000A35F019308230093482205AB615B204665
:109B7000FFF78CFD01238DF8143013227BE742F2AE
:109B8000DC15D822415B42F23627FFF7F9FC42F29E
:109B9000142642F2E612E35F0093A25EA35F0F4930
:109BA0000A4802F0D2FAE35F0293A35F019308230D
:109BB0000093D82205AB615B2046FFF767FD0123C8
:109BC0008DF81430372256E7DE520108E0D9002024
:109BD0000C5301083A5301086953010897530108CF
:109BE00042F2E21310B5C15A42F2E4130446C25ADB
:109BF00042F2DA139142C35A13D2994204D89A42DC
:109C000012D32046FFF7A4FD42F2DA13E25A42F2E1
:109C1000E413E35A9A4207D12046BDE81040FFF70B
:109C2000CFBE9942EBD8ECE710BD000038B500F587
:109C3000095504462888A0B142F23C23DB22E358B0
:109C4000B3FBF0F3C3F3072081F8D90081F8DA30D1
:109C5000054800F0C9FF42F23C220023A3502B80AC
:109C600038BDD922F4E700BFE0D9002042F2E21368
:109C7000F0B5C15A42F2E413BDB0C25A42F2DA134F
:109C800091420446C35A7CD2994204D89A4202D3E4
:109C90002046FFF75DFD42F2DA13E25A42F2E0138A
:109CA000E35A9A426BD142F2F013E35A052B1AD1D0
:109CB00042F2E81342F2E211E35A03F586521F32F0
:109CC00092B2B2F5875F28BF03F1FF3262525A1C8D
:109CD00092B2B2F5875F42F2E41125BFA3F5865335
:109CE0001F3B6252635242F2DE154FF45872615BC1
:109CF000204642F23627FFF743FC42F2142642F296
:109D0000E812E35F0093A25EA35F2649264802F0B3
:109D10001CFAE35F0293A35F019308230093615B46
:109D200005AB4FF458722046FFF7B0FC42F2F01337
:109D3000E55A013DADB2E55235BB1C491A4801F068
:109D4000BBF929461A48FDF7F5F829461848FDF7EA
:109D5000FDF8154800F074FF42F2E01342F20F7272
:109D60002570E25242F238236322E25442F2F213A7
:109D7000E55442F2EC13E55042F24223E5543DB083
:109D8000F0BD994282D883E72B1F5D425D4105A952
:109D90008DF81450FFF74AFF42F2EC130022E25014
:109DA000EDE700BFC7530108E0D90020F5530108D3
:109DB000908A00202DE9F84300F5075504460E4629
:109DC000971E01EB43081835464548D042F23C2225
:109DD00037F8020FA35836F9021B0344A35004F5C9
:109DE00009520029138803F1010313802A8804EB28
:109DF000820242F2DA1953684FEA4303B8BF43F0D4
:109E00000103536034F809300C3324F8131023781D
:109E1000012B05D0022B1ED02046FFF785FD02E066
:109E20002046FFF7DDFE34F8093001339BB2B3F56D
:109E3000875F21BF42F24222002324F80930A35455
:109E400038BF24F809302B8801339BB2042B88BF1C
:109E500000232B80B8E72046FFF708FFE3E7BDE8C3
:109E6000F8830000F8B5044600254FF47A60258198
:109E7000208065816573257306F026FAC4E90455D0
:109E8000C4E9085504F128076060A561A58304F1C1
:109E900048063B4623F8025B9E42FBD104F1C00317
:109EA0003246002122F8021B9342FBD104F5AE6139
:109EB000002203F8012B9942FBD1F023A4F874355A
:109EC00041F27073C4F87835C4F87025C4F87C2565
:109ED00000212022384606F02FFB78220021304650
:109EE00006F02AFB0523237408236382044B2662B1
:109EF000C4E905372023A383024B63622046F8BDE3
:109F00001808002068080020F0B599B005460B46F7
:109F1000002402A94FF4D27040F2EC464FF61437F9
:109F20004FF65C6C03F0C002802A26D0C02A21D0F4
:109F3000002A0CBF62463A4621F8142001349B00E7
:109F4000042CDBB2EED1234604AA05F1100005F083
:109F5000E5FA0EAA04A905F11C00142305F0DAFCA9
:109F6000002300930EAA142321460548FDF7BAFBEF
:109F700019B0F0BD21F81460E0E721F81400DDE726
:109F8000908A002030B599B00546002404AA02A9A1
:109F900004231030CDE9024405F0C0FA0EAA04A94A
:109FA00005F11C00142305F0B5FC009414230EAA3F
:109FB00004210248FDF796FB19B030BD908A0020BD
:109FC00001EB4101890001F51671B1F5966F8ABF69
:109FD0004FF49663A0F87415A0F8743570474FF4E9
:109FE00096635943C0F878157047000073B5B0F810
:109FF0007035044623B34748474EFCF77DFF0546BE
:10A00000142D1BD9B4F872355A1C2344A4F87225B8
:10A0100093F8C0102046FFF777FF3378143DADB2B8
:10A020001BB1D4F87835C4F87C35B4F87225B4F88F
:10A0300070359A42E4D30023C4F8703502B070BD85
:10A04000428903899BB2934218D1037B002B49D0EC
:10A050000388002B46D0314B1B78EBB9B4F874550C
:10A06000772198B28542B4F8702534D9501C224427
:10A07000A4F87005013382F8C010F2E74389028921
:10A080009A429DBF42890188038903898CBF428916
:10A090005B189B1A9BB2DCE70DF106012046FAF72C
:10A0A00026FA00252E469DF80620EBB29A4212D9D8
:10A0B0000DF1070120468DF80760FAF718FAB4F899
:10A0C00070355A1C2344A4F870259DF8072083F8A6
:10A0D000C0200135E7E70023A4F87235B4F87035E5
:10A0E000002B88D1D4F87C35002BA7D00948FCF789
:10A0F00003FF0546142DA1D92046FFF743FFD4F8EE
:10A100007C35143D013BADB2C4F87C35002BF1D158
:10A1100094E700BF908A002031070020CA9A0020EF
:10A1200008B5F8F7A0F8D823B0FBF3F0C0B208BD2B
:10A13000122AF8B504460D46164643D9F8F793F8A7
:10A14000864241D8237B721E03F0FF016BB10123CD
:10A15000637300210120CBB29A4237D9267B06F0E7
:10A16000FF07BEB160730131F5E7606823899BB2D8
:10A17000C254238901339BB22381238920889842CA
:10A1800098BF2181218963899BB28B42E1D1012350
:10A190002373DEE72B44666893F801C023899BB2E2
:10A1A00006F803C0238901339BB2238123892688C3
:10A1B0009E4298BF2781268963899BB2B34208BF1C
:10A1C0002073D0E70420F8BD0520FCE70020FAE763
:10A1D00070B5044600254FF47A60258120806581A2
:10A1E0006573257306F070F8C4E9055504F11C0683
:10A1F0006060258204F5B873324622F8025B934210
:10A20000FBD104F50E71002203F8012B9942FBD11A
:10A210004823C4F83822A4F83C324FF4AA72002133
:10A22000304606F089F906232382024B6661A3615A
:10A23000204670BDA80800202DE9F047ADF5227D2D
:10A2400002ADDFF85890DFF858A007460E46082404
:10A25000A84633064CBF5146494628462822013CB1
:10A2600006F0D0F8760014F0FF04F6B205F12805E8
:10A27000EFD152AA414607F11000A02305F04AFB96
:10A280000094A02352AA06210348FDF72BFA0DF5EE
:10A29000227DBDE8F08700BF908A00203654010877
:10A2A0005E54010801EB41014908483196298ABFF3
:10A2B0009623A0F83C12A0F83C32704708B5B0F8DD
:10A2C00038322BB9F9F748F8003018BF012008BD23
:10A2D0000120FCE738B50446F9F73EF8B4F8381227
:10A2E000E8B981B32F48FCF707FE0546A02D2AD90F
:10A2F000B4F83A325A1C2344A4F83A2293F8701165
:10A300002046FFF799FFB4F83A22B4F83832A03D5E
:10A310009A42ADB2EAD30023C4F8383213E00029E0
:10A32000E0D1214B1B78BBB9B4F83C52AA2198B2BA
:10A330008542B4F8382207D80023A4F83A32B4F89A
:10A340003832002BCED138BD501C2244A4F838023C
:10A35000013382F87011EAE744220B4620896189B3
:10A3600089B2814203D1217B01F0FF0069B16068AD
:10A37000618989B2405C23736189013189B261814D
:10A38000618925888D4298BF6381B4F83812013AFB
:10A390004D1C214412F0FF02A4F8385281F87001DC
:10A3A000DCD1C9E7908A0020CA9A002008B5F7F7E7
:10A3B0005AFF4423B0FBF3F0C0B208BD442AF8B5FD
:10A3C00004460D4624D1F7F74EFF432822D9002238
:10A3D0000121237B03F0FF002BB161730132442A7A
:10A3E000F7D10020F8BD66682389AF5C9BB2F754B3
:10A3F000238901339BB22381238926889E4298BFFB
:10A400002081208963899BB2834208BF2173E5E7DD
:10A410000420E7E70520E5E700B58FB0C27A037AAC
:10A4200001780D92827A0C92427A0B92427B0A92C8
:10A43000027B0992C3F380120892DA090792C3F3F0
:10A44000401203F00F0306920593C37904938379B6
:10A4500003934379029303790193C378009383783C
:10A460004278044801EB8101FAF7FCFA0FB05DF87D
:10A4700004FB00BF087D002070B50346044600F5CC
:10A480000072002503F8015B9A42FBD14FF4B976C4
:10A49000A4F81052C4F80052A4F8125284F80452DE
:10A4A000A4F8086284F8145284F81552304605F076
:10A4B0000BFFA4F82852C4F80C02A4F82A52C4F8DE
:10A4C0001852A4F81C52A4F8206284F82C5284F884
:10A4D0002D52304605F0F8FEC4F82402204670BD27
:10A4E0001FB54FF49C63ADF80C3070238DF80E301F
:10A4F00000238DF80F10009303AA0423012101F01B
:10A50000E7FF05B05DF804FB1FB54FF4BC63ADF881
:10A5100008307F238DF80A3000238DF80B108DF85A
:10A520000C20009302AA0523012101F0D1FF05B000
:10A530005DF804FB10B504468CB06F48FCF70CFEC8
:10A540004FF4A753ADF8103001238DF812306B4B48
:10A5500069481B788DF81330694B0DF10F021B7899
:10A560008DF814300DF10E01FCF7D8FD9DF80E307A
:10A570002BB19DF8143043F002038DF814305E487F
:10A58000FCF7E5FD28B19DF8143043F004038DF885
:10A5900014305948FCF7D4FD28B19DF8143043F02D
:10A5A00008038DF814305448FCF7DDFD28B19DF800
:10A5B000143043F010038DF814309DF80F302BB198
:10A5C0009DF8143043F020038DF814304D4A9DF867
:10A5D00014301278002A14BF4022002213438DF851
:10A5E000143000238DF81530474B1B78002B5ED0BC
:10A5F0004648FAF76FF88DF81600454B1B78002B8C
:10A600005FD0444B1B78002B54D04348F8F70FFE23
:10A610008DF817004048F8F712FE8DF818003F4BF0
:10A620001B78002B52D03E4802F071FD8DF81900C6
:10A630003C4B1B78002B4CD03B48FFF771FD8DF84D
:10A640001A003A4B1B78002B46D03948FEF7D1FE52
:10A650008DF81B00374B1B78002B40D03648FEF797
:10A6600054F88DF81C00354B1B78002B3AD0344839
:10A67000FAF7AEFF8DF81D00324B1B78ABB33248B2
:10A68000FFF794FE8DF81E00304B1B7883B33048E3
:10A69000F6F7A4FA8DF81F0000230893009304AA8C
:10A6A00014230121204601F013FF0CB010BD8DF8DA
:10A6B0001630A2E70A2327488DF81730F7F7F0FD88
:10A6C000ABE78DF817308DF81830A8E78DF8193002
:10A6D000AEE78DF81A30B4E78DF81B30BAE78DF885
:10A6E0001C30C0E78DF81D30C6E78DF81E30CBE773
:10A6F0008DF81F30D0E700BF908A0020C99A002053
:10A70000CA9A0020C89A002030070020607A0020F2
:10A710002F07002031070020A45800203707002011
:10A7200050EF00203507002020D200203407002001
:10A7300048AA002033070020CC95002032070020D3
:10A74000087D002036070020A0D700202E0700201B
:10A7500014140020B831002010B5B4B0174B029388
:10A76000044640F27F331648ADF80C30FDF7CEFAC0
:10A7700010228DF80E0000210DF10F0005F0DCFE17
:10A780000F480DF10F01FDF7C3FA0E481723A3F18F
:10A790001702D2B2825C32B134A91944013301F8F4
:10A7A000C82CDBB2F3E70092012102AA20468DF803
:10A7B000093001F08DFE34B010BD00BFE000000292
:10A7C000908A0020865401082DE9F04F072A97B09F
:10A7D00036D94B788C790E788F7891F803C091F840
:10A7E00004E091F8058003EB830304F00109C4F34E
:10A7F000400A5B00C4F38004002016AD05EB000B9B
:10A80000C51DEDB24D5D0BF8345C00F10805EDB2ED
:10A8100001309542C0B2F0DB16AA1044002200F8C5
:10A82000342C09A9CDE905A4CDE90389CDE901CEF0
:10A83000009732460348FAF7B1F817B0BDE8F08F39
:10A840000420FAE7087D0020F0B5052A93B01646EB
:10A8500028D94B78C8780A788F7891F804C000EB33
:10A86000800003EB830344005B00002012AD05EB86
:10A87000000E451DEDB24D5D0EF8345C851DEDB248
:10A880000130B542C0B2F1DB12A90844002100F842
:10A89000341CCDE9014C009705A90348FAF7BEF82E
:10A8A00013B0F0BD0420FBE7087D00200D2A02D97B
:10A8B0000846FFF7B1BD042070470000F0B5032A39
:10A8C00091B021D988780E784B78CF7800EB800052
:10A8D00044000420051F0DF1400C90425CFA85F500
:10A8E00006DA11F800C005F834CC0130C0B2F1E747
:10A8F000002205F8342C03A9CDE90047324603486D
:10A90000FAF718F911B0F0BD0420FBE7087D00202C
:10A9100010B54FF4E1320446012101F09BFD2046C1
:10A920004FF416520321BDE8104001F093BD000022
:10A9300030B5134B1B78012B91B01FD8114B1B78EE
:10A94000E3B1E023ADF80C3010238DF80E30002475
:10A95000E5B2EB1CAA42DBB206D910AD2B440D5D6B
:10A9600003F8345C0134F3E70332D3B200220092DF
:10A97000012103AA8DF80D3001F0AAFD11B030BD00
:10A98000C99A00203007002030B5134B1B78012BEB
:10A9900089B01FD8114B1B78E3B1E023ADF80C3020
:10A9A00011238DF80E300024E5B2EB1CAA42DBB275
:10A9B00006D908AD2B440D5D03F8145C0134F3E7B0
:10A9C0000332D3B200220092012103AA8DF80D3088
:10A9D00001F07EFD09B030BDC99A0020300700208B
:10A9E0001FB50C4B1B78012B10D80B4B1B786BB190
:10A9F0004FF47873ADF80C3012238DF80E3000232D
:10AA0000009303AA0323012101F062FD05B05DF864
:10AA100004FB00BFC99A0020300700201FB50C4B73
:10AA20001B78012B10D80B4B1B786BB14FF478734C
:10AA3000ADF80C3013238DF80E300023009303AAD9
:10AA40000323012101F044FD05B05DF804FB00BFC4
:10AA5000C99A00203007002030B5154C247814F036
:10AA6000FD048DB022D1134D2D78FDB1002914BF06
:10AA70001A211821E0258DF80A10ADF8085021465A
:10AA8000CDB2EC1CAB42E4B206D90CAD2C44555C03
:10AA900004F8285C0131F3E700220333DBB20092B3
:10AAA000012102AA8DF8093001F012FD0DB030BD70
:10AAB000C99A00202F0700201FB50D4B1B7813F0FB
:10AAC000FD0312D10B4A12787AB14FF47872002943
:10AAD000ADF80C2014BF1B2219228DF80E20009314
:10AAE00003AA0323012101F0F3FC05B05DF804FB88
:10AAF000C99A00202F07002030B5144B1B78032B78
:10AB0000A5B000D0FBB9124B1B78E3B1E023ADF840
:10AB10000C3020238DF80E300024E5B2EB1CAA4245
:10AB2000DBB206D924AD2B440D5D03F8845C0134FF
:10AB3000F3E70332D3B200220092012103AA8DF879
:10AB40000D3001F0C5FC25B030BD00BFC99A002012
:10AB5000370700201FB50C4B1B78032B00D083B99F
:10AB60000A4B1B786BB14FF47873ADF80C3021238E
:10AB70008DF80E300023009303AA0323012101F076
:10AB8000A7FC05B05DF804FBC99A00203707002038
:10AB900030B5134B1C7814F0FB04A1B01ED1114B3F
:10ABA0001B78DBB1E023ADF8083030238DF80A3094
:10ABB000E5B2EB1CAA42DBB206D920AD2B440D5DF9
:10ABC00003F8785C0134F3E70332D3B20022009239
:10ABD000012102AA8DF8093001F07AFC21B030BDC4
:10ABE000C99A00203507002030B5134B1C7814F0AB
:10ABF000FB04C3B01ED1114B1B78DBB1E023ADF8D1
:10AC00000C3031238DF80E30E5B2EB1CAA42DBB2DA
:10AC100006D942AD2B440D5D03F8FC5C0134F3E72B
:10AC20000332D3B200220092012103AA8DF80D3025
:10AC300001F04EFC43B030BDC99A0020350700201A
:10AC40001FB50C4B1B7813F0FB030FD10A4A127887
:10AC500062B14FF47872ADF80C2032228DF80E20DC
:10AC6000009303AA0323012101F032FC05B05DF833
:10AC700004FB00BFC99A00203507002030B5144BF3
:10AC80001B78052BA5B000D0FBB9124B1B78E3B1A4
:10AC9000E023ADF80C3040238DF80E300024E5B2EF
:10ACA000EB1CAA42DBB206D924AD2B440D5D03F8A0
:10ACB000845C0134F3E70332D3B200220092012115
:10ACC00003AA8DF80D3001F003FC25B030BD00BFA4
:10ACD000C99A0020340700201FB50C4B1B78052BA8
:10ACE00000D083B90A4B1B786BB14FF47873ADF881
:10ACF0000C3041238DF80E300023009303AA032368
:10AD0000012101F0E5FB05B05DF804FBC99A0020C4
:10AD10003407002030B5144B1B78072BA5B000D0AA
:10AD2000FBB9124B1B78E3B1E023ADF80C3045239F
:10AD30008DF80E300024E5B2EB1CAA42DBB206D936
:10AD400024AD2B440D5D03F8845C0134F3E703323A
:10AD5000D3B200220092012103AA8DF80D3001F038
:10AD6000B7FB25B030BD00BFC99A002033070020D3
:10AD700030B5144B1B78072BA5B000D0FBB9124B94
:10AD80001B78E3B1E023ADF80C3046238DF80E308C
:10AD90000024E5B2EB1CAA42DBB206D924AD2B4459
:10ADA0000D5D03F8845C0134F3E70332D3B2002273
:10ADB0000092012103AA8DF80D3001F089FB25B026
:10ADC00030BD00BFC99A0020330700201FB50C4BCF
:10ADD0001B78072B00D083B90A4B1B786BB14FF45B
:10ADE0007873ADF80C3049238DF80E3000230093B2
:10ADF00003AA0323012101F06BFB05B05DF804FBFE
:10AE0000C99A0020330700201FB50C4B1B78072B75
:10AE100000D083B90A4B1B786BB14FF47873ADF84F
:10AE20000C3048238DF80E300023009303AA03232F
:10AE3000012101F04DFB05B05DF804FBC99A00202B
:10AE40003307002030B5214B1B780A2BADF5037D6D
:10AE500000D01BBB1E4B1B7803B3E023FC2A8DF8EC
:10AE60000830D4B21FD9053400238DF80A40652478
:10AE70008DF809308DF80B40013903AD11F8014F01
:10AE800005F8014B5C1CA4B2A2420AD10533002292
:10AE900000929BB202AA012101F01AFB0DF5037D7D
:10AEA00030BD2346EAE7033465238DF809408DF869
:10AEB0000A300DF10B048D18A94204D011F8013BA2
:10AEC00004F8013BF8E7D31CE1E700BFC99A002072
:10AED000320700207FB50D4B1B780A2B00D093B9A9
:10AEE0000B4B1B787BB14FF49C63ADF80C306623A1
:10AEF0008DF80E3000238DF80F10009303AA042361
:10AF0000012101F0E5FA07B05DF804FBC99A0020C1
:10AF1000320700207FB50C4B1B780A2B00D083B979
:10AF20000A4B1B786BB14FF47873ADF80C30672384
:10AF30008DF80E300023009303AA0323012101F0B2
:10AF4000C7FA07B05DF804FBC99A00203207002059
:10AF500030B5214B1B780A2BADF5037D00D01BBB10
:10AF60001E4B1B7803B3E023FC2A8DF80830D4B2C3
:10AF70001FD9053400238DF80A4055248DF8093077
:10AF80008DF80B40013903AD11F8014F05F8014B65
:10AF90005C1CA4B2A2420AD10533002200929BB2EB
:10AFA00002AA012101F094FA0DF5037D30BD23467C
:10AFB000EAE7033455238DF809408DF80A300DF186
:10AFC0000B048D18A94204D011F8013B04F8013B91
:10AFD000F8E7D31CE1E700BFC99A00202E07002044
:10AFE00070B5C2B0134602AAE02414808024947085
:10AFF0000024E6B2F51CB342EDB203D90E5D5655FE
:10B000000134F6E70333DBB20021537000910121D4
:10B0100001F05EFA42B070BD30B5124B1B78632B65
:10B02000A5B01CD1E023ADF80C3008238DF80E300C
:10B030000024E5B2EB1CAA42DBB206D924AD2B44B6
:10B040000D5D03F8845C0134F3E70332D3B20022D0
:10B050000092012103AA8DF80D3001F039FA25B0D4
:10B0600030BD00BFC99A002030B5124B1B78602B51
:10B070008BB01CD1E023ADF8083009238DF80A30DD
:10B080000024E5B2EB1CAA42DBB206D90AAD2B4480
:10B090000D5D03F8205C0134F3E70332D3B20022E4
:10B0A0000092012102AA8DF8093001F011FA0BB0CB
:10B0B00030BD00BFC99A002010B590F80432A4B08A
:10B0C000C3B1E023ADF80C30F1238DF80E3003232B
:10B0D000DA1ED2B28A5C32B124AC1C44013304F8CB
:10B0E000842CDBB2F4E70121009103AA8DF80D3026
:10B0F00001F0EEF924B010BD5F2910B50C4600F048
:10B10000888020D806297ED00ED8032975D005D88E
:10B11000012939D0022961D0454960E004296ED067
:10B120000529F9D143495AE05B297CD005D8072984
:10B1300067D00A29F0D1404951E05C2971D05D29DE
:10B14000EAD13E494BE0672965D00ED863295CD02F
:10B1500005D860295BD06229DED139493FE06529F5
:10B1600063D06629D8D1374939E06A29FBD005D8A0
:10B17000682952D06929CFD1334930E06B294ED0AC
:10B180006C29C9D131492AE031493248FFF794FF8F
:10B190003148F7F7D8F83148F6F7F7FB3048F7F7BA
:10B1A000BDFA032C23D12F48FEF7B6F9052C04D0A5
:10B1B0002D48FDF7B1FC072C04D02C48FCF7EAFD24
:10B1C0000A2C02D02A48F9F798FB2A48F6F7A2FB86
:10B1D00021462948BDE81040FBF7BCBE27491D4861
:10B1E000FFF76AFF2648F8F78DFA022CD0D12548E0
:10B1F00001F00AFB042CDBD0D5E72349EFE7234914
:10B20000EDE72349EBE72349E9E72349E7E723494A
:10B21000E5E72349E3E72349E1E72349DFE723495A
:10B22000DDE72349DBE72349D9E72349D7E700BF17
:10B230008559010896570108CA570108E4580108C2
:10B24000F657010847580108A65801086B5901082C
:10B2500049570108E0D90020AC360020FC1A002034
:10B26000FC3B0020DCAF0020CC9A0020E08D0020C9
:10B27000087D00200C170020908A00205C570108F0
:10B280009059002010DC00206C57010886570108F7
:10B29000A7570108B7570108D957010810580108E6
:10B2A0002B5801086658010887580108C55801083D
:10B2B000065901082B5901084E5901082DE9F04F94
:10B2C000242AA9B003D8042029B0BDE8F08F0E7855
:10B2D000C6F3001380F804324C78CD7804F01003E4
:10B2E000129304F020031193322D04F0400304F074
:10B2F000020A04F0040904F008081093E3D891F856
:10B3000004C091F802B0BCF1050F17D9BCF1070FCA
:10B3100000F02781BCF1060F00F02581BCF10A0F77
:10B3200000F02481ACF15B03DBB2112BCBD8904A47
:10B3300022FA03F313F0010F0DD1C4E7BCF1010FA2
:10B3400002D114F0010FF7E7BCF1020F40F0F080DA
:10B35000BAF1000FB7D08F7E0F2FB4D80B7F0F93A9
:10B360007C3B0E2BAFD84B7913938B791493CB790D
:10B3700015930B7A16934B7A17938B7A1893CB7A93
:10B3800019930B7B1A934B7B1B938B7B1C93CB7B6F
:10B390001D930B7C1E934B7C1F934B7D0A7D20934A
:10B3A0008B7D27922193CB7D2293CB7E26934B7F5F
:10B3B00023938B7F2493CB7F25936146FFF79CFEDD
:10B3C0006C48F143C1F3C01101706B496B4804F044
:10B3D00001040C702946F9F77BF81AF1000A684954
:10B3E000684818BF4FF0010A81F800A02946F6F717
:10B3F0002BFF39466448F7F7F5FE39466348F7F7FF
:10B4000075F9269B61481946F7F77CF9394660487B
:10B41000F6F75AFC39465F48F7F720F919F10009A9
:10B420005D4B5E4818BF4FF00109294683F8009034
:10B4300001F056FE279A5948C6F3C00101F05FFE9D
:10B4400018F10008564B574818BF4FF0010829461D
:10B4500083F80080FEF7B4FD20995248FEF7BFFD47
:10B46000129B514A5148003318BF012329461370DB
:10B47000FDF7AAFF21994D48FDF7B5FF109B4C4AF7
:10B480004C48003318BF012329461370FDF728F9F3
:10B4900022994848FDF733F9474B48480BF0010221
:10B4A00029461A70FEF7FEFE454A23994548CBF31C
:10B4B00040031370F5F78CFB0F9B4348A3F1800109
:10B4C00049B2DDE92423F5F7BEF9119B3F4A404814
:10B4D000003318BF01231370C6F340130D93149B60
:10B4E000803B0C93139B803B0B931F9B0A931E9BEB
:10B4F00009931D9B08931C9B07931B9B06931A9B08
:10B500000593199B0493189B0393179B0293169B17
:10B510000193159B0093C6F34002C6F3800306F027
:10B520000101FBF78CFD2A48FBF77AFD0020CBE6F2
:10B53000BCF1030F04D1B9F1000F7FF40CAFC2E6E8
:10B54000BCF1040F04D1B8F1000F7FF404AFBAE6E8
:10B55000BCF1050F7FF4FFAE129B002B7FF4FBAE16
:10B56000B1E6109BF9E71BF0010FE5E6119BF4E74C
:10B57000BFFD03003107002030070020607A002063
:10B580002F070020B8310020A4580020FC3B0020E9
:10B59000FC1A0020AC3600203707002050EF0020B6
:10B5A0003507002020D200203407002048AA0020C0
:10B5B00033070020CC95002036070020A0D70020BC
:10B5C0002E07002014140020880A002032070020D3
:10B5D000908A002008B502B31E4B09781B788B4275
:10B5E00013D0052913D907292DD006292DD00A29D2
:10B5F0002DD0A1F15B03DBB2112B0ED8164A22FA33
:10B6000003F3DB0709D5FFF777FD002115E00129DA
:10B6100005D1124B1B78002BF5D104210DE0022936
:10B6200001D10F4BF6E7032901D10E4BF2E70429B4
:10B6300005D10D4B1B78002BE5D1084608BD052927
:10B64000E1D10A4BE6E70A4BE4E70A4BE2E70A4B93
:10B65000E0E700BFC99A0020BFFD030030070020CB
:10B660002F0700203707002035070020340700206F
:10B6700033070020360700203207002070B590F80D
:10B680000432A4B013B3E023ADF80C30F2238DF8EC
:10B690000E300323DC1EE4B224AD0E5D5C1CE4B26C
:10B6A0001D441EB105F8846C2346F3E7111205F81A
:10B6B000841C24A90C440233012104F8842CDBB23D
:10B6C000009103AA8DF80D3000F002FF24B070BD88
:10B6D00020292DE9F04104460D4616461F4600F08C
:10B6E000A9826BD8102900F0E1811FD8032900F04E
:10B6F000F0800FD8012900F0E68040F2E7801A467A
:10B700003146FFF7DBFD0221024620465AB1FEF723
:10B71000FBFED3E0082900F021810A2900F0B08166
:10B72000042940F0A480FEF7DBFEC7E01A2900F0F0
:10B730001C8225D8132900F0DE81182900F0F2813F
:10B74000112940F09480B34B1B78002B00F0D1817D
:10B75000DFF8E88298F80030012B00F2CA813A46FF
:10B760003146AD48F9F704F80546002800F0AE81EF
:10B770002AB2AA49AA48FFF781FF2A461121BFE051
:10B780001D2900F014821E2900F03E821C296ED172
:10B79000A44B1B78002B00F035823A463146A24874
:10B7A000F7F746FC0546002800F088802AB29F493A
:10B7B0009B48FFF763FF2A461C21A1E0552900F0B2
:10B7C00038834CD8452900F0CE8223D8312900F0A7
:10B7D0005A82402900F07382302948D1944B1B785B
:10B7E000002B00F04782DFF8548298F8003013F005
:10B7F000FB0F40F03F823A4631468E48FEF798FCF8
:10B800000546002840F0378298F80030002B55D1CB
:10B81000042161E1492900F0C882502900F0E0824A
:10B82000462924D1844B1B78002B00F0BC82834B2B
:10B830001A78984612B1072A40F0B582FAB231461A
:10B840007F48FCF76AFF0546002800F09C822AB278
:10B850007C497348FFF712FF2A46462150E06329CE
:10B8600072D006D861294DD05CD8602938D0012229
:10B8700056E0802900F0F8821BD86529F7D1724B79
:10B880001B78002B00F0CC826C4B1A78984612B1D2
:10B890000A2A40F0C582FAB231466C48F9F7A2FE96
:10B8A0000546002840F0BD8298F8003033B90A21DF
:10B8B00012E101F17003DBB2012BD8D80023C4F8E8
:10B8C0000032BDE8F081FEF735FEF7E7FEF744FFF2
:10B8D000F4E71A463146FFF77DFE2946024614E793
:10B8E0001A463146FEF770FF054610B96021204622
:10B8F00019E702B256494A48FFF7C0FE2A466021BE
:10B90000204604E731461A46FEF79EFF064608B970
:10B910002946ECE74F4902B24148FFF7AFFE3246F5
:10B920002946EDE70D2B06D91046FEF775FD0546B5
:10B9300010B96221DBE704252AB247493848FFF7EE
:10B940009DFE2A466221DBE731461A46FEF7B6FF26
:10B9500006460028DCD002B24049DDE7374B1A78B2
:10B96000632A98464CD13A4631463D48F5F734FDB6
:10B97000054698F800305C3BDBB2062B0AD84D2216
:10B9800022FA03F3DB0705D53A4631463548F5F789
:10B990003FFB054698F80030663B052B05D83A4634
:10B9A00031463148F5F7D4FD054698F800305D2B57
:10B9B00005D13A4631462D48F5F766FE054698F81A
:10B9C00000305B2B05D13A4631462948F5F71EFE7B
:10B9D000054698F800306C2B05D13A46314625488B
:10B9E000F5F7DCFD054698F80030652B05D13A46A1
:10B9F00031462148F5F772FE05461DB9082176E764
:10BA00000225B6E72AB21D490548FFF737FE2A4648
:10BA1000082175E730070020607A00207D55010875
:10BA2000E0D900202F070020A4580020EB55010882
:10BA30003507002020D2002033070020C99A0020BB
:10BA4000CC950020BD56010832070020087D00205B
:10BA5000B5540108D2540108EF5401080C550108EF
:10BA6000E416002078160020E8160020FC160020BE
:10BA7000F9160020F8160020FE16002029550108AE
:10BA80009B4B1B7883B93A4631469A48F5F7D0FE6E
:10BA9000054600283FF412AF2AB297499748FFF7AE
:10BAA000EDFD2A460A212BE70525F5E7944B1B7887
:10BAB000B3B1DFF83C8298F80030012B10D83A4639
:10BAC00031469048F8F72EFE054650B998F80030F8
:10BAD000002B7FF4F3AE01212046FFF70DFBEDE6CE
:10BAE00002252AB288498548FFF7C8FD2A46102159
:10BAF00006E702253CE6824B1B7853B17C4E327838
:10BB0000012A06D87F48F8F759FE054610B9337860
:10BB1000DEE702252AB27D497848FFF7AFFD2A46C5
:10BB20001321EDE67A4B1B78B3B1714B1A7812F002
:10BB3000FD0F984610D1774B1B786BB13A463146D2
:10BB40007548F7F785FB054638B998F80030002BA3
:10BB50007FF4B4AE0221BFE702252AB26F496748DD
:10BB6000FFF78CFD2A461821CAE6694B1B78E3B122
:10BB70005F4B1A7812F0FD0F984616D1654B1B7873
:10BB80003A4631466BB16448F7F7A4FB05460028F6
:10BB9000DBD02AB261495948FFF770FD2A461A21C5
:10BBA000AEE65F48F6F784FBF0E70225F1E7584B75
:10BBB0001B78E3B1012F23D1117801290CD14C4B13
:10BBC0001B78022B1CD1574B1B78002B7FF476AED1
:10BBD0005148F7F777FA71E691B9454B1B78022B7C
:10BBE0000ED1504B1B78002B3FF468AEF0E70225D6
:10BBF0002A464D494148FFF741FD2A461D217FE66F
:10BC00000425F5E70225D1E5414B1B7883B13A467F
:10BC100031464148F7F740FA054600283FF44EAE5A
:10BC20002AB242493548FFF729FD2A461E2167E618
:10BC30000225F5E73E4B1B789BB12D4B1A789846B1
:10BC40000AB1032A0DD13A4631463A4801F067FA63
:10BC5000054638B998F80030002B7FF42FAE032149
:10BC60003AE702252AB234492448FFF707FD2A465D
:10BC7000202145E602252AB230492048FFF7FEFC84
:10BC80002A4630213CE62E4B1B78B3B1184B1A786C
:10BC900012F0FB0F984610D13A4631462948FEF77C
:10BCA00047FA054600283FF4AFAD2AB226491348AB
:10BCB000FFF7E4FC2A46312122E60225F5E7234B73
:10BCC0001B78002B46D00A4B1A7898460AB1052AF1
:10BCD00040D13A4631461E48FDF793FB0546D0BB9E
:10BCE00098F80030002B7FF4E9AD0521F4E600BFA1
:10BCF000C99A00200C1700204B550108E0D90020FC
:10BD000030070020607A00205E5501089A5501082E
:10BD10002F07002031070020A4580020B655010845
:10BD2000B8310020CA9A0020D055010809560108F0
:10BD30003707002050EF002024560108485601081C
:10BD40003507002020D20020645601083407002067
:10BD500048AA002002252AB25B495C48FFF78EFC06
:10BD60002A464021CCE55A4B1B789BB1594B1A7897
:10BD700098460AB1072A0DD1FAB231465648FCF767
:10BD8000CCFC054638B998F80030002B7FF496AD0E
:10BD90000721A1E602252AB250494C48FFF76EFC64
:10BDA0002A464521ACE5022551E5494B1B78ABB14C
:10BDB000484B1A7898460AB1072A0FD1FAB2314691
:10BDC0004548FCF7AAFC05460028DCD02AB24449C5
:10BDD0003E48FFF753FC2A46492191E50225F5E745
:10BDE000404B1B789BB13B4B1A7898460AB1062A08
:10BDF0000DD13A4631463C48FEF7E0FA054638B9DF
:10BE000098F80030002B7FF459AD062164E6022536
:10BE10002AB236492D48FFF731FC2A4650216FE5FA
:10BE200002252AB232492948FFF728FC2A46652113
:10BE300066E5304B1B78ABB1264B1B780BB10A2B58
:10BE400010D13A4631462C48F4F7DAFE0546002870
:10BE50003FF434AD2AB229491C48FFF70FFC2A46AB
:10BE600055214DE50225F5E70022012193B29F42BD
:10BE70007FF624AD94F8143203F0FF001BB184F870
:10BE800015120132F2E7D4F80C52B4F8103216F859
:10BE900002C09BB205F803C0B4F8103201339BB264
:10BEA000A4F81032B4F81032B4F808529D4298BF8A
:10BEB000A4F81002B4F81002B4F812329BB2834214
:10BEC00008BF84F81412DCE77D560108E0D9002091
:10BED00033070020C99A0020CC950020985601080D
:10BEE000DE56010836070020A0D70020F7560108CB
:10BEF000145701082E070020141400202D570108A4
:10BF00002DE9F0410446C2B00126C51C071D0121E0
:10BF1000204600F0A9FA8046002840D001212046A2
:10BF200000F0C6FAB4F8003201463BB9E02806BF7B
:10BF30002070C4F80062A4F80232E8E7012B06D1B1
:10BF400002236070A4F80202A4F80032DFE7022B9B
:10BF5000B4F8022210D10323A070A4F800321AB959
:10BF6000FF31A4F80212D2E7032AD0D100232A46D7
:10BF70002046FFF7ADFBCAE7E05401339BB2934282
:10BF8000A4F80032C3D1FF2B89BF043B033B9BB213
:10BF90003A468FBFE178A1789BB22A46E8E74E483F
:10BFA000FBF7DEF84BF67F339842B4F81222B4F870
:10BFB000103288BFC4F800829BB2934240D194F8FB
:10BFC0001432002B51D0B4F80852002D4DD003216B
:10BFD000204600F05BFA00268542C8BF85B237468E
:10BFE000B3B29D4241D9B4F81022B4F812328DF8A0
:10BFF0000C709BB2934202D194F81432BBB1D4F8C6
:10C000000C22B4F812329BB2D35C84F814728DF80F
:10C010000C30B4F8123201339BB2A4F81232B4F8E7
:10C020001232B4F808229A4298BFA4F8127200970C
:10C03000012303AA0321204600F04AFA0136CFE784
:10C04000B4F81232B4F810229A429DBFB4F81232FA
:10C05000B4F80822B4F81052B4F810528CBFB4F8F7
:10C060001232AD18ED1AADB2AFE70321204600F051
:10C07000FBF9051E2DDDD4F81822AA4227D1B4F809
:10C080001C32632B03D8F92A01DC01331AE003AE1A
:10C0900037460321204600F00BFAD4F8182206F8A0
:10C0A000010B08F10108013A4545C4F8182202D0F5
:10C0B000B8F1FA0FEDD1AA1AD2B239462046FEF7EE
:10C0C0008FFF0023A4F81C3242B0BDE8F081F92DA7
:10C0D000DDDCC4F81852F4E7908A0020F0B51E4663
:10C0E00090F80432A5B073B3E023ADF80C30F3231D
:10C0F0008DF80E300324E51EEDB224AB4F5D651CB8
:10C10000EDB223441FB103F8847C2C46F3E71112EF
:10C1100003F8841C24AB1D44012105F8842CA21CC7
:10C1200053FA82F2331202F8843C221DD3B2033454
:10C1300024AA52FA84F403AA04F8846C00918DF8BE
:10C140000D3000F0C5F925B0F0BDF0B590F804420F
:10C15000A5B0BDF9A860002C3CD0E024ADF80C409F
:10C16000F4248DF80E400324E51EEDB224AF11F83F
:10C1700005C0651CEDB22744BCF1000F03D007F8E1
:10C1800084CC2C46F0E7111207F8841C24A90D4436
:10C1900005F8842CA21C51FA82F2191202F8841CB0
:10C1A00024A9E21C51FA82F202F8843C231D51FAC0
:10C1B00083F3321203F8842CA31D053451FA84F45E
:10C1C000012104F8846CDBB2009103AA8DF80D30D4
:10C1D00000F07EF925B0F0BDF0B590F80442A5B0AE
:10C1E000BDF9A870BDF9AC60002C49D0E024ADF8D1
:10C1F0000C40F5248DF80E400324E51EEDB20DF140
:10C20000900C11F805E0651CEDB2A444BEF1000FDE
:10C2100003D00CF884EC2C46EFE711120CF8841CC8
:10C2200024A90D4405F8842CA21C51FA82F219129B
:10C2300002F8841C24A9E21C51FA82F202F8843C20
:10C24000231D51FA83F33A1203F8842C631D51FA2B
:10C2500083F3321203F8847CA31D51FA83F303F8AD
:10C26000842C04F10803073451FA84F4012104F802
:10C27000846CDBB2009103AA8DF80D3000F028F930
:10C2800025B0F0BD30B5ADF5037DE023FC2A8DF877
:10C290000830D4B21FD9053400238DF80A40FA249F
:10C2A0008DF809308DF80B40013903AD11F8014FBD
:10C2B00005F8014B5C1CA4B2A2420AD1053300224E
:10C2C00000929BB202AA012100F002F90DF5037D54
:10C2D00030BD2346EAE7FA2303348DF80A308DF89F
:10C2E00009400DF10B038D18A94204D011F8014B40
:10C2F00003F8014BF8E7D31CE1E70000014800F028
:10C3000065B900BF4CF4002030B5012189B0224C42
:10C310000546084601F0ECFE0121102001F020FF47
:10C3200020460722092101F02EFB07220A21204680
:10C3300001F029FB194B019301A800F029FF02A885
:10C3400001F0E8FA164B4FF4C06202A92046CDE98D
:10C350000223A4F5704401F08FFA04A802F07AFEDB
:10C3600000234FF4402204A92046CDE90532ADF860
:10C370001C30049502F016FE2046012102F089FED1
:10C380000122204640F2255102F031FF21460548A6
:10C3900000F0D9F809B030BD0000024025010101CC
:10C3A000020200014CF40020014800F00FB900BF68
:10C3B0005804012030B5012189B0224C05460846B9
:10C3C00001F096FE01214FF4003001F0BBFE204643
:10C3D0000722022101F0D7FA07220321204601F0AB
:10C3E000D2FA194B019301A800F0D2FE02A801F085
:10C3F00091FA164B0C2202A92046CDE90223A4F59E
:10C40000DE3401F039FA04A802F024FE00234FF4D0
:10C41000402204A92046CDE90532ADF81C30049530
:10C4200002F0C0FD2046012102F033FE0122204629
:10C4300040F2255102F0DBFE2146054800F083F86A
:10C4400009B030BD000002402601010102020001D6
:10C45000580401200129104602D0032902D0704758
:10C46000FFF7A8BFFFF750BF012908B503D0032984
:10C4700005D0002008BD034800F00FF9FAE7024894
:10C48000FAE700BF580401204CF40020012908B548
:10C4900003D0032905D0002008BD034800F006F9A9
:10C4A000FAE70248FAE700BF580401204CF40020E4
:10C4B000012903D0032904D000207047024800F06E
:10C4C00078B80248FBE700BF580401204CF4002074
:10C4D00010B50846012811469DF808401A4602D0BA
:10C4E00003280AD010BD084800F02FF8002CF9D01E
:10C4F0000548BDE8104000F0C5B8044800F025F834
:10C50000002CEFD00148F4E7580401204CF400203F
:10C5100008B5044800F00AF80348BDE8084000F0F8
:10C5200005B800BF4CF400205804012041F2080176
:10C530000022A0F804280260A0F80628425241F226
:10C540000A014252704701607047F8B504460D4633
:10C5500016466AB3006858B341F208070978E35BEE
:10C560009BB25A1CC3F30A03234492B2E25383F8EA
:10C570000818012240F2277102F039FE27440022F8
:10C58000013293B29E420BD93B88A85C9BB2591CE6
:10C59000C3F30A03234489B2398083F80808EFE71C
:10C5A0002068012240F22771BDE8F84002F01FBE6A
:10C5B000F8BDB0F806389BB25A1CC3F30A0392B216
:10C5C0000344A0F8062818797047000010B5044607
:10C5D0000068002853D040F2255102F02BFEE0B154
:10C5E000B4F80438B4F8062801335340C3F30A03FF
:10C5F00073B1206802F078FDB4F804389BB25A1C7D
:10C60000C3F30A032344C0B292B2A4F804281871F9
:10C6100040F225511A4802F02CFE40F227712068A2
:10C6200002F008FE58B341F20A0241F20803A15A8F
:10C63000E35A9BB28B420CD0A35A9BB2591C89B2CD
:10C64000C3F30A03A1522344206893F8081802F0A8
:10C6500047FD40F22771206802F00BFE41F20A0309
:10C66000E25A41F20803E35A9BB2934207D1206891
:10C67000002240F22771BDE8104002F0B8BD10BDA5
:10C680000010014010B5036804462BB180212068DA
:10C6900002F0D0FD0028F9D110BDB0F80628B0F89E
:10C6A00004389BB2981A18BF0120704741F2080362
:10C6B00041F20A02C35A825A581C5040C0F30A0081
:10C6C000003018BF01207047014B185C704700BF55
:10C6D00096590108034AC3B2000AD35C105C18449F
:10C6E000C0B2704796590108084AC3B2C0F3072187
:10C6F000D35C515C0B44C0F30741000E515C105CED
:10C7000051FA83F350FA83F0C0B27047965901088A
:10C71000124A10B5C3B2C0F30724D35C145D23449E
:10C72000C0F30744000E145D105C54FA83F350FA12
:10C7300083F0CBB2D35C53FA80F0C1F30723D35C10
:10C7400053FA80F0C1F30743090ED35C53FA80F02B
:10C75000535C53FA80F0C0B210BD00BF9659010877
:10C760000023C0E90133C0E9033300F5965203709A
:10C77000436100F11801183221F8023B9142FBD1CC
:10C7800041F2D82241F2DC2183501E4A425000F58A
:10C7900097510A6041F2E42242F20F71815241F254
:10C7A000E8220021835041F2EC22835241F2EE2331
:10C7B0004FF00002C25400F5975300F59852103321
:10C7C000103223F8021B9342FBD141F210330022B6
:10C7D000C15200F5985300F599511233123123F8E4
:10C7E000022B9942FBD141F232336321C25241F212
:10C7F0003433C15441F23833C25041F23C33C25257
:10C80000704700BF0F270F2741F2E8220023037073
:10C81000835041F234326321815441F2D82241F2F3
:10C82000DC2183500E4A425000F597510A6041F2D4
:10C83000E42242F20F71815241F21032835241F2EE
:10C840003232835241F2EC22835241F2EE2283547F
:10C8500041F23832835041F23C328352704700BF7C
:10C860000F270F27F7B53E4E4FF47A5304464FF08B
:10C87000000C1F4630461FFA8CF5AA421ED901F162
:10C880000C0534F91550002D11DDA842B8BF28461B
:10C89000AF42A8BF2F464D1DADB2B5F5166F24BFF0
:10C8A000A1F65B118DB20CF1010C2946E3E7AB4216
:10C8B000A8BF2B46AE42B8BF2E46ECE7C2193344A0
:10C8C00052105B10D5186D102EB2551B2DB21BB235
:10C8D00012B224492448CDE90065FFF77DFC41F2FE
:10C8E000343104F59752635C04F59850632B02F1E0
:10C8F000100200F1100024D1134623F8026B984275
:10C900001D84FAD141F234330021E15441F2103157
:10C910000023635241F232316352194632F9025B0D
:10C920002944158C90422B4409B21BB2F6D141F236
:10C9300010320911A15241F232321B11A35203B03D
:10C94000F0BD04EB430741F2F02C013327F80C60F3
:10C95000DBB241F212360F2BBD536354D2D8D5E768
:10C9600080C1FFFFFF5A0108E0D900202DE9F04FF8
:10C9700085B0DFF8B8B0BDF940A0BDF93C400294E5
:10C98000BDF838500192CAF100044FF00009039439
:10C99000019A1FFA89F4944244D201F10C0405F182
:10C9A000010C30F81460029C039A361B1FFA8CFCB1
:10C9B0004FEAE50805F0070736B24FEAEC040CF041
:10C9C000070C0235964213F808E01BF807701BF8B5
:10C9D0000CC0ADB207DA2EEA070703F808701E5D37
:10C9E0004CEA060C08E0002E14DA2EEA070703F8DA
:10C9F00008701E5D26EA0C0C03F804C04C1DA4B29E
:10CA0000B4F5166F24BFA1F65B118CB209F10109D0
:10CA10002146BDE74EEA070703F8087056451E5D3C
:10CA2000DEDAE7E705B0BDE8F08F00BF965A0108EF
:10CA300041F2D8232DE9F04FC35A00EB830304469B
:10CA40005B685B48C3F3130387B05840FFF74CFEA5
:10CA5000032800F2A88041F2DA23DFF85CE1E35A10
:10CA6000544903F60117BFB2B7F5166F24BFA3F1FF
:10CA70005F07BFB23A46142500264FF47A534FF6AB
:10CA8000FD784FF0030902F10C001EF901CB34F9D7
:10CA900010008142B8BF01468342A8BF0346BCF1E3
:10CAA000010F7BD0BCF1030F04D0BCF1FF3F77D165
:10CAB000064401E010FB0866501D80B2B0F5166F09
:10CAC00028BFA2F65B1205F1FF352CBF92B20246D9
:10CAD00015F0FF05D7D141F2E822A258B24264DA3C
:10CAE00041F23432A25C632A0CD10B4441F2103281
:10CAF0005B10A352CB1A44F63E114B4341F2323243
:10CB0000DB13A35241F232331422E35E029341F26B
:10CB100010333946E35E019300230093204604ABB3
:10CB2000FFF724FF2378DFF894A0002B0CBF4FF011
:10CB3000020B4FF0040B0DF110094FF0050819F826
:10CB4000010B1AF8013B5840FFF7BEFD054408F100
:10CB5000FF3010F0FF08EDB2F1D15D4523D841F26E
:10CB6000E8230522E65041F2EC2341F2DE21E252B5
:10CB700041F2DA2304F59752E35A138041F2DC22A2
:10CB80000120A75203F6FB0292B2B2F5166F2ABF3C
:10CB9000653B6252635207B0BDE8F08F361A8BE7EF
:10CBA00010FB096688E70020F5E72846F3E700BF99
:10CBB000ADB5070080C1FFFFA35A01089E5A0108C6
:10CBC00038B50446FFF734FFB8B141F2EE25635D96
:10CBD0009BB941F238320121A35041F23C321C484A
:10CBE000A352FAF7A7F901211948FAF7AFF941F270
:10CBF00034336322E2540523635541F2EE22A35CF1
:10CC00002BB3013BDBB2012BA35420D104F5975386
:10CC100041F2E2211B8803F65F1292B2B2F5166F61
:10CC200028BF03F1FF3262525A1C92B2B2F5166F5E
:10CC300041F2E42124BFA3F65F1363524FF00103D6
:10CC400038BF6252237041F2EE230022E25438BD15
:10CC5000908A002041F23C3310B50446C05AB0B16E
:10CC600041F238337B22E358B3FBF0F3C3F30720E0
:10CC700081F8790081F87A300648FDF73DFF41F2EE
:10CC800038320023A35041F23C32A35210BD792226
:10CC9000F2E700BFE0D9002041F2E2232DE9F041A4
:10CCA000C15A41F2E423A4B0C25A41F2DA239142BC
:10CCB0000446C35A79D2994204D89A4202D32046F4
:10CCC000FFF7B6FE41F2DA23E25A41F2DE23E35ADD
:10CCD0009A4267D141F2EC2304F59755E35A052BAC
:10CCE00016D12B8803F65F1292B2B2F5166F41F29D
:10CCF000E22128BF03F1FF3262525A1C92B2B2F510
:10CD0000166F41F2E4212ABFA3F65F136252635209
:10CD100041F2DC2641F232384FF4F072A15B20463A
:10CD2000FFF7A0FD41F2103734F908300093B5F950
:10CD30000020E35F25492648FFF707FA34F9083059
:10CD40000293E35F0193082300934FF4F07205AB65
:10CD5000A15B2046FFF70AFE41F2EC23E55A013DB4
:10CD6000ADB2E55225BB1B491948FEF7A5F9294686
:10CD70001948FAF7DFF829461748FAF7E7F8144890
:10CD8000FDF7E8FE41F2DE2342F20F722570E25217
:10CD900041F234336322E25441F2EE23E55441F28E
:10CDA000E823E55024B0BDE8F081994285D886E7B4
:10CDB0002B1F5D425D4105A98DF81450FFF74AFF16
:10CDC00041F2E8230022E250ECE700BFB75A010825
:10CDD000E0D90020DE5A0108908A00202DE9F843AE
:10CDE00000F5965504460E46971E01EB430818358C
:10CDF00046453BD041F2383237F8020FA35836F996
:10CE0000021B0344A35041F23C320029A35A03F110
:10CE10000103A3522A8804EB820241F2DA29536803
:10CE20004FEA4303B8BF43F00103536034F80930BD
:10CE30000C33204624F813102378012B13D1FFF76D
:10CE40002BFF34F8093001339BB2B3F5166F28BFBE
:10CE5000002324F809302B8801339BB2042B88BFB0
:10CE600000232B80C4E7FFF7ABFEEAE7BDE8F883B9
:10CE700070B5044600254FF47A60258120806581D5
:10CE80006573257303F020FAC4E9045504F11C0608
:10CE90006060A56104F13C03324622F8025B9342D4
:10CEA000FBD104F2EC41002203F8012B9942FBD1A3
:10CEB000F023A4F8F0344FF49653C4F8EC2484F82B
:10CEC000F224C4F8F434C4F8F824002120223046B7
:10CED00003F032FB0523237409236382024B2046AF
:10CEE000C4E9053670BD00BFB4080020F0B590F964
:10CEF000F2341D4D1D4E002B1D4B8FB008BF1D463B
:10CF0000A3F2EE430A4640F2657740F2772C0EBF5B
:10CF10001E464FF46D774FF49E7C002302A902F069
:10CF2000C004802C1DD0C02C18D0002C0CBF2C4667
:10CF3000344621F8134001339200042BD2B2EED1D3
:10CF400004AA103002F0EAFA0023009304AA142382
:10CF500003210848FAF7C6FB0FB0F0BD21F81370A3
:10CF6000E9E721F813C0E6E7C4FEFFFF4CFCFFFF32
:10CF700089FDFFFF908A002010B58EB0002404AA1E
:10CF800002A904231030CDE9024402F0C7FA00944C
:10CF9000142304AA03210248FAF7A4FB0EB010BD23
:10CFA000908A002070B5B0F8EC3404461BB34948B1
:10CFB000494EF9F7A1FF0546142D1BD9B4F8EE34FC
:10CFC0005A1C2344A4F8EE2493F83C102046FFF7A3
:10CFD0008DFF3378143DADB21BB1D4F8F434C4F8EE
:10CFE000F834B4F8EE24B4F8EC349A42E4D30023D5
:10CFF000C4F8EC3470BD428903899BB293422DD1B1
:10D00000037BA3B1038893B1344B1B78002B3BD136
:10D01000B4F8F054772198B2A842B4F8EC242BD39A
:10D020000023A4F8EE34B4F8EC34002BBFD1D4F8CC
:10D03000F834002BDED02748F9F75EFF0546142DA3
:10D04000D8D92046FFF798FFD4F8F834143D013BB7
:10D05000ADB2C4F8F834002BF1D1CBE74389028993
:10D060009A429DBF42890188038903898CBF428906
:10D070005B189B1A9BB2C6E7501C2244A4F8EC0430
:10D08000013382F83C10C6E77823002021896289A9
:10D0900092B28A4203D1227B02F0FF016AB1616839
:10D0A000628992B2895C20736289013292B2628194
:10D0B00062892588954298BF6081B4F8EC24013BD1
:10D0C000551C224413F0FF03A4F8EC5482F83C10E2
:10D0D000DCD1A5E7908A002031070020CA9A002001
:10D0E00001EB4101890001F51671B1F5966F8ABF18
:10D0F0004FF49663A0F8F014A0F8F03470474FF4A2
:10D1000096635A4380F8F214C0F8F424704708B5C7
:10D11000F5F7A9F87823B0FBF3F0C0B208BD792A7F
:10D12000F8B504460D4624D1F5F79DF8772822D9A5
:10D1300001231946227B02F0FF002AB161730133FB
:10D14000792BF7D10020F8BD66682289EF5C92B296
:10D15000B7542289013292B22281228926889642CE
:10D1600098BF20812089628992B2824208BF2173D0
:10D17000E5E70420E7E70520E5E7000040F0BF60B1
:10D18000024B40F40030D860704700BF00ED00E073
:10D19000017870B501F01F0301269E40C3784D0948
:10D1A000CBB10F4BDA684378D243C2F30222C2F10B
:10D1B0000404E4B2A340DCB20F2343FA02F2837802
:10D1C0001340084A23431B011144DBB281F80033AA
:10D1D00042F8256070BD2035024B43F82560F9E721
:10D1E00000ED00E000E100E021F0604121F07F016E
:10D1F000014B01439960704700ED00E0054B19B108
:10D2000019690143196170471A6922EA00021A611B
:10D21000704700BF00ED00E0044B1A6804280CBF03
:10D2200042F0040222F004021A60704710E000E0AD
:10D2300008B501214FF4807000F0D8FF00214FF4B1
:10D240008070BDE8084000F0D1BF000043680A7953
:10D2500023F0407323F4807343EA02230A681343E4
:10D260004360D1E9032313438A6810B513438468EC
:10D27000084A224013434A7943EA420383600A7D05
:10D28000C36A013A23F47003D2B243EA0253C36281
:10D2900010BD00BFFDF7FFC0002303608380C0E91D
:10D2A000023303610123037570470000D0E90032A7
:10D2B000064910B513434C68054A2240134382685F
:10D2C0001343C26813434B6010BD00BF00230140ED
:10D2D000E030FCFF0023C0E90033C0E902337047AF
:10D2E000836819B143F001038360704723F00103A1
:10D2F000FAE7436823F4400323F4007319434160C1
:10D300007047416282627047436823F01F031943EC
:10D3100041607047044B5A6818B142F400025A60E9
:10D32000704722F40002FAE700230140044B5A68D8
:10D3300018B142F480025A60704722F48002FAE782
:10D3400000230140092970B51BD9A1F10A04C56861
:10D3500004EB44040726A64025EA060503FA04F474
:10D360002C43C460062A18D8013A436B02EB8202B0
:10D370001F24944023EA040301FA02F21A43426391
:10D3800070BD056901EB41060724B44025EA040598
:10D3900003FA06F42C430461E4E70C2A0CD8073A9C
:10D3A000036B02EB82021F24944023EA040301FA78
:10D3B00002F21A430263E3E70D3AC36A02EB820208
:10D3C0001F24944023EA040391401943C162D7E724
:10D3D000836843F08043836070478068C0F3807047
:10D3E0007047836819B143F480638360704723F406
:10D3F0008063FAE7836819B143F0020383607047E2
:10D4000023F00203FAE74368013923F4604343EA57
:10D41000413343607047436819B143F4006343608C
:10D42000704723F40063FAE7C06C80B270470000D5
:10D43000014B1868704700BF08230140836819B189
:10D4400043F480738360704723F48073FAE7836842
:10D4500019B143F400738360704723F40073FAE753
:10D46000044B5A6818B142F400525A60704722F4D3
:10D470000052FAE700230140092970B51CD9A1F137
:10D480000A04C56804EB44040726A64025EA0605FD
:10D4900003FA04F42C43C460836B0232C3F30154D7
:10D4A000121BD2B202EB82021F24944023EA04032F
:10D4B00091401943816370BD056901EB4106072462
:10D4C000B44025EA040503FA06F42C430461E3E7BB
:10D4D000836B013923F4401343EA0153836370479C
:10D4E00082B0002301930190019B19440191019B9B
:10D4F0001A6002B07047836823F470231943816077
:10D500007047836823F44013194381607047836830
:10D5100043F48003836070478068C0F38050704795
:10D52000436819B143F480634360704723F4806318
:10D53000FAE7436819B143F480534360704723F41A
:10D540008053FAE782B0002301930190019B2833B6
:10D5500019440191019B186880B202B07047012301
:10D56000C9B203FA01F1436812B11943416070472F
:10D5700023EA0101FAE70368194214BF01200020E1
:10D580007047C943016070474268006810EA112083
:10D5900007D00123C9B203FA01F1114214BF1846A2
:10D5A000002070476FEA11210160704708B5012122
:10D5B0004FF0005000F00CFE00214FF00050BDE88D
:10D5C000084000F005BE000030B5094C40F6FE737F
:10D5D0002268834022EA0302D1E900352B438D689B
:10D5E000C9682B430B4383401343236030BD00BF06
:10D5F000007400400023C0E90033C0E902337047E3
:10D60000012303FA00F0044B1A6811B110431860AB
:10D61000704722EA0000FAE7007400400123000985
:10D6200003FA00F0044B5A6811B110435860704778
:10D6300022EA0000FAE700BF00740040044B5A6879
:10D6400018B142F003025A60704722F00302FAE771
:10D650000074004001FA00F0044B1AB11A6802434A
:10D660001A6070471A6822EA0002F9E70074004065
:10D6700082B000230193054B0193019B08331844AA
:10D680000190019B196002B0704700BF0074004018
:10D6900082B000230193054B0193019B143318447E
:10D6A0000190019B196002B0704700BF00740040F8
:10D6B0000828044B0CBF42EA012242EA0142C25050
:10D6C000704700BF2074004082B000230193064BD6
:10D6D0000193019B2C3303EB90000190019B186890
:10D6E00080B202B0704700BF007400404FF4805316
:10D6F00003FA00F0044B1A6811B110431860704728
:10D7000022EA0000FAE700BF00740040FFF7A2BF62
:10D71000034B5B6B8140194214BF0120002070470E
:10D7200000740040014B8140596370470074004011
:10D73000054B81401A68586B084003D00A4214BF59
:10D7400001200020704700BF00740040014B814061
:10D75000596370470074004008B53C4B984209D1AA
:10D760000121084600F00AFD00210120BDE8084023
:10D7700000F004BD364B984206D10121022000F092
:10D78000FDFC00210220F1E7324B984206D1012135
:10D79000042000F0F3FC00210420E7E72E4B984220
:10D7A00006D10121082000F0E9FC00210820DDE776
:10D7B0002A4B984206D10121102000F0DFFC002105
:10D7C0001020D3E7264B984206D10121202000F0FB
:10D7D000D5FC00212020C9E7224B984206D1012127
:10D7E000402000F0CBFC00214020BFE71E4B9842B8
:10D7F00006D10121802000F0C1FC00218020B5E786
:10D800001A4B984208D101214FF4807000F0B6FC09
:10D8100000214FF48070A9E7154B984208D10121EF
:10D820004FF4007000F0AAFC00214FF400709DE757
:10D83000104B984208D101214FF4806000F09EFC0B
:10D8400000214FF4806091E708BD00BF0000024056
:10D850000004024000080240000C02400010024098
:10D860000014024000180240001C02400020024048
:10D8700000240240002802402DE9F0430D680022F8
:10D880000126032406FA02FE3EEA05033DD15700B5
:10D89000D0F800C004FA07F3DB430CEA030CC0F82D
:10D8A00000C091F804C0D0F800900CFA07F80CF111
:10D8B000FF3C48EA0908BCF1010FC0F8008017D806
:10D8C000D0F808C003EA0C0383604B79D0F808C095
:10D8D000BB4043EA0C038360436823EA0E034360C2
:10D8E0008B79D0F804C093409BB243EA0C034360A9
:10D8F000C36804FA07FC23EA0C03C360CB79D0F8B1
:10D900000CC0BB4043EA0C03C3600132102AB9D1FA
:10D91000BDE8F0834FF6FF720023C0E90023704793
:10D9200082B04FF480330193019B0B430193019B21
:10D93000C361C161019BC361C3690193C369019361
:10D9400002B070470369194214BF012000207047DC
:10D95000006980B270474369194214BF012000205A
:10D960007047406980B270470183704741837047B8
:10D970000AB1018370474183704741617047436931
:10D9800059404161704701F00703C90800EB81006D
:10D9900010B5016A9B000F249C4021EA040101623A
:10D9A000016A9A400A43026210BD000008B5144B98
:10D9B00098420BD101214FF4001000F009FC002126
:10D9C0004FF40010BDE8084000F002BC0D4B984237
:10D9D00008D101214FF4800000F0FAFB00214FF440
:10D9E0008000EFE7084B984208D101214FF4000076
:10D9F00000F0EEFB00214FF40000E3E708BD00BF9C
:10DA00000054004000580040005C00407FB586880C
:10DA100026F03F060446360468460D46360C00F0F4
:10DA20007FFA029A2949B2FBF1F188B20643A68037
:10DA30002388274E23F001031B041B0C23802B6833
:10DA4000B3421ED85B000130B2FBF3F39BB2042B50
:10DA500080B238BF04232084A3832388AA886989DD
:10DA600043F001032380238823F481630A4323F0D6
:10DA70000203134323802A89AB891343238104B013
:10DA800070BDEE884BF6FF7086421BBF19204343E2
:10DA900003EB4303B2FBF3F315BF9BB2B2FBF3F30B
:10DAA00043F480439BB2C3F30B020AB943F0010372
:10DAB0004FF496724A434FF47A71B2FBF1F201329D
:10DAC00092B243F400432284C6E700BF40420F00F5
:10DAD000A0860100054B41F28832C0E900230023F3
:10DAE00083604FF480438381704700BF0000FFBF15
:10DAF000038819B143F001030380704723F0010349
:10DB00001B041B0CF8E7838C29B123F010031B04C2
:10DB10001B0C8384704743F01003FAE7838C9BB29D
:10DB200001F00F0123F00F030B4383847047038838
:10DB300019B143F480730380704723F480731B048E
:10DB40001B0CF8E7038819B143F400730380704796
:10DB500023F400731B041B0CF8E722B141F0010110
:10DB600089B20182704701F0FE01F9E7038819B11B
:10DB700043F480630380704723F480631B041B0C11
:10DB8000F8E783899BB201F0FE0123F0FE030B430B
:10DB900083817047838919B143F001038381704702
:10DBA00023F001031B041B0CF8E7038819B143F0B1
:10DBB00040030380704723F040031B041B0CF8E76D
:10DBC000038819B143F4004303807047C3F30E0385
:10DBD000FAE7038819B943F080030380704723F004
:10DBE00080031B041B0CF8E7838BB1F5804F1DBF2E
:10DBF00023F480431B041B0C43F48043838370474E
:10DC00000388B1F5006F1BBF23F400631B0443F4CA
:10DC100000631B0C038070470388B1F5005F1BBFD6
:10DC200023F400531B0443F400531B0C0380704780
:10DC3000038819B143F010030380704723F01003E9
:10DC40001B041B0CF8E701827047008AC0B27047C2
:10DC5000038819B143F480530380704723F4805341
:10DC60001B041B0CF8E7FFF7CBBF038819B143F087
:10DC700020030380704723F020031B041B0CF8E7EC
:10DC8000008B000A7047838819B143F400638380D6
:10DC9000704723F400631B041B0CF8E7838819B159
:10DCA00043F480538380704723F480531B041B0C80
:10DCB000F8E782B0002301930190019B1944019180
:10DCC000019B188802B07047838812B11943818084
:10DCD000704723EA0101FAE7838A008B43EA004395
:10DCE0000B4023F07F435B1A584258417047838AA8
:10DCF000008B43EA004020F07F40704782B0002351
:10DD0000009301930B0F01900093009B21F07F4142
:10DD100053B1019B14330193019B1B680B4214BF49
:10DD20000120002002B07047019B090C1833F2E774
:10DD3000C94389B2818270478388808A08409BB238
:10DD400006D003EA114313F4E06F14BF0120002052
:10DD50007047C94389B28182704700000E4B1A6830
:10DD6000002142F001021A6099601A6822F0A8525C
:10DD700022F410221A60094A5A60094AC3F8842022
:10DD800002F18062C3F888201A6822F480221A60A7
:10DD9000D960C3F88C10704700380240103000245E
:10DDA00000300020024B00221A701870704700BF2C
:10DDB00002380240034A136823F0F80343EAC00024
:10DDC0001060704700380240014B1860704700BF78
:10DDD00000004742064B002201281A701A7002D038
:10DDE000042802D070471870704705221A707047D7
:10DDF00070380240014B1860704700BF800E4742E8
:10DE000010B5029C40EA0460039C40EA0470084399
:10DE10005B08013B40EA821040EA0340014B586036
:10DE200010BD00BF00380240014B1860704700BFB2
:10DE30006000474210B5029C240744EA036404438F
:10DE4000520844EA8114013A024B44EA0244C3F8FE
:10DE5000844010BD00380240014B1860704700BF7D
:10DE60006800474240EA036343EA81115308013BDB
:10DE7000024A41EA0343C2F8883070470038024042
:10DE8000014B1860704700BF70004742014B18609B
:10DE9000704700BF4C004742034A936823F0EC638D
:10DEA000194301439160704700380240034A936868
:10DEB00023F07843194301439160704700380240D2
:10DEC000034A936823F0030318439060704700BF30
:10DED00000380240024B986800F00C00704700BF09
:10DEE00000380240034A936823F0F003184390601F
:10DEF000704700BF00380240034A936823F4E053A0
:10DF000018439060704700BF00380240034A93688E
:10DF100023F4604343EAC000906070470038024039
:10DF2000294A936803F00C03043B10B5082B06D86C
:10DF3000DFE803F01E050505200505053700234B26
:10DF4000214A036093682249C3F30313CC5C03683E
:10DF5000E34043609468C4F382240C5D23FA04F424
:10DF600084609268C2F342328A5CD340C36010BDC1
:10DF7000184BE5E75468516852686402C2F388128E
:10DF800001F03F014CBF134B104BB3FBF1F3534374
:10DF90000D4A5268C2F3014201325200B3FBF2F360
:10DFA000CEE75468516852686302C2F3881201F0E8
:10DFB0003F014CBF074B054BB3FBF1F35343024A00
:10DFC0005268C2F30272E7E7003802400024F4000E
:10DFD0000E09002000127A0000F44073B3F5407F70
:10DFE000084A08D1916820F0704321F4F81123F415
:10DFF00040730B439360136FC0F30B00184310671B
:10E00000704700BF00380240014B1860704700BFE6
:10E010003C0E4742014B1860704700BF400E47421C
:10E020000D4B58B9D3F88C0020F0C060C3F88C00B9
:10E03000D3F88C000843C3F88C007047D3F88C00E9
:10E0400020F0C050C3F88C00D3F88C2042EA810243
:10E05000C3F88C20704700BF003802400D4B58B900
:10E06000D3F88C0020F44010C3F88C00D3F88C0057
:10E070000843C3F88C007047D3F88C0020F44000AC
:10E08000C3F88C00D3F88C2042EA8102C3F88C20BC
:10E09000704700BF00380240044AD2F88C30013883
:10E0A00023F01F031843C2F88C0070470038024069
:10E0B000054AD2F88C30013823F4F85343EA0023A0
:10E0C000C2F88C30704700BF00380240044AD2F8D2
:10E0D0008C3023F440331843C2F88C00704700BFE3
:10E0E00000380240014B1860704700BFE011474202
:10E0F000054B19B1196B0143196370471A6B22EA7A
:10E1000000021A63704700BF00380240054B19B186
:10E11000596B0143596370475A6B22EA00025A63F4
:10E12000704700BF00380240054B19B1996B01439D
:10E13000996370479A6B22EA00029A63704700BFA6
:10E1400000380240054B19B1196C0143196470473E
:10E150001A6C22EA00021A64704700BF00380240BD
:10E16000054B19B1596C0143596470475A6C22EA46
:10E1700000025A64704700BF00380240054B19B1D5
:10E1800019690143196170471A6922EA00021A618C
:10E19000704700BF00380240054B19B1596901436F
:10E1A000596170475A6922EA00025A61704700BFFC
:10E1B00000380240054B19B19969014399617047D4
:10E1C0009A6922EA00029A61704700BF0038024053
:10E1D000054B19B1196A0143196270471A6A22EA9C
:10E1E00000021A62704700BF00380240054B19B1A7
:10E1F000596A0143596270475A6A22EA00025A6218
:10E20000704700BF00380240054B19B1196D01433A
:10E21000196570471A6D22EA00021A65704700BF3F
:10E2200000380240054B19B1596D014359657047DB
:10E230005A6D22EA00025A65704700BF003802405A
:10E24000054B19B1996D0143996570479A6D22EAA2
:10E2500000029A65704700BF00380240054B19B1B3
:10E26000196E0143196670471A6E22EA00021A6697
:10E27000704700BF00380240054B19B1596E014389
:10E28000596670475A6E22EA00025A66704700BF0C
:10E2900000380240044B1A6F01280CBF42F00802FC
:10E2A00022F008021A67704700380240054BD3F885
:10E2B000942001280CBF42F0006222F00062C3F8F3
:10E2C0009420704700380240054BD3F89420012871
:10E2D0000CBF42F0805222F08052C3F89420704765
:10E2E00000380240074B31B1D3F8901021EA000109
:10E2F000C3F890107047D3F890200243C3F89020E1
:10E30000704700BF00380240054BD3F89420012825
:10E310000CBF42F0005222F00052C3F89420704724
:10E3200000380240054BD3F8942001280CBF42F07E
:10E33000806222F08062C3F8942070470038024067
:10E34000064BD3F8942022F44002C3F89420D3F86B
:10E3500094201043C3F89400704700BF0038024077
:10E36000054B19B119780143197070471A7822EAE0
:10E3700000021A70704700BF0D3802404209012A9E
:10E38000074B07D11B6800F01F0023FA00F000F0D4
:10E3900001007047022A0CBF1B6F5B6FF3E700BFE1
:10E3A0000038024007B5002301933120FFF7E6FF54
:10E3B000019B01330193019BB3F5A04F01D00028CD
:10E3C000F3D03120FFF7DAFF003018BF012003B08F
:10E3D0005DF804FB024A536F43F080735367704744
:10E3E00000380240034BDB68184214BF01200020B4
:10E3F000704700BF00380240014B1870704700BFE3
:10E400000E38024030B5048C24F001042404240C9E
:10E410000484048B058C24F0F304ADB22404240C92
:10E4200042EA031325F00A051C430D43A4B245F04C
:10E4300001050483058430BD30B5048C24F010043C
:10E440002404240C0484058B048C25F44075A4B2A8
:10E450002D05120224F0A0042D0D42EA033344EAF4
:10E4600001141D43A4B2ADB244F01004058304842A
:10E4700030BD000008B54D4B984209D10121084636
:10E48000FFF7B4FE00210120BDE80840FFF7AEBE53
:10E49000B0F1804F09D101210846FFF799FE002114
:10E4A0000120BDE80840FFF793BE414B984206D1DA
:10E4B00001210220FFF78CFE00210220F1E73D4BF5
:10E4C000984206D101210420FFF782FE002104209A
:10E4D000E7E7394B984206D101210820FFF778FE83
:10E4E00000210820DDE7354B984206D1012110209C
:10E4F000FFF76EFE00211020D3E7314B984206D182
:10E5000001212020FFF764FE00212020C9E72D4BC8
:10E51000984206D101210220FFF768FE0021022067
:10E52000B2E7294B984208D101214FF48030FFF720
:10E530005DFE00214FF48030A6E7244B984208D1BD
:10E5400001214FF40030FFF751FE00214FF400305D
:10E550009AE71F4B984208D101214FF48020FFF722
:10E5600045FE00214FF480208EE71A4B984206D1D9
:10E5700001214020FFF72CFE0021402091E7164B9F
:10E58000984206D101218020FFF722FE0021802041
:10E5900087E7124B984208D101214FF48070FFF7B2
:10E5A00017FE00214FF480707BE708BD000001409A
:10E5B0000004004000080040000C00400010004033
:10E5C00000140040000401400040014000440140AC
:10E5D0000048014000180040001C0040002000409E
:10E5E0001C4A038890429BB212D002F5806290428E
:10E5F0000ED0B0F1804F0BD0A2F58032904207D000
:10E6000002F58062904203D002F58062904203D10D
:10E610004A8823F0700313430F4A904208D002F552
:10E62000806290421FBF23F440730A899BB2134358
:10E6300003804B68C3620B880385064B984203D066
:10E6400003F58063984201D18B7A0386012383828C
:10E65000704700BF000001400010004000234FF051
:10E66000FF32C0E9003203818372704701858282E4
:10E670007047038823F070031B041B0C19430180AF
:10E68000704741627047C1627047406A7047008DB1
:10E690007047038819B143F002030380704723F0E9
:10E6A00002031B041B0CF8E7038819B143F00403B1
:10E6B0000380704723F004031B041B0CF8E7038856
:10E6C00019B143F080030380704723F080031B04DB
:10E6D0001B0CF8E7038823F008031B041B0C0380C2
:10E6E0000388194301807047038823F440731B0497
:10E6F0001B0C03800388194301807047038819B1FC
:10E7000043F001030380704723F001031B041B0C3B
:10E71000F8E70000038C23F001031B041B0C0384A7
:10E7200070B5038C8288048B0D884E8824F07304A6
:10E730002404240C2C4323F002038D891B0435434D
:10E740001B0C2B430D4DA84292B203D005F58065FA
:10E75000A8420DD1CD894E8A23F008032B438D8822
:10E7600023F004032B430D8A22F4407235432A43DD
:10E7700082808A6804834263038470BD0000014084
:10E78000038C23F010031B041B0C038470B5038C53
:10E790008488028B0D884E8822F4E6421204120C03
:10E7A00042EA052223F020038D891B0435431B0C0C
:10E7B00043EA0513114DA842A4B292B29BB203D012
:10E7C00005F58065A84213D1CD894E8A23F08003D8
:10E7D00043EA05134FF6BF751D408B8845EA0313C6
:10E7E0000D8A24F44064354344EA85049BB2A4B204
:10E7F000848002838A688263038470BD00000140C4
:10E80000038C23F480731B041B0C038470B5038CEE
:10E810008288848B0D884E8824F073042404240C91
:10E820002C4323F400738D891B0435431B0C43EAEE
:10E830000523114DA84292B29BB203D005F5806525
:10E84000A84213D1CD894E8A23F4006343EA0523FD
:10E850004FF6FF351D408B8845EA03230D8A22F4CD
:10E860004052354342EA05129BB292B282808A68D6
:10E870008483C263038470BD00000140038C23F4D1
:10E8800080531B041B0C038470B5038C8488828B1B
:10E890000D884E8822F4E6421204120C42EA052248
:10E8A00023F400538D891B0435431B0C43EA0533C5
:10E8B0000A4DA842A4B292B29BB203D005F580657E
:10E8C000A84205D10D8A24F4804444EA8514A4B2F8
:10E8D000848082838A680264038470BD00000140E2
:10E8E000002303608380C0E902330361704730B5C1
:10E8F000048C01258D4024EA050400F118030484EA
:10E9000021F0080050B94908C85820F070000004F0
:10E91000000CC850C8580243CA5030BD0439C1F376
:10E920004E011202C85820F4E0400004000CC85008
:10E9300092B2C858EFE74163704781637047C16383
:10E94000704701647047038B23F070031B041B0C9A
:10E95000194301837047038B23F4E0431B041B0C12
:10E9600043EA012189B201837047838B23F070034E
:10E970001B041B0C194381837047838B23F4E043F2
:10E980001B041B0C43EA012189B281837047038B6E
:10E9900023F008031B041B0C194301837047038BEE
:10E9A00023F400631B041B0C43EA012189B2018399
:10E9B0007047838B23F008031B041B0C19438183CE
:10E9C0007047838B23F400631B041B0C43EA012173
:10E9D00089B281837047038B23F004031B041B0C53
:10E9E000194301837047038B23F480631B041B0CC2
:10E9F00043EA012189B201837047838B23F004032A
:10EA00001B041B0C194381837047838B23F48063A1
:10EA10001B041B0C43EA012189B281837047038BDD
:10EA200023F080031B041B0C194301837047038BE5
:10EA3000C3F30E0343EA012189B201837047838B3C
:10EA400023F080031B041B0C194381837047838BC5
:10EA5000C3F30E0343EA012189B281837047038C1B
:10EA600023F002031B041B0C194301847047038C21
:10EA700023F008031B041B0C194301847047038C0B
:10EA800023F020031B041B0C43EA011189B201840B
:10EA90007047038C23F080031B041B0C43EA011115
:10EAA00089B201847047038C23F400731B041B0C90
:10EAB00043EA012189B201847047038C23F4006387
:10EAC0001B041B0C43EA012189B201847047038CAB
:10EAD00023F400531B041B0C43EA013189B2018467
:10EAE0007047038C10B501248C4023EA040303848F
:10EAF000038C02FA01F1194389B2018410BD038C21
:10EB000010B504248C4023EA04030384038C02FA26
:10EB100001F1194389B2018410BD00230122038051
:10EB200043808280C38003817047406B7047806B55
:10EB30007047C06B7047006C7047038B23F00C0369
:10EB40001B041B0C0383038B194301837047038B46
:10EB500023F440631B041B0C0383038B43EA012152
:10EB600089B201837047F8B50C464988A288B4F889
:10EB700000C0238900290CBF02260026012A0CBFF1
:10EB800002270127BCF1000F0ED1FFF73BFCE18803
:10EB9000FFF7D3FF314623893A46FFF74DFCE18862
:10EBA000BDE8F840FFF7D3BFFFF746FCE188FFF769
:10EBB000CEFF314623893A46FFF724FCE188BDE8C1
:10EBC000F840FFF7BABF838B23F00C031B041B0C28
:10EBD0008383838B194381837047838B23F4406342
:10EBE0001B041B0C8383838B43EA012189B281833D
:10EBF0007047F8B50D460E88AA8849882B8936B922
:10EC0000FFF700FCE988BDE8F840FFF796BF042E47
:10EC100006D1FFF711FCE988BDE8F840FFF797BF80
:10EC2000082EEF88058C1CD125F480752D042D0C41
:10EC30000584868B058CB6B2ADB226F0F30625F4BA
:10EC4000206545EA0125164346EA0316ADB2B6B281
:10EC500045F48075868339460584BDE8F840FFF7A2
:10EC6000B2BF25F480552D042D0C0584B0F81CC0CE
:10EC7000058C25F400552CF4407C6D041E034FEAEE
:10EC80000C5C6D0C45EA01354FEA1C5C46EA022635
:10EC90004CEA0606ADB2B6B245F4805586833946D5
:10ECA0000584BDE8F840FFF798BF4A880B881343F6
:10ECB0008A881343CA8813430A8913434A89134332
:10ECC0008A891343A0F844307047002303804380AF
:10ECD0008380C3800381438183817047B0F84430CF
:10ECE00021B143F40043A0F844307047C3F30E034E
:10ECF000F9E7838819B143F004038380704723F058
:10ED000004031B041B0CF8E7838819B143F00103CB
:10ED10008380704723F001031B041B0CF8E78389F1
:10ED200012B119438181704723EA0101FAE7818218
:10ED30007047038A194214BF012000207047C9435D
:10ED400089B201827047038A828911EA030092B274
:10ED500003D00A4214BF012000207047C94389B282
:10ED6000018270470A43A0F848207047FFF7D7BFD9
:10ED7000838819B143F008038380704723F00803A8
:10ED80001B041B0CF8E7038923F007031B041B0C6F
:10ED900003817047038923F070031B041B0C194384
:10EDA0000181038943F007030381704738B50D469D
:10EDB000602D114604464FF001020DD1FFF73CFBD8
:10EDC000218921F070010904090C2943218123893B
:10EDD00043F00703238138BDFFF714FBF0E70389F5
:10EDE00023F070031B041B0C1943018170478388B7
:10EDF00023F070031B041B0C8380838819438180DC
:10EE00007047038923F007031B041B0C038103894C
:10EE1000194301817047038923F080031B041B0CF5
:10EE20000381038919430181704710B504890A439E
:10EE3000E4B242EA03231C43A4B2048110BD10B51E
:10EE4000FFF7F3FF038923F077031B041B0C43F048
:10EE50007703038110BD10B5FFF7E7FF038943F483
:10EE60008043038110BD70B50589068B048C25F0A5
:10EE700007052D042D0C24F022042943240426F434
:10EE8000407525F00305240C42EA031345F4807510
:10EE90001C4345F00105A4B201810583048470BDC3
:10EEA000838819B143F080038380704723F0800387
:10EEB0001B041B0CF8E7A0F85010704708B5314B45
:10EEC000984209D101211020FFF790F9002110206C
:10EED000BDE80840FFF78AB92B4B98420BD10121BE
:10EEE0004FF40030FFF774F900214FF40030BDE813
:10EEF0000840FFF76DB9254B984208D101214FF426
:10EF00008020FFF765F900214FF48020EFE7204BC8
:10EF1000984208D101214FF40020FFF759F9002150
:10EF20004FF40020E3E71B4B984208D101214FF436
:10EF30008010FFF74DF900214FF48010D7E7164BF2
:10EF4000984206D101212020FFF750F9002120200E
:10EF5000BEE7124B984208D101214FF08040FFF7E5
:10EF600037F900214FF08040C1E70D4B984208D19E
:10EF700001214FF00040FFF72BF900214FF0004036
:10EF8000B5E708BD001001400044004000480040C3
:10EF9000004C004000500040001401400078004048
:10EFA000007C0040028A30B50D4692B2EB88898918
:10EFB00022F440521A4302828389044623F4B05259
:10EFC0002889AB880343688922F00C02034313436A
:10EFD000A381A38A9BB223F440730B4385B0A38221
:10EFE0006846FEF79DFF1A4B9C4203D003F58063F1
:10EFF0009C4222D10399A2891923100403FB01F337
:10F00000A28929684FF064054CBF490089001204A9
:10F01000B3FBF1F1B1FBF5F34FEA031005FB13135A
:10F020000DD5DA003232B2FBF5F202F0070242EA05
:10F0300000039BB2238105B030BD0299DBE71B01C1
:10F040003233B3FBF5F303F00F030343F1E700BFE3
:10F05000001001404FF416520023C0E900234FF482
:10F060004022826083817047038A9BB223F47062DE
:10F0700010B50B884C8823438C88C98823430B43E5
:10F080001343038210BD0023038043808380C38029
:10F090007047838919B143F400538381704723F487
:10F0A00000531B041B0CF8E7038B03F47F4303831B
:10F0B000038B194301837047838919B143F40043DB
:10F0C00083817047C3F30E03FAE7838A19B143F4CF
:10F0D00000638382704723F400631B041B0CF8E772
:10F0E000C1F30801818070478088C0F30800704731
:10F0F000038A23F00F031B041B0C0382038A1943AA
:10F1000001827047838919B143F0020383817047FC
:10F1100023F002031B041B0CF8E7838923F400632C
:10F120001B041B0C83818389194381817047038AE7
:10F1300023F020031B041B0C0382038A1943018262
:10F140007047038A19B143F480430382704723F464
:10F1500080431B041B0CF8E7838943F00103838180
:10F160007047838A19B143F008038382704723F004
:10F1700008031B041B0CF8E7038BDBB20383038B30
:10F1800043EA012101837047838A19B143F02003C8
:10F190008382704723F020031B041B0CF8E7838A4B
:10F1A00019B143F010038382704723F010031B044E
:10F1B0001B0CF8E7838A23F004031B041B0C8382D7
:10F1C000838A194381827047838A19B143F002030D
:10F1D0008382704723F002031B041B0CF8E7838A29
:10F1E00012B119438182704723EA0101FAE710B591
:10F1F000C1F3421401F01F03012C4FF0010101FA89
:10F2000003F105D10C3003683AB11943016010BD18
:10F21000022C0CBF10301430F5E723EA0101F5E7AA
:10F220000388194214BF012000207047C94389B2E6
:10F2300001807047C1F3421210B5012301F01F0491
:10F24000012A03FA04F30DD182891340028892B295
:10F250006BB10123090A03FA01F10A4214BF1846EF
:10F26000002010BD022A0CBF028A828AEDE71846F0
:10F27000F7E7090A01238B40DB439BB20380704709
:10F280003F4AD2F8883043F47003C2F888303D4BCF
:10F290001A68002142F001021A6099601A6822F08F
:10F2A000847222F480321A60374A5A601A6882B037
:10F2B00022F480221A60D960009101911A6842F408
:10F2C00080321A6019461A6802F400320192009ADC
:10F2D00001320092019A1AB9009AB2F5A04FF2D108
:10F2E0000B6813F4003318BF01230193019B012B1A
:10F2F0003FD1244B1A6C42F080521A64234A1168A1
:10F3000041F44041116099689960996841F4004165
:10F310009960996841F4A05199601D495960196834
:10F3200041F08071196019688901FCD5136843F4B4
:10F3300080331360154B19465A68D203FCD51A68FE
:10F3400042F400321A604B689B03FCD5114B40F22B
:10F3500005721A60A3F580639A6822F003029A602E
:10F360009A6842F002029A609A6802F00C02082A37
:10F37000FAD1034B4FF000629A6002B0704700BFB1
:10F3800000ED00E000380240103000240070004022
:10F39000085A4077003C0240234A2449936803F00E
:10F3A0000C03043B10B5082B06D8DFE803F0110569
:10F3B0000505130505052A001D4B0B601A4B1D4A58
:10F3C0009B68C3F30313D25C0B68D3400B6010BD82
:10F3D000194BF2E75468506852686402C2F388120D
:10F3E00000F03F004CBF144B114BB3FBF0F3534301
:10F3F0000D4A5268C2F3014201325200B3FBF2F3EC
:10F40000DBE75468506852686302C2F3881200F068
:10F410003F004CBF084B064BB3FBF0F35343024A8B
:10F420005268C2F30272E7E7003802403009002058
:10F430000024F4001E09002000127A0038B50446AA
:10F440000D46AC4200D338BD54F8043B9847F8E76A
:10F45000FEE7000008B5104A104B11498B4216D345
:10F46000144815494FF000028842B8BF40F8042BF9
:10F47000FADBFFF705FF0B490B48FFF7DFFF0B49EE
:10F480000B48FFF7DBFFBDE80840F9F75BBA52F81D
:10F49000040B43F8040BE1E728AA0408000000204D
:10F4A0009C0900200CAA04080CAA040818AA040845
:10F4B0000CAA0408A00900206C1401202DE9F00317
:10F4C0005FEA92098446884619D000F108040B4689
:10F4D0004F4614E90300060C0D0C360400042D04FD
:10F4E0000904013F83E84100DD60996004F10804EC
:10F4F00003F11003EDD10CEBC90C08EB091812F065
:10F50000030207D03CF9023B013A4FEA034348F8B3
:10F51000043BF7D1BDE8F003704700BF2DE9F00FC1
:10F52000A0B00E901A910E99408889681B910E9C8C
:10F530001B9E1D9000F10041013903F00100646839
:10F54000119406EB41015B08149219911E901F93D0
:10F5500000F0E2800C461D991D9B30461A9E8908DA
:10F56000CA0004360C9103F00303043402301F99DF
:10F570001C920F93169417960D9018913246169C74
:10F5800032F8043C24F8043C32F8023C0E9E24F885
:10F59000023C36781596002E00F0A6810D9A1C9933
:10F5A000149C08941144B146701C012613911290CA
:10F5B0000996CDF81C9049463246881A119C0D9E3A
:10F5C0000C9A36F8021C04EB4000002A78D0079B06
:10F5D00010901446DB004FF0000A4FF0000B01942E
:10F5E000079C0693D046D9463246034615881E88A6
:10F5F00033F81400B2F802C033F82470C6FB85ABB0
:10F60000C1FB86894FF0060616FB0431C5FB8089D5
:10F6100096880D88D188C0FB8CABCCFB8789C7FB53
:10F6200086ABC6FB8589019E0698013E0344C5FB57
:10F6300081AB02F108020196D8D103460C9A1098CA
:10F64000139D03FB02000F9C74B1079A23465600DA
:10F6500000E0A1B2028835F8024B013B3044C2FB06
:10F6600084ABC1FB8289F4D14FEAD83343EA4944E1
:10F670000899029420464FEAE9364FEADA320E9CA6
:10F6800000F30F0303960B8042EA4B460998237858
:10F6900004964FEAEB3134460591089E129904F323
:10F6A0000F02013026F81320884206F10206099065
:10F6B00008960DD00E9A127807921146099A7CE7A7
:10F6C0004FF0000A4FF0000B3546D046D946BAE756
:10F6D000149C159B0E9E04EB43043378149420462F
:10F6E00000EB43001699179A0D9B189C1490043157
:10F6F00004320433013C169117920D9318947FF451
:10F700003EAF1F9E19981A991B9CB30018441944C8
:10F710001C4419901A911B941E9E002E00F0A0808C
:10F720001D981D9A1B9C10968008C10002F00302D0
:10F7300002901291079209941A9E199836F8023B8A
:10F7400020F8023B0E991A96097819900F9100291A
:10F7500079D0129B099C149E04964A1C01202344D4
:10F760000C920D938A4606900246119C029EC2EBB3
:10F770000A0104EB4101002E00F0B0804FF00200BE
:10F780001AFB00F04FEA400C04466444099A0190C9
:10F790004FEA800B0B4630464FF000084FF000094F
:10F7A000089127461D88168833F81A105488C6FB1E
:10F7B00085893CF803509688C4FB8189D95BD4883D
:10F7C000C6FB858901385B44C4FB818902F10802CC
:10F7D000E8D1019B0899029C4FF0020212FB0A3B00
:10F7E00012FB0ABB12FB0ABB0D9A04FB0B11079E0E
:10F7F00056B14FEA4A0A3346088832F8024B013BB9
:10F800005144C4FB8089F7D14FEAD830069A049E50
:10F8100040EA49414FEAE9330C980B9301320C4618
:10F8200004F30F0326F8023B82420A9106920496E3
:10F8300004D00E9C069A94F800A096E714980F9EA8
:10F8400000EB460014900999109A0231013A09918F
:10F8500010927FF471AF1B9C1E9E04EB46041B9418
:10F860001D980E9C471EBD08A06829D01B9E00F164
:10F87000080206F10803964238BF984234BF0021BF
:10F880000121022D94BF002101F0010179B346EA64
:10F89000000189072BD10021013153F8086C53F87E
:10F8A000044C42F8044CA94242F8086C03F10803E6
:10F8B00002F10802F0D11B99ED00294428441B9164
:10F8C00017F0030706D01B9B33F8022B20F8022BFE
:10F8D000013FF9D120B0BDE8F00F7047099A4FF011
:10F8E00000084FF0000982E733461498F8E61B9BA6
:10F8F000024629461C8814805C8854809C88948029
:10F90000DC88D480013903F1080302F10802F1D147
:10F91000D1E700BF2DE9F00F92B00F9010930F9B2D
:10F9200000885B680A930E9000F100430F9C0A9DCB
:10F930001098A4680994013B05EB430380080791E4
:10F9400008920693119000F0A9808B460E990290C0
:10F950008908CA009A4614440E9B0D94089C049191
:10F9600003F003030B93083453460835DA460C9230
:10F97000019400959B46BAF80030ABF80030BAF815
:10F980000230ABF80230BAF80430ABF80430BAF801
:10F99000063000980499ABF8063010E90C000029F5
:10F9A00000F0FA8000F10804099803940E46002143
:10F9B0002546CDF814A089460F468C4600F1080470
:10F9C000B24654F8086C22FB06CC23FB0699C3EA26
:10F9D000020855F8082C28FB1677C2EA030828FB12
:10F9E000161654F8040C23FB00CC55F8043C22FBFB
:10F9F000009928FB1077C3EA020121FB1061BAF1DC
:10FA0000010A05F1080504F10804DAD1009C0C98FC
:10FA1000DDF814A020440D9C0B9D6DB1246822FBE1
:10FA200004CC23FB0499C3EA020222FB1477026888
:10FA3000C2EA030323FB14110198029B039A00926C
:10FA40004FEAEC3CFF130CF30F0C07F30F074FEAE0
:10FA5000E939CCEA074709F30F0940F8087CC913D4
:10FA6000083001F30F01013BC9EA014140F80C1CC9
:10FA70000AF1080A0BF1080B019002937FF47BAFA7
:10FA8000119C069D07980899E3000A9C1D441844A0
:10FA900019441C440695079008910A94109D15F08E
:10FAA0000305009539D009980E9B0A9C00F1040BC0
:10FAB0004FEA530AA8464FF0000C04F10409079DD1
:10FAC000069835F80C3020F80C305A4609EB0C0338
:10FAD0005146002033F8047C32F8046C33F8025CA1
:10FAE00032F8024C17FB0600013903F1040315FB41
:10FAF000040002F10402EDD10899B8F101084FEABF
:10FB0000E03000F30F0021F80C000CF1020CD6D10C
:10FB10000A9B009C03EB44030A930E9D0F986F1EF3
:10FB2000BE0845682AD00A9B0A9C03F1080205F129
:10FB300008039C4238BF954234BF00210121022EA8
:10FB400094BF002101F0010171B344EA0501890766
:10FB50002AD10021013152F8084C52F8040C43F824
:10FB6000040CB14243F8084C02F1080203F1080307
:10FB7000F0D10A98F600304435440A9017F0030398
:10FB800006D00A9A32F8021B25F8021B013BF9D174
:10FB900012B0BDE8F00F704700F10805099C03950D
:10FBA00089460F468C4637E70A9A2B46314610881D
:10FBB00018805088588090889880D088D8800139E3
:10FBC00002F1080203F10803F1D1D2E72DE9F00FA9
:10FBD0002DED108B8AB00290029C0088D4F804802E
:10FBE000019000F1804A0AF1FF3AD8080393D4F853
:10FBF0000890049008EB8A0A00F0E181019BCDF89F
:10FC000018A0D808430109EB03041C330593019B9A
:10FC1000009403F0070B049BCDF81C805446DDF8DC
:10FC200014A008910E4608F11C0C47461546D8460C
:10FC3000194609923368236073686360B368A360F0
:10FC4000F368E3603369236173696361B369A36136
:10FC50009FEDAB8AF369E361D7ED004AD7ED017AF6
:10FC600097ED027AD7ED036A97ED046AD7ED055A4E
:10FC700097ED065A6246F0EE488AB0EE489AF0EEEA
:10FC8000489AB0EE48AAF0EE48AAB0EE48BAF0EEB4
:10FC900048BA002800F0DF814A466346834692ED69
:10FCA000000AD3ED003AD2ED010A92ED021AD2ED2C
:10FCB000031A92ED042AD2ED052A92ED063A92ED4E
:10FCC000074A24EE80EA27EE80FAD3ED014A27EEB8
:10FCD00000CA66EE80DA26EE00DA65EE80CA65EECE
:10FCE00000EA23EE800A67EE20FA7BEE8EBA3BEE46
:10FCF0000FBA27EEA0EA26EEA0FAD3ED027A7AEE4A
:10FD00008CAA3AEE2DAA26EE20CA65EEA0DA79EE8C
:10FD10008D9A39EE2C9A25EE20DA78EEAE8A38EEFE
:10FD2000008A63EEA0EA64EEA00A27EE010A63EE01
:10FD300081CA93ED037A7BEE8EBA3BEE2FBA26EEA4
:10FD400081EA66EE01FA7AEE8FAA3AEE0CAA25EE67
:10FD500081FA25EE01CA79EEAD9A39EE0D9A78EE68
:10FD6000AE8A38EE208A64EE81EA27EE811A66EECA
:10FD7000A10A63EEA1DAD3ED046A3AEE0FAA24EEEB
:10FD8000A1DA7BEE80BA3BEE0EBA25EE210A26EE12
:10FD900021EA7AEEAFAA79EE8C9A65EEA1FA39EEF5
:10FDA0002C9A78EEAE8A38EE018A67EEA1EA67EE09
:10FDB000211A65EE82CA26EE02FA7AEEAFAA93ED18
:10FDC000056A25EE02CA3AEE000A79EEAD9A39EEDE
:10FDD0000D9A7BEEA0BA3BEE0EBA64EE82DA23EE09
:10FDE00082EA27EE82DA78EEAE8A38EE218A67EE72
:10FDF00002EA26EE822A25EE22AA65EEA2FA3AEE61
:10FE00008CCA39EE0DDA63EEA2AAD3ED065A3BEEA8
:10FE10002CBA30EE0EEA79EEADDA24EEA20A67EEE5
:10FE2000A29A27EE229A78EEAE8A7BEE8FBA66EE21
:10FE3000A2EA38EE028A66EE222A25EE031A63EE63
:10FE400083CA67EE030A3BEE0ABA7CEE2AAA3EEEAC
:10FE500000EA24EE83CA27EE830A3DEE099A78EE83
:10FE6000AE8A26EE83DA66EE03EA93ED075A25EEB4
:10FE7000833A7BEEAFBA7DEEA99A38EE228A7BEE0A
:10FE800081BA63EE843A3BEE2CBA7AEE8CAA64EE29
:10FE900084CA27EE84CA3EEE00EA79EEA09A27EEE5
:10FEA000040A66EE840A26EE041A38EE038A39EE56
:10FEB0000D9A25EE843A78EEAE8A25EE044ABBF11F
:10FEC000010B02F120027BEEA3BA3BEE2CBA7AEED4
:10FED0008CAA3EEE00AA79EEA09A39EE019A78EE4D
:10FEE000838A38EE048A03F120037FF4D8AEDDF86C
:10FEF00000B007EB0A02B8F1000F37D043460FE01D
:10FF000000000000F0EE674AF0EE477AB0EE667A45
:10FF1000F0EE466AB0EE656AF0EE455AB0EE635A0E
:10FF2000BBEC014AF2EC013A64EE844A67EE840AC3
:10FF300027EE041A66EE841A26EE042A65EE842A59
:10FF400025EE043A23EE844A013B7BEEA4BA3BEE55
:10FF500020BA7AEE81AA3AEE21AA79EE829A39EE97
:10FF6000229A78EE838A38EE048ACBD10139C5ED26
:10FF700000BA85ED01BAC5ED02AA85ED03AAC5ED6B
:10FF8000049A85ED059AC5ED068A85ED078A07F185
:10FF9000200706F1200605F1200504F120040CF1EC
:10FFA000200C7FF447AE049CDDF818A0DDF81C801F
:10FFB0000899099A63019A44194498441A44039889
:10FFC00010F007071ED0DDF804C03E46454651F844
:10FFD000043B5FED357A4AF8043B4C4663462846BD
:10FFE000F0EC016AB4EC017A26EE877A013B77EEF9
:10FFF000877AF5D1013EE2EC017A05F10405E6D1FC
:020000040801F1
:1000000008EB8708019B029C5D1EAE08606813D058
:1000100042460346314614681C6054685C6094682C
:100020009C60D468DC60013902F1100203F1100316
:10003000F1D133011844984415F0030305D058F862
:10004000042B40F8042B013BF9D10AB0BDEC108B16
:10005000BDE8F00F7047CB464DE700BF2DE9F00F2C
:100060001C469EB0037B4568066880681290A7080E
:100070003801C3F11F0C1792024413910133CCF1E4
:10008000200104F003041D9205F110021B9011954C
:10009000159616971C9310911A941492E2461046E6
:1000A000129B50F8104C5D689E68DF68D3F80080A2
:1000B00004950596D3F810B0119D119B169E0697D6
:1000C000D5F80C905F689B68002E00F0DB8030460E
:1000D000A446139E179D09904C46D146C246DDF8B2
:1000E00070803168049A079181FB0A01C2FB0C0100
:1000F000059AC2FB0701069FC7FB0301CBFB040166
:1001000020FA09F001FA08F404432C607068049F97
:10011000089000220392079A029180FB0A01C7FB14
:100120000201059A069FC2FB0C01C7FB0401CBFB31
:1001300003010A9120FA09F001FA08F10843686006
:10014000B76801900499089800220B9287FB0A2354
:10015000C1FB002307980599C1FB0023019806996C
:10016000C1FB0023CBFB042322FA09F203FA08F4B3
:100170001443AC60D6F80CC00C9300200D9004988A
:1001800008998CFB0A23C0FB07230598C0FB0123B9
:1001900006990198C1FB0423CBFB002300210E9399
:1001A0000F91099922FA09F203FA08F3134301396E
:1001B000EB6006F1100605F11005099191D1139A33
:1001C0001B9D1D9E2A44D0461392CA46A1466446F2
:1001D0001A98002851D0CDF81C80CDF820B009978E
:1001E000984601968446DDF84CB003E0C146099478
:1001F00090462C465BF8045B079E049F85FB060136
:10020000C7FB0401099E059FC7FB0601069E109FC0
:10021000C6FB0801089EC6FB090101FA07F920FA8E
:100220000AF2BAF1200742EA090258BF41FA07F779
:10023000019858BF3A4340F8042BBCF1010C41FA35
:100240000AF301901146D1D1CDE918234346149AFF
:10025000119E42F8105C159F129D7460B160F360AE
:10026000143510321036013F1295149211961597DD
:100270000AD017981390149812E7194625464B4652
:100280003C46E4E7179EA3E71EB0BDE8F00F7047B9
:10029000F0B40C49860DC0F3150051F82640400219
:1002A000C0F100470136A7FB0423E51707FB05371C
:1002B00051F826103B460022C1FB00235800F0BC39
:1002C000704700BFD4F5020800F000B810B5041E56
:1002D00008BF0124204600F085F830B900F016F878
:1002E00008B900F01FF88047F4E710BD064BBFF3D4
:1002F0005B8F024653E8000F43E800210029F9D143
:10030000BFF35B8F704700BF64140120024B186875
:10031000BFF35B8F704700BF6414012000F000B88A
:1003200000F068B808B5062000F0A8FA012000F037
:1003300011FC00BF002301461A46184600F0D6BA49
:1003400008B5074B044613B1002100F01FFB054B15
:100350001868836A03B19847204600F0FBFB00BF92
:100360008D090108F0A9040838B50A4C0A4D641B30
:10037000A4100AD004F18043013B05EB8305013C46
:1003800055F804399847002CF9D1BDE838403AF0C7
:1003900037BB00BF1CAA040818AA040870B50D4E8C
:1003A0000D4D761BB61006D00024013455F8043BE1
:1003B0009847A642F9D1094E094D761B3AF01AFB2F
:1003C000B61006D00024013455F8043B9847A642E5
:1003D000F9D170BD0CAA04080CAA040818AA0408D4
:1003E0000CAA0408024B0146186800F04BB900BF84
:1003F00034090020024B0146186800F0EDB800BF38
:1004000034090020844641EA000313F003036DD150
:10041000403A41D351F8043B40F8043B51F8043BC7
:1004200040F8043B51F8043B40F8043B51F8043BCE
:1004300040F8043B51F8043B40F8043B51F8043BBE
:1004400040F8043B51F8043B40F8043B51F8043BAE
:1004500040F8043B51F8043B40F8043B51F8043B9E
:1004600040F8043B51F8043B40F8043B51F8043B8E
:1004700040F8043B51F8043B40F8043B51F8043B7E
:1004800040F8043B51F8043B40F8043B51F8043B6E
:1004900040F8043B403ABDD2303211D351F8043B0E
:1004A00040F8043B51F8043B40F8043B51F8043B4E
:1004B00040F8043B51F8043B40F8043B103AEDD2BD
:1004C0000C3205D351F8043B40F8043B043AF9D20E
:1004D000043208D0D2071CBF11F8013B00F8013BE1
:1004E00001D30B8803806046704700BF082A13D3EE
:1004F0008B078DD010F003038AD0C3F10403D21A06
:10050000DB071CBF11F8013B00F8013B80D331F839
:10051000023B20F8023B7BE7043AD9D3013A11F8B9
:10052000013B00F8013BF9D20B7803704B78437024
:100530008B78837060467047F0B4860746D0541EAF
:10054000002A3CD0CAB2034602E014F1FF3436D38D
:1005500003F8012B9D07F8D1032C29D9CDB245EA28
:1005600005250F2C45EA054533D9A4F110063609B7
:1005700003F1200707EB061703F1100242E90455C7
:1005800042E902551032BA42F8D1721C14F00C0F35
:1005900003EB021204F00F0613D0331F23F0030302
:1005A0000433134442F8045B9342FBD106F0030486
:1005B0002CB1C9B21C4403F8011B9C42FBD1F0BC16
:1005C000704734461346002CF3D1F8E7144603462F
:1005D000C2E71A462646E0E700293CD038B551F874
:1005E000043C0C1F002BB8BFE418054600F01CFAB1
:1005F000234B1A682AB1A2420DD9216860188242A1
:1006000023D0626028461C60BDE8384000F00EBA76
:10061000A34203D81A465368002BF9D11168501829
:10062000A04219D024D821686018834206D06360A4
:1006300054602846BDE8384000F0F8B9D3E900031B
:100640000144636021605460F3E7D2E90002014491
:1006500062602160D6E770472068014450188342E9
:100660001160E6D1D3E90003014453601160E0E773
:100670000C232B602846BDE8384000F0D7B900BFF6
:10068000BC090020F8B5CD1C25F0030508350C2D5C
:1006900038BF0C25002D064633DBA94231D82A4F3E
:1006A00000F0C2F93A6852B113685B1B04D43FE012
:1006B00023685B1B29D522465468002CF8D1796841
:1006C00000293BD02946304600F040F8431C28D092
:1006D000C41C24F00304A04205D0211A304600F0C7
:1006E00035F801301DD02560304600F09FF904F147
:1006F0000B0020F00700231DC21A01D01B1AA350C3
:10070000F8BD0C2232600020F8BD0B2B05D8A242A8
:10071000636811D05360E7E7144623601C442560EA
:10072000E2E70C233046336000F080F90020F8BD8A
:100730000B2BF1D8536814463B60D5E7304600F0E8
:1007400005F87860BEE700BFBC09002038B5074C4B
:10075000002305460846236000F0EEF9431C00D054
:1007600038BD2368002BFBD02B6038BD68140120F6
:1007700010B580210446FFF785FF606440B1031F78
:1007800000227C3043F8042F8342FBD1002010BDAF
:100790004FF0FF3010BD00BF436C0BB1002070471D
:1007A000E6E700BF1F2970B5054608D8436C16461A
:1007B0000C464BB153F8240043F8246070BD162258
:1007C00002604FF0FF3070BDFFF7D2FF08B96B6CCD
:1007D000F0E74FF0FF3070BD1F2938B521D8426CCB
:1007E00005460C466AB152F8213053B1012B16D0A0
:1007F000591C10D00025204642F82450984728461E
:1008000038BD284600F070F8224601462846BDE86B
:10081000384000F055B816230360012038BD002091
:1008200038BD162303604FF0FF3038BD1F2921D893
:1008300038B5436C05460C4683B153F8242003EBCE
:1008400084034AB1511C10D0012A0CD00025204647
:100850001D609047284638BD012038BDFFF788FF4E
:1008600028B96B6CE9E7032038BD022038BD4FF092
:10087000FF3038BD4FF0FF30704700BF024B0146DC
:100880001868FFF7A9BF00BF34090020024B0A46D1
:1008900001461868FFF786BF34090020034B18682B
:1008A000436C0BB10020704762E700BF34090020A1
:1008B000024B01461868FFF7B9BF00BF340900209A
:1008C00038B50B46074C05461146184600232360F1
:1008D00000F02AF9431C00D038BD2368002BFBD060
:1008E0002B6038BD6814012000F016B92DE9F843DB
:1008F000224C25680DB36C681F2C3BDC9846914652
:100900000F46064688B1D5F8880028B3D0F80031E4
:1009100040F824900122A24000EB84011343022EF0
:10092000C0F80031C1F8808010D0A31C01346C6085
:1009300045F823700020BDE8F883114E114D256065
:10094000002ED8D03468C5F88840D4E7D0F80431F8
:100950001A43C0F80421E8E70B4B5BB14FF48470F5
:10096000FFF740FD30B100236C68C0E94033C5F8A3
:100970008800CDE74FF0FF30DDE700BF500A0020D0
:1009800000000000C4090020E50301082DE9F04F34
:10099000DFF8908083B0D8F8005001900F464FF0F8
:1009A000010A8DB16C68D5F88860013C0CD405F162
:1009B000080B67B12EB106F1800353F82430BB4217
:1009C00005D014F1FF34F4D203B0BDE8F08F6B68AA
:1009D0005BF82420013BA34216BF00236C604BF858
:1009E0002430002AEDD0D5F80490B6B1D6F8001125
:1009F0000AFA04F30B4210D0D6F8040156F824107A
:100A000003420CD1019890476B68D8F800204B4501
:100A100001D1AA42D5D01546C3E79047F4E708466E
:100A20009047F1E7500A0020704700BF704700BFB1
:100A300038B50C460968054609B1FFF7F9FF2146AC
:100A40002846BDE83840FFF7C7BD00BF314B1B68E3
:100A500083425AD0426A70B50546002A50D0D36806
:100A60009BB10026995941B10C682846FFF7B4FDA7
:100A70002146002CF8D16B6ADB680436802EF1D158
:100A800019462846FFF7A8FD6A6A116800293DD07B
:100A90002846FFF7A1FD696911B12846FFF79CFDC3
:100AA0006A6A1AB111462846FFF796FDA96B11B183
:100AB0002846FFF791FDE96B11B12846FFF78CFD41
:100AC000296C11B12846FFF787FDE96D11B1284661
:100AD000FFF782FDA96D11B12846FFF77DFD696B17
:100AE00011B12846FFF778FDAB696BB1AB6A2846B8
:100AF0009847A96C41B12846BDE87040FFF798BF00
:100B000041690029C9D1D1E770BD704769690029E1
:100B1000C3D1C7E734090020024B58221A604FF0B6
:100B2000FF30704768140120024B58221A604FF0C2
:100B3000FF30704768140120044A05491368002BF0
:100B400008BF0B461844106018467047540A00202E
:100B50006C140120FEE700BF0000803F819231C08D
:100B600023A13D400E10B8BFE49D883E3D2C8D3A38
:100B70003F2C8D3B5DC2D33B3F2C8D3B3D2C8D3AB2
:100B80000000891112239B322446AD573665BF748D
:100B9000488CC19D5AAFD3BE6CCAE5DB7EE9F7F83D
:100BA0008110080193331A22A5562C47B7753E646D
:100BB000C99C408DDBBF52AEEDDA64CBFFF976E81D
:100BC00002218B30100299132667AF763444BD554D
:100BD0004AADC3BC588ED19F6EEBE7FA7CC8F5D9FD
:100BE00083310A2091121803A7772E66B5543C452D
:100BF000CBBD42ACD99E508FEFFB66EAFDD874C9DD
:100C000004428D5316619F702004A9153227BB360C
:100C10004CCEC5DF5EEDD7FC6888E1997AABF3BABC
:100C200085520C4397711E60A1142805B3373A26EC
:100C3000CDDE44CFDFFD56ECE9986089FBBB72AA9C
:100C400006638F7214409D512225AB343006B917CC
:100C50004EEFC7FE5CCCD5DD6AA9E3B8788AF19B7C
:100C600087730E6295501C41A3352A24B1163807AC
:100C7000CFFF46EEDDDC54CDEBB962A8F99A708B5C
:100C8000088481951AA793B62CC2A5D33EE1B7F08C
:100C90004008C919522BDB3A644EED5F766DFF7C3C
:100CA000899400859BB712A6ADD224C3BFF136E06C
:100CB000C1184809D33B5A2AE55E6C4FF77D7E6C1C
:100CC0000AA583B4188691972EE3A7F23CC0B5D14C
:100CD0004229CB38500AD91B666FEF7E744CFD5DFC
:100CE0008BB502A499961087AFF326E2BDD034C12C
:100CF000C3394A28D11A580BE77F6E6EF55C7C4DDC
:100D00000CC685D71EE597F42880A1913AA3B3B20B
:100D1000444ACD5B5669DF78600CE91D722FFB3EBB
:100D20008DD604C79FF516E4A9902081BBB332A2EB
:100D3000C55A4C4BD7795E68E11C680DF33F7A2E9B
:100D40000EE787F61CC495D52AA1A3B03882B193CB
:100D5000466BCF7A5448DD59622DEB3C700EF91F7B
:100D60008FF706E69DD414C5ABB122A0B9923083AB
:100D7000C77B4E6AD5585C49E33D6A2CF11E780F5B
:100D80004465636F6465722031207265706F7274A0
:100D90006564004465636F6465722032207265701B
:100DA0006F72746564004465636F646572203320FC
:100DB0007265706F727465640080402010080402D0
:100DC000010102040810204080000000D600AC01A0
:100DD000810253032404F104BC0582064307000882
:100DE000B6086709110AB40A500BE30B6E0CF10C3C
:100DF0006A0DDA0D410E9D0EEF0E370F730FA60F21
:100E0000CD0FE90FF90FFF0FF90FE90FCD0FA60F67
:100E1000730F370FEF0E9D0E410EDA0D6A0DF10CB8
:100E20006E0CE30B500BB40A110A6709B6080008F0
:100E300043078206BC05F104240453038102AC017C
:100E4000D60000002AFF54FE7FFDADFCDCFB0FFB4B
:100E500044FA7EF9BDF801F84AF799F6EFF54CF53A
:100E6000B0F41DF492F30FF396F226F2BFF163F1A2
:100E700011F1C9F08DF05AF033F017F007F001F0DE
:100E800007F017F033F05AF08DF0C9F011F163F16B
:100E9000BFF126F296F20FF392F31DF4B0F44CF585
:100EA000EFF599F64AF701F8BDF87EF944FA0FFB21
:100EB000DCFBADFC7FFD54FE2AFF333AA030005529
:100EC000A65F500755FD7DF75F7001300000900967
:100ED0001001700090000740017000314007400190
:100EE00050A171D1707001100000000E2007F7D5DD
:100EF000DD57DFD001300000900910017000900034
:100F00000740017000314007400150A171D170705D
:100F100001100000000E2000002008080238150013
:100F20002CA01460846DFF57D75DF5DE30300110C2
:100F3000014003C013C11E806F00004F08DC02880F
:100F400015782CD014C084ADFF57D75DF5D9652432
:100F5000022806200F801BC107805C0000200808C3
:100F6000023815002CA01460846D5D7F77FD757EBE
:100F700030300110014003C013C11E806F00CEA8A5
:100F8000FE83ACC458200ACEA8FE83A00000000057
:100F9000000CC458200ACEA8FE83ACC458200A0016
:100FA000004F08DC028815782CD014C084AD5D7F1A
:100FB00077FD75796524022806200F801BC1078004
:100FC0005C9E8D3288261A3F61E8552D1600000080
:100FD000444952454354202044495245435420201B
:100FE00043514351435120204D4D44564D20202024
:100FF00054455354A96A0000BF090A00B5814E0D3B
:101000001F080C002C87160B61060F00DF96B50831
:10101000DF0413001892A6060F04170096438B05F1
:10102000BC0319003842190500777777777777770F
:101030007777777777777777777777777777777740
:101040007777777777777777777777777777777730
:1010500077777777777777777700CDF59D5D7CFA2F
:101060000A6E8A2356E84CAADE8B26E4F28288C6F2
:101070008A7429A4ECD00822CEA2FC018CECDA0AF6
:10108000A0EE8A7E2B26CCF88A0800CDF59D5D7CEB
:101090006DBB0EB3A426A84CAADE8B26E4F2828890
:1010A000C68A7429A4ECD00822CEA2FC018CECDA0A
:1010B0000AA0EE8A7E2B26CCF88A0800CDF59D5D2D
:1010C000763A1B4A81A8E2804CAADE8B26E4F282A3
:1010D00088C68A7429A4ECD00822CEA2FC018CEC2C
:1010E000DA0AA0EE8A7E2B26CCF88A0800CDF59D80
:1010F0005D74288302B02D07E24CAADE8B26E4F251
:101100008288C68A7429A4ECD00822CEA2FC018C65
:10111000ECDA0AA0EE8A7E2B26CCF88A08000000C2
:1011200041000000000000B808000000420000007C
:10113000000080EA0C000000430000000000A0EB6B
:101140000E00000044000000000000EA0A00000059
:101150004500000000000080040000004600000080
:10116000000080AE0C00000047000000000080EE90
:101170000C00000048000000000000AA0A00000067
:1011800049000000000000A0060000004A00000026
:101190000000B8BB100000004B000000000080EB16
:1011A0000C0000004C000000000080BA0C000000A1
:1011B0004D000000000000EE0A0000004E0000009C
:1011C000000000E8080000004F0000000000E0EE12
:1011D0000E000000500000000000A0BB0E00000048
:1011E000510000000000B8EE1000000052000000A6
:1011F000000000BA0A00000053000000000000A830
:101200000800000054000000000000E0060000009C
:1012100055000000000000AE0A000000560000006B
:10122000000080AB0C00000057000000000080BBF5
:101230000C000000580000000000E0EA0E00000072
:10124000590000000000B8EB100000005A00000038
:101250000000A0EE0E000000310000000080BBBBCB
:1012600014000000320000000000EEAE120000008A
:10127000330000000000B8AB100000003400000094
:101280000000E0AA0E00000035000000000080AA67
:101290000C000000360000000000A0EA0E00000074
:1012A000370000000000A8EE100000003800000029
:1012B0000000EAEE12000000390000000080EEEEAF
:1012C000140000003000000000E0EEEE1600000008
:1012D0002F0000000000E8EA100000003F000000BE
:1012E0000000EAAE120000002C00000000E0AEEEAC
:1012F000160000002D0000000000AEEA1200000001
:101300003D0000000000B8EA100000002E000000C0
:101310000080EBBA14000000200000000000000074
:1013200004000000000000000000000000000000B9
:1013300080402010080402014D65737361676520C9
:10134000637265617465642077697468206C656E8A
:101350006774680080402010080402010FFFFFFF3F
:10136000FFFFF00D5D7F77FD757007F7D5DD57DF67
:10137000D0FD030303FD0303FDFDFD03FD03FDFDA0
:10138000FDFD0303FD030303FD03FDFDFD03FDFD63
:10139000030303FD03FD03030303FDFD03FDFDFD47
:1013A00003444D52444D4F52583A206461746120B9
:1013B00068656164657220666F756E6420706F7316
:1013C0002F63656E7472652F7468726573686F6CD5
:1013D0006400444D52444D4F52583A206461746148
:1013E000207061796C6F616420666F756E64207027
:1013F0006F732F63656E7472652F7468726573689E
:101400006F6C6400444D52444D4F52583A20766FF1
:101410006963652068656164657220666F756E64D6
:1014200020706F732F63656E7472652F74687265B8
:1014300073686F6C6400444D52444D4F52583A20CB
:10144000766F6963652070692068656164657220E4
:10145000666F756E6420706F732F63656E7472654E
:101460002F7468726573686F6C6400444D52444D0C
:101470004F52583A20766F696365207465726D69C2
:101480006E61746F7220666F756E6420706F732F5B
:1014900063656E7472652F7468726573686F6C64CF
:1014A00000444D52444D4F52583A206373626B20B2
:1014B000666F756E6420706F732F63656E747265EE
:1014C0002F7468726573686F6C6400444D52444DAC
:1014D0004F52583A20766F6963652073796E6320A6
:1014E000666F756E6420706F732F63656E747265BE
:1014F0002F7468726573686F6C640063EA00766CC1
:1015000076C452C878092DB87927579B31BC3EEA7A
:1015100045C330491793AE8B6DA4A5ADA2F135B587
:101520003C1E80402010080402010FFFFFFFFFFF58
:10153000F00D5D7F77FD7570FD030303FD0303FD73
:10154000FDFD03FD03FDFDFDFD0303FD030303FDA1
:10155000444D5249646C6552583A2064617461206C
:1015600073796E6320666F756E642063656E747246
:10157000652F7468726573686F6C6400804020101A
:10158000080402010FFFFFFFFFFFF00D5D7F77FDF5
:10159000757007F7D5DD57DFD0FD030303FD0303A7
:1015A000FDFDFD03FD03FDFDFDFD0303FD03030341
:1015B000FD03FDFDFD03FDFD030303FD03FD03032B
:1015C0000303FDFD03FDFDFD03444D52536C6F7499
:1015D00052583A20646174612068656164657220C4
:1015E000666F756E6420736C6F742F706F732F63EA
:1015F000656E7472652F7468726573686F6C6400D1
:10160000444D52536C6F7452583A20646174612097
:101610007061796C6F616420666F756E6420736CA5
:101620006F742F706F732F63656E7472652F74689B
:10163000726573686F6C6400444D52536C6F7452E2
:10164000583A20766F696365206865616465722029
:10165000666F756E6420736C6F742F706F732F6379
:10166000656E7472652F7468726573686F6C640060
:10167000444D52536C6F7452583A20766F696365CB
:101680002070692068656164657220666F756E649C
:1016900020736C6F742F706F732F63656E74726537
:1016A0002F7468726573686F6C6400444D52536C9C
:1016B0006F7452583A20766F696365207465726D55
:1016C000696E61746F7220666F756E6420736C6FE3
:1016D000742F706F732F63656E7472652F746872E8
:1016E0006573686F6C6400444D52536C6F7452584C
:1016F0003A206373626B20666F756E6420736C6F43
:10170000742F706F732F63656E7472652F746872B7
:101710006573686F6C6400444D52536C6F7452581B
:101720003A20766F6963652073796E6320666F7502
:101730006E6420736C6F742F706F732F63656E749B
:1017400072652F7468726573686F6C6400000000C6
:101750000000000001000000020000000300000083
:101760000400000005000000060000000700000063
:1017700008000000090000000A0000000B00000043
:101780000C0000000D0000000E00000020400200D0
:101790001000000011000000120000001300000003
:1017A00014000000150000001600000017000000E3
:1017B00018000000190000001A0000001B000000C3
:1017C0001C0000001D000000408004008014000088
:1017D0002000000021000000220000002300000083
:1017E0002400000025000000260000000840020040
:1017F00028000000290000002A0000000440020028
:101800002C000000024002000140020000400200E3
:101810003000000031000000320000008081000034
:1018200034000000400C000036000000420C0000B4
:1018300038000000003004003A00000002300400CC
:10184000022900001240020000290000104002009E
:101850004000000041000000420000004300000082
:101860004400000045000000460000004700000062
:1018700048000000490000004A0000000025000068
:101880004C0000004D000000108004001180040096
:101890005000000051000000520000000012020041
:1018A00054000000200C000008800400098004009F
:1018B0005800000059000000048004000580040066
:1018C0000280040003800400008004000180040002
:1018D0006000000061000000620000006300000082
:1018E00064000000100C00000003010000B00000C4
:1018F00068000000690000008018000081180000E6
:1019000081010400800104004140020040400200C7
:1019100070000000040C000072000000060C0000C3
:10192000010C0000000C0000030C0000020C000081
:10193000045200000C0C00002480040025800400E8
:1019400000520000080C00002080040021800400E8
:101950008000000081000000820000008300000081
:101960008400000085000000860000008700000061
:1019700088000000890000008A00000000020500C5
:101980008C00000000A800001114000010140000DA
:1019900090000000910000009200000020810000F3
:1019A0009400000095000000004A000008140000A8
:1019B00098000000990000000514000004140000C5
:1019C00003140000021400000114000000140000C1
:1019D000A0000000A1000000A20000001081000093
:1019E000A4000000A500000000240400012404005D
:1019F000A8000000A90000004018000041180000E5
:101A000041010400400104008140020080400200C6
:101A1000B000000002810000018100000081000090
:101A2000B400000006810000058100000481000070
:101A3000010A0200000A020009810000088100007A
:101A400023140000221400002114000020140000C0
:101A5000C0000000C1000000C2000000C300000080
:101A6000C4000000C5000000C6000000C700000060
:101A7000C8000000C9000000201800002118000064
:101A80000006020020010400006001000160010066
:101A9000D0000000D100000001280400002804004C
:101AA00000310000008201000231000002820100CA
:101AB000D8000000D9000000848004004414000015
:101AC0008280040042140000808004004014000062
:101AD000E00000000020030008180000004600009D
:101AE00009010400080104000C1800000A010400A8
:101AF0000218000004010400001800000118000092
:101B000001010400000104000418000002010400A7
:101B100008A40000428100004181000040810000D3
:101B2000810C0000800C0000830C0000820C00007F
:101B300000A4000001A4000010180000111800000B
:101B40001101040010010400141800001201040027
:101B5000000100000101000002010000030100007B
:101B60000401000005010000060100000018040047
:101B700008010000090100000A01000040240000E3
:101B80000C0100000D0100000E01000044240000C3
:101B9000100100001101000012010000A0800000EF
:101BA000140100001501000016010000A4800000CF
:101BB000180100001901000000500100015001004F
:101BC00022280000232800002028000021280000EF
:101BD000200100002101000022010000908000008F
:101BE0002401000025010000400201004102010023
:101BF00028010000290100002A0100000441020020
